:020000040000FA
:040000006FD00400B9
:101000006F00907E00000000000000009020002093
:10101000AA220020A9BDF9F56C23002000000000E1
:10102000000000006C230020902000200000000041
:101030000000000090200020000000009020002010
:101040000000000090200020902000209020002030
:101050009020002090200020582F00209424002071
:101060000000000090200020902000201E2400207E
:1010700090200020D22300209020002090200020EB
:101080009020002090200020902000209020002020
:101090009020002001A04111B7170040985F3AC688
:1010A000945F3247E39CE6FE3245410182800111A4
:1010B00013078008F337078093F787083EC20100C3
:1010C0000100B7170040930570052380B70413068D
:1010D00080FA2380C7040100010083C6B70493F699
:1010E000F60DA385D704238007049246F3A6068055
:1010F0000100010093760502D5CEF336078093F602
:10110000860836C4010001002380B7042380C70489
:1011100001000100B70614007D89558D88C70100C4
:1011200001000100010023800704A246F3A6068007
:101130000100010073370780137787083AC6010062
:1011400001002380B7042380C704010001000100CF
:1011500001003727004093061005A303D7802380A2
:101160000704B247F3A70780010001009307800836
:10117000F3B7078093F787083ECE01000100B71749
:101180000040130770052380E704130780FA2380CB
:10119000E7040100010003C7B70413670708A3852C
:1011A000E70423800704F247F3A70780010001004A
:1011B0000561828093760504BDC6F336078093F6F9
:1011C000860836C8010001002380B7042380C704C5
:1011D00001000100B7061400938606047D89558D31
:1011E00088C7010001000100010023800704C246F6
:1011F000F3A6068001000100733707801377870884
:101200003ACA010001002380B7042380C70401000B
:1012100001003727004093062005A303D7802380D1
:101220000704D24781B773370780137787083ACC12
:10123000010001002380B7042380C70401000100DE
:1012400098471367070C98C723800704E24719BF24
:101250000111814601468145114506CE97000000E7
:10126000E780605893078008F3B7078093F78708F3
:101270003EC601000100B717004013077005238028
:10128000E704130780FA2380E7040100010003C785
:101290006704136717002383E70423800704B2471A
:1012A000F3A7078001000100F2400561828041112F
:1012B000814601468145114597000000E780A05214
:1012C00013078008F337078093F787083EC40100AF
:1012D0000100B7170040130670052380C70493066A
:1012E00080FA2380D70401000100FD552396B70240
:1012F00023800704A245F3A5058001000100733790
:101300000780137787083AC6010001002380C704CD
:101310002380D7040100010003C767041367170087
:101320002383E70423800704B247F3A70780010063
:10133000010001A0BD473305F50201007D1575FDD3
:101340008280411122C426C206C6AA8401446317C2
:101350009400B24022449244410182800504130566
:10136000803E420497000000E78000FD4180C5B741
:101370009305000273A04580824573901534924016
:101380002242B2424243D2436244F2440255925551
:101390002256B2564257D2576258F25806499649D9
:1013A000264AB64A464BD64B664CF64C065D965DD1
:1013B000265EB65E465FD65F09617300203041113C
:1013C000B7170040985F3AC6945F3247E39CE6FE49
:1013D000324541018280B71700401307000323887C
:1013E000E702854717170000232EF74673002030C9
:1013F000411122C42D6426C24AC006C637190040D6
:101400001304A4AAB704002023208900977000E0E9
:10141000E78060939C408297977000E0E780A092FD
:10142000E5B737370040834747009146BD8B639E41
:10143000D702B73600401306F00F973500009385AA
:10144000651E9737000083D7E72D03C7A6001377E3
:10145000F70F1DE3B7E70400BC4F09468945171590
:1014600000000345A5F7829731A099466394D70001
:10147000834757007300203003C786001377F70FA8
:10148000E365F6FC13851700AE9717380000231BA1
:10149000A8282380E70075B7B787004003C7670017
:1014A000098B6309071003C77700930600031377BE
:1014B0000703630DD708173800000348F87717367D
:1014C0000000130666740547B30606012380E60094
:1014D00083C577001737000013070775429793F508
:1014E000F50F2300B70003C58700973500009385EB
:1014F000A572C2951375F50F2380A5000347070059
:1015000089451377F703630CB70C63E7E50A6306B5
:10151000071A8545630CB7129737000083C7D77148
:101520003307F600034707001377F70F19CB85073A
:1015300093F7F70F3D476363F71A17370000A30DC2
:10154000F76EB787004009472383E700B78700405D
:1015500083C77700E207E18763DE0704973700005F
:1015600083C7976D173700001307076A3E978546B4
:101570002300D700173700001307076B3E97930629
:1015800000032300D700173700001307E7683E97D2
:10159000A14685072300D70093F7F70F3D47636403
:1015A000F71417370000A309F768B7870040094709
:1015B0002383E70073002030930610026300D70EE8
:1015C000930620026305D70693060002E316D7F4BC
:1015D00003C727021377C70F13672700D5A803C7D0
:1015E00067001377070465CB03C7A702173800000D
:1015F00013080843173500001305453A1347070839
:101600002385E70203C7A7021377370F1367870005
:101610002385E702814713070004B305F5008C41D9
:10162000B306F80091078CC2E399E7FEF5B503C74E
:10163000A702134707042385E70203C7A70213770E
:10164000C70F136727002385E702F9B503C76700B3
:101650001377070449C303C767021738000013084C
:10166000E82F1735000013052527134707082383A4
:10167000E70203C767021377370F136787002383D7
:10168000E702814713070004B305F5008C41B30658
:10169000F80091078CC2E399E7FEBDBD03C767025E
:1016A000134707042383E70203C767021377C70FB3
:1016B000136727002383E70285B503C76700137705
:1016C000070411CB03C727021377370F136787006F
:1016D0002381E70291B5238006003DBD97370000C6
:1016E000A38C0754B9BD97370000A387075475BD75
:1016F0002303048015472303E48001002302A48010
:10170000828083076480E3CE07FE23030480828007
:1017100083076480E3CE07FE03454480828083070D
:101720006480E3CE07FE2302A4808280411126C498
:101730004AC24EC006C61377F50BAD47AA892E895B
:101740009544630CF700194597000000E78080FA84
:1017500097000000E78020FB8D444E859700000035
:10176000E78040F9FD59FD1463983401B240A2446A
:101770001249824941018280135509011375F50F01
:1017800097000000E780E0F92209F1BF011126CCA3
:1017900006CEB704080097000000E780C0F61545A4
:1017A00097000000E78000F597000000E78080F6D2
:1017B00097000000E78000F62AC697000000E78047
:1017C00080F432459377150089EB13651500137586
:1017D000F50FF240E24405618280FD14E9F0014515
:1017E000CDBF397126DC4ADA4ED852D656D45AD2F9
:1017F0005ED006DE62CE66CCB7E700E07D5783AAF6
:10180000070022C603AA470023A0E71823A2E7186F
:10181000B7170040130770052380E704130780FA09
:101820002380E70483C74704930B75FFB684E20760
:1018300093FBFB0F8546AA892E8B32893724004003
:10184000E187015763FA76016308D50089461307DB
:1018500000026313D5000157D98F93F7F70FB71C18
:1018600000402382FC0411472303E4801305F00F9A
:1018700097000000E78000E8094C97000000E7802F
:1018800080E863657C15B7050700DA9537870700A0
:10189000795563FEE504B3879500636AF704370B57
:1018A0000800A94733EB65016395F90881E8814495
:1018B00097000000E78020E5268515A8DA85094510
:1018C00097000000E780C0E605090345F9FFFD1415
:1018D000050B97000000E780C0E481C49377FB0FFD
:1018E000E5F797000000E780A0EA69F17D55B7179A
:1018F0000040130770052380E704130780FA238054
:10190000E70403C74704418B2382E704F250B7E79B
:1019100000E023A0571123A24711E2543244525948
:10192000C259325AA25A125B825B724CE24C21615C
:101930008280A547639BF90685691309F00FB306FA
:101940009900B3742B01B6941349F9FFB37499004D
:10195000856B33796901416B9387F9FFB3F72701F1
:1019600099E363FC340193D94900C147E3E637FFAB
:101970003DBF0569C1697D19D9B71305800D63881D
:101980006901130500026384790113051008CA85F3
:1019900097000000E780C0D997000000E78040DF93
:1019A00031D54E99B38434416DBFDA852D4597000A
:1019B0000000E780E0D7CA94E30B99EE0509970091
:1019C0000000E78020D5A30FA9FEFDB79387F9FF9C
:1019D00093F7F70F636DFC0C83C71C0413073008E3
:1019E0006315F706370708006361EB06B3079B0032
:1019F000B706100063FBD704334BEB0089476399AC
:101A0000F9068980D549E38404EADA850945970017
:101A10000000E780E0D111090327C9FF9147232087
:101A2000E48003076480E34E07FE23033481FD173F
:101A3000EDFBFD14110B81C49377FB0FE9FF9700B9
:101A40000000E780E0D461F155B5B717004003C747
:101A50005704B70708001377070219E3B787070091
:101A60007955E376FBE833079B00E3F9E7F841B5E6
:101A70008547E380F9F0DA852D4597000000E7807F
:101A800020CB9389F4FFE38404E297000000E78011
:101A900060C893F7390091EB83260480032709007F
:101AA00093074900E396E6E03E89CE84D9BFB54767
:101AB0006399F9001305900B97000000E78080C33D
:101AC000FDB3B1471305B00AE388F9FE9947639760
:101AD000F904B7050800B365BB002D459700000069
:101AE000E78000C581448D4BA14997000000E78045
:101AF00060C263967401832704802320F900850463
:101B0000E39534FF8327048013172B0163550700E7
:101B10002312F90069BB2322F90051BB9D47639F43
:101B2000F90281451305B00497000000E78040C02A
:101B3000BD442320090023220900FD59970000001D
:101B4000E78040BD93F77400CA9703C70700FD14F0
:101B5000398D2380A700E39334FF91BBA14763979E
:101B6000F90697000000E780A0C28144630D0B00D6
:101B70008D479304C0036308FB00930400056304CE
:101B80008B01930440041375C507E30295D21945F0
:101B900097000000E78000B697000000E780A0B63D
:101BA000054597000000E780E0B426859700000017
:101BB000E78020B7094597000000E78080B69700CE
:101BC0000000E780E0BCE31405CE0DB39147639FAE
:101BD000F9001305600697000000E780A0B19700A8
:101BE0000000E78040B213059009F9B5E38109CC04
:101BF000F1547DB9BD660147173600001306063063
:101C0000938606A685458347060093F7F70F91C391
:101C100082800507E3F9E6FE973700002380B72EA0
:101C2000DDB77D166206618693178601E18763D46E
:101C3000070001458280931726003307F500AE9711
:101C400018439C4363E7E7007D16E37FF7FC7D556F
:101C5000828005458280FD15E205E18513978501A7
:101C6000618793F7F50F63480700FD15139725006B
:101C70002A97584365D713851700620561858280CE
:101C80003308B5021C4283A80600B335B502C297DB
:101C900033B50701AE98469585486367B5006394F0
:101CA000A50063E3070181480C43C6950CC388C2B5
:101CB0001CC2828081471397870161876343B70005
:101CC0008280139727002A97232007008507E5B70E
:101CD0008147014793968701E18663C5B6001335B6
:101CE0001700828093962700AA9694428507558F05
:101CF000D5B793D755408A07AA979C430545331516
:101D0000B5007D8D828017F3FFDFE702833D2A84D3
:101D100097000000E78060F405C5931725003E9406
:101D20000327C4FF814711EB7D1516053E9542053B
:101D3000418517F3FFDF6700033D05838507E5B79E
:101D40000145C5BF81471397870161876343C7007A
:101D5000828013972700B386E50094422A9785076F
:101D600014C3D5B77D1662066186014793178601B5
:101D7000E18763D50700133517008280931726008B
:101D8000B306F500AE9794429C437D16B58F5D8FE8
:101D9000F1BF8A05AA9501476363B500828083A6D7
:101DA000C5FFF11593D71600D98F9CC11397F60183
:101DB000E5B72A830148014701456343D700828084
:101DC000B387050183A80700B30706019C43C697A4
:101DD000AA976384F80033B517010507B308030118
:101DE000620723A0F80061871108C1BF2A83014759
:101DF0008147014563C3D70082803388E50083288B
:101E00000800330EE600032E0E003388A840330886
:101E1000C8416384080133B508018507B308E300AE
:101E2000E20723A00801E1871107E9B717F3FFDFF5
:101E3000E702232B0111B286B2842E86AA850A8579
:101E400097000000E780C0FA2A84A6850A859700DB
:101E50000000E78020E833348000060413351500C5
:101E6000018D056117F3FFDF6700E32917F3FFDF3B
:101E7000E702A3244111AA89AE8A328BB68402C23A
:101E800002C402C60144131C8401135C8C416349E3
:101E90009C02939B1400FD1B0549138CF4FFF15C1D
:101EA00033048901620461846340740792478E049D
:101EB000CE9423AEF4FE410117F3FFDF67006323E6
:101EC00013192400B30B2B01014A93172A00D6974C
:101ED00083A50B0088437800340050009700000071
:101EE000E78040DA050A93178A01E187F11BE35E78
:101EF000FCFC92474E9905042320F900A2473EC2FC
:101F0000B24702C63EC441B7131A8901135A8A4127
:101F1000131D240093178A01E18763CF970092472E
:101F20000A044E941CC0A24705091379F90F3EC25A
:101F3000B24702C63EC4ADB7B3079A0313152A00D1
:101F400056950841780034005000050AEA97DA9760
:101F50008C4397000000E780E0D26DBF197106C284
:101F600012C416C61AC81ECA22CC26CE2AD02ED219
:101F700032D436D63AD83EDA42DC46DECAC0CEC2C9
:101F8000D2C4D6C6DAC8DECAE2CCE6CEEAD0EED2F9
:101F9000F2D4F6D6FAD8FEDA971500009385058CB0
:101FA0008841E700050092402242B2424243D243B8
:101FB0006244F244025592552256B2564257D257C5
:101FC0006258F25806499649264AB64A464BD64BBD
:101FD000664CF64C065D965D265EB65E465FD65F45
:101FE0000961730020300000972100209381810156
:101FF000175100201301018117F5FFFF1305C500DC
:102000009705002093850500171600201306C6FDCE
:1020100063FAC5008322050023A055001105910530
:10202000E3EAC5FE17050200130545539715002086
:102030009385C5FB171600201306C66563FAC50015
:102040008322050023A0550011059105E3EAC5FE92
:102050001715002013050564974500209385053664
:102060006377B500232005001105E36DB5FEFD4241
:10207000739002BC8D4273904280B722000093821D
:10208000828873900230970200209382A2F793E235
:1020900032007390523097520000938202A57390E1
:1020A00012346FB0F47573002030397101436EC67D
:1020B00019A0397141536AC866CA62CC5ECE19A0B4
:1020C000397101535AD056D252D44ED64AD826DA54
:1020D00022DC06DE33016140828241114AC026C201
:1020E00022C406C68282B24D4101024D924C224C5E
:1020F000B24B4101024B924A224AB2494101024984
:1021000092442244B240410182803D432A87637356
:10211000C3029377F700BDEFADE5937606FF3D8AE6
:10212000BA960CC34CC30CC74CC74107E36BD7FE30
:1021300011E28280B306C3408A0697020000969699
:102140006780A6002307B700A306B7002306B700E1
:10215000A305B7002305B700A304B7002304B70005
:10216000A303B7002303B700A302B7002302B700FD
:10217000A301B7002301B700A300B7002300B700F5
:10218000828093F5F50F93968500D58D9396050182
:10219000D58D61B7939627009702000096968682A8
:1021A000E78086FA9680C1171D8F3E96E374C3F8C8
:1021B000A5B73367B500FD530D8B79E7B7877F7FF0
:1021C0009387F7F710419441B372F6003363F6003A
:1021D000BE92B3E262006397720C6318D606504158
:1021E000D441B372F6003363F600BE92B3E26200EC
:1021F0006398720A631BD60410459445B372F600C7
:102200003363F600BE92B3E262006391720A631E0A
:10221000D6025045D445B372F6003363F600BE9241
:10222000B3E26200639A72086311D60210499449BE
:10223000B372F6003363F600BE92B3E262006393BA
:1022400072085105D105E30FD6F6131706019397CF
:102250000601631CF7001357060193D706013305E7
:10226000F7409375F50F91E982804183C18333056F
:10227000F7409375F50F91E182801377F70F93F78D
:10228000F70F3305F74082800346050083C605003B
:10229000050585056313D60065FA3305D6408280AF
:1022A00011059105E312D6FE014582802105A105A5
:1022B000E31CD6FC014582803105B105E316D6FC4E
:1022C000014582804105C105E310D6FC01458280AD
:1022D000B717004003C777051377E70FA38BE70411
:1022E000130700F8A38DE7043D47238CE704130789
:1022F0005003A38CE70403C7A7051377D70F238DDB
:10230000E7048280B717004003C7E7020D89411137
:102310001377C70F498F93068008F3B6068093F6AC
:10232000860836C601000100930670052380D70495
:10233000930680FA2380D704010001002387E70277
:1023400023800704B247F3A7078001000100410181
:10235000828041112A83014E930E407E130F001993
:10236000930F400663E56E129308001913034006AD
:10237000B3781503854E0D4FA14F337365020D8958
:102380001335150063EFBE121308F6FF79467298F5
:102390004208135808013307C70213D61700BE07B7
:1023A00032976146B3F6C60213068070B386C60242
:1023B0003697A166F58F42075D8FB716004083C739
:1023C000F60293F70708A303F1000346710083C7E1
:1023D000F60293F70708E394C7FE83477100B71628
:1023E000004093F7F70F6388071293078008F3B74D
:1023F000078093F787083EC401000100B71700402B
:10240000930670052380D704930680FA2380D704AF
:102410000100010023AA070383C6170393E60608F9
:10242000A388D70223800704A247F3A707800100EF
:1024300001001166B71700407D16D45BC85F938515
:102440004703A98EF18EF5FA93068008F3B606804D
:1024500093F6860836C601000100930670052380B6
:10246000D704930680FA2380D7040100010098C1A5
:1024700003C7170313670704A388E7022380070431
:10248000B247F3A7078001000100410182807D135C
:102490003368E3039308E016630E08003368F30320
:1024A0009308D016630808009378330093B8180097
:1024B0009388D81633081E01131E0801135E0E01FF
:1024C00055B56393E5030548638608000148630337
:1024D00003002A8871087298FD15131E0801C205B1
:1024E000135E0E01C18179BD13F8150063F4BF00BE
:1024F0007908D5B713381800E5BF83C7F60293F7FC
:102500000708A303F1000346710083C7F60293F79F
:102510000708E394C7FE8347710093F7F70FF1DFD5
:10252000E9B531714AD966CB06DF22DD26DB4ED70D
:1025300052D556D35AD15ECF62CD6AC96EC7AA8C26
:1025400002D897100000E78020B12A8993078008FD
:10255000F3B7078093F787083EDA01000100B71749
:102560000040130770052380E704130780FA2380D7
:10257000E7040100010003C7F7021377770FA38771
:10258000E70203C7F70213678700A387E7022380E8
:102590000704D257F3A70780010001000545970003
:1025A0000000E78060D6130780C13347E902116A53
:1025B00093070AE893065002BD69930BA004814A71
:1025C000014B13048008930470057D1AB347F90288
:1025D0003307D7023EC0FD873ECC938709A69309F7
:1025E000803E3347F7023AC27D873AC43347390306
:1025F0008549B399990193D93940B306D702B30BF2
:102600007703B3C6F602B3CBFB0236C6FD8636C8E7
:1026100093D6FB4136CEB7460F0093860624334946
:10262000D9028566938606FAB3969601B389E902C4
:10263000130760553309D90293060010B389E902E4
:102640003349D902B3C9F9029316390036CA37198A
:102650000040FD8636D0930D090493D7F9413ED250
:10266000F336048093F6860836DC010001009307F8
:1026700070052380FD00930680FA2380DD000100B1
:1026800001008346390593F6860FA309D9048346D2
:10269000390593E61600A309D90423800D00E256FC
:1026A000F3A6068001000100130C80FA116DF336C9
:1026B000048093F6860836DE01000100930770055A
:1026C0002380FD0023808D01010001008346390530
:1026D000216693E60602A309D90483560905B3E6E9
:1026E000A6012318D90483560905D18E2318D904CD
:1026F00023800D00F256F3A60680010001008346F8
:10270000390593F606026381061A03463905218AC4
:102710006DDE081897100000E7800098733604807B
:1027200013768608B2C20100010023809D00238039
:102730008D0101000100B717004003C6370513766D
:10274000F60DA389C70403C6370513660602A389DD
:10275000C704835609052166B3E6A6012318D904E8
:1027600083560905D18E2318D90423800D0096467F
:10277000F3A60680010001008346390593F60602A0
:10278000638B061483463905A18AEDFE970000206D
:10279000E7806090AA8636D497000020E780A08F5B
:1027A000A256E30AD5FE835609054255B3E6A601B3
:1027B0002318D90497100000E780C08F834639059D
:1027C000A18AEDDE03560905834629058247337643
:1027D000CA00B306DA0293D5F641B296B388F64042
:1027E000E24733B8C6002E983308F840A247B3B684
:1027F00016013308D84063C70701631DF8009247EC
:1028000063FA1701C247634FF80E63950701B24799
:1028100063EAF80E894663E9660FF24693151800DD
:1028200013D3F8015E8613951800B365B30042D642
:1028300046D497C00100E780C0323258050B137BA5
:10284000FB0F63470001631A0838A25863870838F2
:1028500013081500B336A800B69513D6F5013298C3
:10286000B336C800AE9613581800FE06B3E606014C
:102870007336048013768608B2C6010001002380F7
:102880009D0023808D01010001000356C902B2960C
:10289000C206C1822316D90223800D00B646F3A6D4
:1028A00006800100010021B5F336048093F6860806
:1028B000B6C00100010023809D0023808D0101002E
:1028C00001008346390593E60602A309D904238053
:1028D0000D0086460DB5F336048093F68608B6C41F
:1028E0000100010023809D0023808D010100010073
:1028F0008346390593E60602A309D90423800D0017
:10290000A646BDB5E30B0BF0F336048093F68608BC
:10291000B6C801000100930680FA23809D00238041
:10292000DD00010001008346390593F5FC0F93F6A5
:10293000860FA309D90483463905CD8EA309D9048E
:1029400023800D00C646F3A6068001000100130592
:1029500080FA03463905930639051D8A631C9629BA
:102960007336048013768608B2CC0100010013068A
:1029700080FA23809D002380CD000100010003C662
:1029800006001376F60D2380C60003C60600136604
:1029900006022380C600835609051166D18E2318CE
:1029A000D904835609052166D18E2318D9042380C2
:1029B0000D00E646F3A6068001000100130680FA2A
:1029C0008346390593F60602638006268346390559
:1029D000130C3905A18AFDDA081897000000E7807A
:1029E000A06BF336048093F68608B6D00100010090
:1029F000930680FA23809D002380DD000100010002
:102A000083460C00116693F6F60D2300DC00834626
:102A10000C0093E606022300DC0083560905D18EE4
:102A20002318D904835609052166D18E2318D904A9
:102A300023800D008656F3A60680010001001306D0
:102A400080FA8346390593F60602638A0620834698
:102A50003905A18AEDFE97F0FF1FE780C0632A8C3D
:102A600097F0FF1FE7802063E30C85FF835609057D
:102A700011664255D18E2318D90497000000E780D3
:102A800060638346390513063905A18AFDDAF336FA
:102A9000048093F68608B6D401000100930680FAFC
:102AA00023809D002380DD00010001008346060095
:102AB00093F6F60D2300D60023800D00A656F3A64C
:102AC0000680010001008356090503462905D24707
:102AD000B376DA003306CA021305800C9355F6412B
:102AE0003696330DF6408257333CD6002E9C333653
:102AF000A601330CFC40330CCC40330885039256BE
:102B00004E86B335A5033305A503C29597C00100D2
:102B1000E780200563468001631E0C16630C0D16CA
:102B2000130615003335A6002E959356F5013696FB
:102B3000B335D600AA959396F50105828585D18E89
:102B40006346B000639D051A638B061A0356C902DB
:102B500015823305D6003336C500B2956348B00000
:102B6000639105241306F00F637DA622894663F363
:102B7000561593078008F3B7078093F78708BED6EA
:102B80000100010037170040930770052300F70488
:102B9000930780FA2300F704010001008356C7025F
:102BA00089678117D58FC207C1832316F7022300D7
:102BB0000704B657F3A7078001000100FA506A54D2
:102BC000DA544A59BA592A5A9A5A0A5BFA4B6A4C49
:102BD000DA4C4A4DBA4D296182801308F5FF33352E
:102BE000A800FD152E951356F5013298B336C8008E
:102BF000AA9695B9F336048093F68608B6CA010002
:102C0000010023809D002380AD0001000100834668
:102C10003905CD8EA309D90423800D00D646F3A62D
:102C200006800100010035B3F336048093F6860870
:102C3000B6CE0100010023809D002380CD0001005D
:102C400001008346390593E60602A309D9042380CF
:102C50000D00F646F3A606800100010095B3F33699
:102C6000048093F68608B6D20100010023809D00FF
:102C70002380CD00010001008346390593E606025A
:102C8000A309D90423800D009656F3A606800100FF
:102C9000010045BB9306F5FF33B5A600FD152E9543
:102CA0009355F501AE96B3B5B600AA951396F50106
:102CB000858269B5F336048093F68608B6D801009C
:102CC0000100930680FA23809D002380DD0001002F
:102CD00001008356C9020566011693F6F60FD18EE0
:102CE000C206C1822316D90223800D00C656F3A660
:102CF000068001000100850A93FAFA0F95B233E6C7
:102D0000B60045C20356C9023305D0403338A0008F
:102D1000B305B040B385054115826345B000D1E1EC
:102D20006371A608894663F0560593078008F3B7D8
:102D3000078093F78708BEDA01000100B71700404B
:102D4000130770052380E704130780FA2380E70444
:102D50000100010003D7C7027D8B2396E702238081
:102D60000704D65781BDF336048093F68608B6DC97
:102D700001000100930680FA23809D002380DD007E
:102D8000010001008356C9020566011693F6F60F8D
:102D9000D18EC206C1822316D90223800D00E656C9
:102DA000B9B793078008F3B7078093F78708BEDEAB
:102DB0000100010037170040930770052300F70456
:102DC000930780FA2300F704010001000356C702AD
:102DD00093975600B297C207C1832316F7022300C8
:102DE0000704F657C1BB914763EEB70217D701003E
:102DF000130787758A05BA959C41BA978287B717DA
:102E0000004003A7470B1345F5FF698F23AAE70A84
:102E100003A7070B698F23A8E70A03A7070A798D81
:102E200023A0A70A8280B717004083A6470B134749
:102E3000F5FFF98E23AAD70A83A6070B558D23A881
:102E4000A70A83A6070A758F23A0E70A8280B7170F
:102E5000004003A7470B498F23AAE70A03A7070BE4
:102E60001345F5FF45BFB717004083A6470B13472F
:102E7000F5FF758F23AAE70A03A7070A598D4DB7F7
:102E8000B717004003A7470B498FEDB7914763EE93
:102E9000B70217D701001307676C8A05BA959C41E2
:102EA000BA978287B717004003A7470D1345F5FF70
:102EB000698F23AAE70C03A7070D698F23A8E70CE6
:102EC00003A7070C798D23A0A70C8280B7170040B9
:102ED00083A6470D1347F5FFF98E23AAD70C83A6C7
:102EE000070D558D23A8A70C83A6070C758F23A06B
:102EF000E70C8280B717004003A7470D498F23AA2C
:102F0000E70C03A7070D1345F5FF45BFB7170040B2
:102F100083A6470D1347F5FF758F23AAE70C03A778
:102F2000070C598D4DB7B717004003A7470D498FC0
:102F3000EDB7797122D43714004026D24AD0035914
:102F400024028354040206D64209C2044ECE52CC57
:102F500056CA13590901C1802DE11379F9F793F489
:102F6000F49F4209C20413590901C18093078008E4
:102F7000F3B7078093F787083EC401000100930769
:102F800070052300F404930780FA2300F404010081
:102F90000100231124032310940223000404A247F8
:102FA000F3A7078001000100B25022549254025945
:102FB000F249624AD24A45618280B7F507008146EC
:102FC0003000B105194597000020E7808081A247B5
:102FD00013972701E34A07FC1369090893E40440A7
:102FE00093098008F3B7098093F787083EC0010072
:102FF0000100930A700523005405130A80FA230088
:10300000440501000100231124032310940223002E
:1030100004048247F3A7078001000100294597F0C7
:10302000FF1FE7802031F3B9098093F989084EC268
:1030300001000100230054052300440501000100A4
:103040008357040293E707202310F40223000404AB
:103050009247B9B7B7170040884742054181937737
:10306000050491EB9377F5013755E80113050580C9
:103070003345F50282809377050C130700046397AC
:10308000E7009377F50137459C1CCDB72165130503
:1030900005D0828037E700E01C435443A183E20659
:1030A000D58F1CC1FD572320F7182322F7188280E3
:1030B00013178500B7E700E023A0E710618123A282
:1030C000A7108280B7F700E08847CC47828081470D
:1030D00037370040A14663C4C7003285828003456C
:1030E000B740E38EA6FE3385F5000345050085074E
:1030F0002304A740CDB797070020938727EF9C4371
:10310000173700201307872B3E95636EE5001737AE
:1031100000201307273F6368A70017070020232715
:10312000A7EC3E858280FD57EDBF8280411122C40D
:1031300006C62A8497000000E78000F22947B307FB
:10314000E502B2408D83B3D7870222449507B3D7F7
:10315000E70237370040C207C1832316F700410159
:103160008280411137150E0006C697000000E780E7
:1031700020FCB7370040130770F82381E7000D47A4
:10318000A381E70013070004A380E7000547238716
:10319000E700B24041018280373700408347270073
:1031A0001A0593F7F703C98F93F7F70F2301F70079
:1031B0008280B737004003C7170019C9D98DA38093
:1031C000B70003C70700136787002380E7008280EA
:1031D00093C5F5FFF98DA380B7008280AE872A875B
:1031E000B736004021463738004089E71703000012
:1031F0006700E3F383C8B600E30916FF05078348B9
:10320000F7FFFD17C20723041801C183F9BF41115D
:1032100022C406C62A8497000000E780E0E329471D
:10322000B307E502B2408D83B3D7870222449507E6
:10323000B3D7E70237370040C207C1832316F740F0
:1032400041018280716541111305052006C6970072
:103250000000E78000FCB7370040130770F82381B7
:10326000E7400D47A381E74013070004A380E74030
:1032700005472387E740B24041018280CC4141119C
:1032800006C6328503C6150083C5050022064D8E8D
:1032900042068D654186138875A2630C0611634B47
:1032A000C804138845A26300060D634AC8009385CD
:1032B00035A26301B6082390060029464DA0138865
:1032C00055A26305060D938565A2E316B6FE8D45EE
:1032D0001D4663E6E5081146198E63F3C7003E8676
:1032E000B7E704002390C600FC4797D501009385FB
:1032F00025299DA0138895A263030611634E060D30
:103300001388A5A263000613938505A5E315B6FAF5
:1033100099451D4663E5E504198E63F3C7003E86B3
:10332000B7E704002390C600FC479705002093856B
:1033300025D61DA09D451D4663E3E5022146198E55
:1033400063F3C7003E86B7E70400FC472390C6003E
:103350009705002093858534BA9582970146B2403F
:10336000328541018280AD451D46E3EAE5FE3146E6
:10337000198E63F3C7003E86B7E704002390C600AA
:10338000FC4797D5010093852522F9B7B1451D4625
:10339000E3E7E5FC3546198E63F3C7003E86B7E7E1
:1033A00004002390C600FC4797D501009385C520F3
:1033B00065B78D451D46E3E4E5FA1146198E63F3C2
:1033C000C7003E86B7E704002390C600FC4797D5A8
:1033D00001009385A51B49B78D451D46E3E1E5F83E
:1033E0001146198E63F3C7003E86B7E704002390A9
:1033F000C600FC4797D501009385C51DB1BFA54503
:103400001D46E3EEE5F42946198E63F3C7003E86B8
:10341000B7E704002390C600FC4797D501009385C9
:10342000A5171DBFB5451D46E3EBE5F23946198EDC
:1034300063F3C7003E86B7E704002390C600FC474D
:1034400097D501009385C51201BFB7E7040003A318
:103450000713970600209386A6C24146A545170587
:1034600000201305E5B802832D455DE703C505007F
:103470000947631FE50803A84500411106C6034735
:10348000180032850346080022074168518F9308CF
:1034900028FE6307170563E9E800051863030703BF
:1034A00023900600294591A8130648FE630AC70425
:1034B0001518E31707FF15463E87637BF60015478F
:1034C00001A8130600023E876374F600130700028A
:1034D000B7E704002390E600FC471316070111A884
:1034E0003E8691C30546B7E70400FC472390C6001B
:1034F0004206CC45418282970145B240410182801B
:10350000130600083E87E375F6FC13070008C9B7E9
:103510002390060005458280828041677917630405
:10352000E504411122C406C685472A84639FF5003D
:10353000B7E7040022852244B24003A3871397050E
:1035400000209385E52F4101028389476399F500A7
:10355000B7E7040083A7070B8545829771D9B2406E
:103560002244410182808280797126D252CCAE847D
:103570002A8A97D501009385E50717D50100130521
:10358000E50906D63AC622D44AD0368432894ECED0
:1035900097C00100E78020A8A28517D50100130578
:1035A000E50897C00100E78000A7294597C0010002
:1035B000E78040AB83C7840093F70702F9E383C930
:1035C00004008947054532476396F908D44083C70C
:1035D000160083C60600A207D58FC166138616FEA5
:1035E000638CC7028D16638FD7068D6693862690EF
:1035F00029456391D706B7E70400A286225403A3A6
:103600004714B250F2494A86A6850259925452850F
:10361000624A8547456102832D450DEF93070002FD
:10362000354563E98702B7E70400FC47C844130641
:103630000002CA8582978149970700209387072156
:103640009C43014581CB9C4391C74E852286CA8508
:1036500082970145B250225492540259F249624A6B
:10366000456182802D457DF79307700F3545E3E373
:1036700087FEB7E70400FC47C8442286CA858297C4
:1036800065BF2145C1BF411122C437E4040083272F
:10369000841326C2AA84416506C697050020938537
:1036A000251A7D1582978327C40A17050000130584
:1036B00005E78588829795C0032304132244B2400E
:1036C000924497060020938626AE4146C5451705CD
:1036D00000201305659C41010283B24022449244BC
:1036E00001454101828019C59707002023A0A71634
:1036F00001458280454582801147636AA70A97D6B3
:1037000001009386E6ED0A0536951841411106C67B
:103710003697AE87B2850287130700026145639D25
:10372000E700B7E70400FC47130600021705002076
:10373000130545F782970145B24041018280054754
:103740006145E39BE7FEB7E70400FC470546170524
:103750000020130525F7F9BF1307700F6145E39D9E
:10376000E7FCB7E70400FC471306700F17050020BD
:10377000130585F5C1B7130700086145E39EE7FA15
:10378000B7E70400FC4713060008170500201305DF
:1037900025034DB715476145E390E7FAB7E7040005
:1037A000FC471546170500201305C50961B70945F3
:1037B0008280411126C2B7E4040083A7C41322C447
:1037C0004AC006C62E8497050020938565072A897E
:1037D0008297058905C5970700209387E78B83D7D4
:1037E000A70BA28503A3440D2310F4002244B2408A
:1037F00092444A850249014641010283B240224473
:103800009244024949454101828097070020238163
:1038100007049707002023AF0702B717004003A74C
:10382000070CB706C0FFFD16758F23A0E70C03A792
:10383000070DB7064000558F23A8E70C03A7070C18
:103840003D9B23A0E70C03A7070D1367070123A8DF
:10385000E70C8280B717004003A5470C83A7470CED
:10386000598113451500C18B058999E3136525001E
:103870009707002083C7C7FD6380A7029707002032
:103880002388A7FC11C9970700209387A7FC03A3EF
:1038900007006303030002838280114517F3FFFFD3
:1038A000670063C8011122CC06CE3714004026CA37
:1038B0004AC84EC652C483447405034AB4058349BA
:1038C00084050349940597F0FFFFE780A0A0834794
:1038D000A40593F4F40F137AFA0F93E71700230D5E
:1038E000F40493F9F90F1379F90FB717004003C7E0
:1038F000A705058B6DFF03D5C705A38D4705238C51
:103900003705A38C2705A38B9704F2406244D24469
:103910004249B249224A05618280411193970501CB
:1039200022C406C626C2C1872E8463DC0700B7E422
:103930000400FC54829719C1BC5482972165218DE3
:1039400015A893F7150013C515008DE793F725000B
:103950009DC797000000E78020F0B7E70400BC4F48
:103960001306000A894517050020034525EF8297B5
:1039700013452400B240224492444101828093972F
:10398000250163D80702B7E4040083A7C41E829709
:1039900097000000E780A0F0BC4C375607001306E4
:1039A0000630896517050020034545EB82970965B8
:1039B00079B7939715010145E3DE07FA17D50100A2
:1039C0001305C5CE97B00100E780C07CB7E70400BF
:1039D000BC4F13060064916517050020034505E8F8
:1039E00082971165A9BF1D71A2CC37E404005C5C0D
:1039F000485886CE494697D501009385A5C682973B
:103A000011E917D50100130525C797B00100E7801C
:103A1000607801A0B7F600E0795798CAFD57DCCA74
:103A20000567B7E700E023A0E7101306F00290C295
:103A300023A0E718010001003707002018471306EC
:103A4000000481459706002023A8E6E04157A38A99
:103A5000E7403C4408088297970700209387077C3B
:103A60003EC8856713870740938757D1231AE10023
:103A70002312F1021307B00F97F7FFFF9387C76474
:103A80002310E1023ED81547970700009387C7E14E
:103A9000B7F50700A30FE1003EDC054797070000DC
:103AA0009387E7DF81463000E10519452301E102F4
:103AB0003EDE97F0FF1FE780C0D218088147994685
:103AC00030003E960346060085070507A30BC70096
:103AD000E398D7FEC24791C70357410185676373D7
:103AE000F70001A0B7E7040083A7470A08088297F8
:103AF000AA8511C917D50100130545B997B0010072
:103B0000E780605101A0F640664425618280411142
:103B100026C2B7E4040083A7040806C622C417051A
:103B200000001305C5DF829717040020130404D397
:103B30002300A40097000000E780800297000000A7
:103B4000E780E0CC03450400224403A38405B2408F
:103B5000924413060032896541010283797106D6C9
:103B600022D413078008F337078093F787083EC2F3
:103B700001000100B7170040930570052380B704CA
:103B8000130680FA2380C7040100010083C6F702F0
:103B900093F6A60FA387D702238007049246F3A6C5
:103BA00006800100010073370780137787083AC445
:103BB000010001002380B7042380C7040100010035
:103BC00003C7F70213672700A387E70223800704D0
:103BD000A247F3A7078001000100054597E0FFFF1A
:103BE000E780807297000000E78060CB0147814644
:103BF0008147054685451305407E97E0FFFFE78036
:103C0000807537E404003C44680051468145829742
:103C1000B707C0A83EC8B787E803938707D03ECA56
:103C200097E7FF1F9387A7793EC67C586800829765
:103C3000B250225445618280411197D5010093858D
:103C4000250917D501001305659D06C697B001002B
:103C5000E780603C17D501001305451F97B00100B0
:103C6000E780603BB2402945410117B3010067007E
:103C7000633F411197D501009385C50617D5010013
:103C80001305C59906C697B00100E780C03817D55F
:103C900001001305651A97B00100E780C037B240F4
:103CA0002945410117B301006700C33B411122C4FC
:103CB00006C6834705002A849DC797D501009385D2
:103CC000250817D501001305659597B00100E78019
:103CD00080344C4017D501001305053097B0010022
:103CE000E78060333DA058410DEF97D501009385E3
:103CF000250517D501001305659297B00100E780EF
:103D0000803117D501001305A52E97B00100E7807B
:103D100080302244B2402945410117B301006700B9
:103D20006334A1679386D7036313D70297D5010045
:103D30009385050117D501001305458E97B0010045
:103D4000E780602D17D501001305852B7DBFED079A
:103D500097D501009385C5FE17D501001305058C85
:103D6000631BF70097B00100E780E02A17D5010038
:103D70001305452A59BF97B00100E780C0294C4080
:103D800017D501001305052B91BF411197D50100EF
:103D9000938585F617D501001305458806C697B0AB
:103DA0000100E7804027B2402945410117B30100D7
:103DB0006700432B797122D426D24AD02E842A89D7
:103DC000B28481457146480006D697E0FFFFE78040
:103DD000003497F7FF1F9387275EDC4783D70700E0
:103DE000231421012313F10097500000E780C03E07
:103DF0008547A305F1009307401F2305A1003EC698
:103E00002686FD57A2854800230AF100975000003E
:103E1000E780603FB250225492540259456182803B
:103E20004111814617F6FF1F1306465685451705B3
:103E300000200355252406C697D00000E780608F38
:103E400015C997D50100938565EE17C501001305C7
:103E5000E57C97B00100E780001C17D50100130531
:103E6000A51397B00100E780001B294597B001001A
:103E7000E780401F97D50100938545EB17C50100EA
:103E80001305C57997B00100E780E01817D5010048
:103E90001305C51197B00100E780E017294597B0D9
:103EA0000100E780201C97F7FF1F9387E750DC474E
:103EB000054797D50100938565E72390E70017C56F
:103EC00001001305A57597B00100E780C01417D550
:103ED00001001305E50E97B00100E780C013B24062
:103EE0002945410117B301006700C317011122CC16
:103EF00006CE26CA4AC84EC693F715002E84B5CB07
:103F000097000000E78000F2930710F817070020E1
:103F1000230AF7209707002083D78715170700206B
:103F2000A302F7209145A183170500201305851FE3
:103F3000170700202309F71E97070020A385071EF7
:103F400097600000E78080EAB7E70400BC4F1306E3
:103F5000001493050010170500200345A5908297D3
:103F600013451400F2406244D2444249B24905610B
:103F7000828093F70510B1C3054597600000E78084
:103F8000E0EF171500200355C57997600000E78022
:103F900060BB97200000E780805D9707002083C703
:103FA000B72789E797600000E780801197600000DD
:103FB000E780C0121345041075B793F72500E9CFC9
:103FC000170700200357871469C7AD64B71900406D
:103FD0009384A4AA23A099009706002093864613F1
:103FE000944297D701009387E70C170600200346F9
:103FF0000612814517D501001305C50C97800000F6
:10400000E780A08F23A0990097F7FF1F239AA72A84
:104010002A8941C197D50100938505D817C50100AC
:104020001305C55F97B00100E780E0FECA8517C59C
:1040300001001305657697B00100E780C0FD2945B2
:1040400097B00100E7800002970700202390070C3B
:10405000930710F8170700202306F70C9707002096
:1040600083D7070117070020A30EF70AA1831707BC
:104070000020230AF70A91458D47170500201305F4
:10408000650A17070020A300F70A97600000E78081
:10409000E0D513452400F9B593F74500D1C397D572
:1040A0000100938565CF17C501001305255797B00B
:1040B0000100E78040F617C501001305A56F97B012
:1040C0000100E78040F5294597B00100E78080F9BD
:1040D000930720F8170700202306F704970700200E
:1040E00083D747FB17070020A30EF702A18317070A
:1040F0000020230AF702854717070020A305F702CF
:1041000097500000E7804024170500201305850123
:10411000914597600000E78060CD1345440099B554
:1041200093F78500A9C797D501009385E5C617C504
:1041300001001305A54E97B00100E780C0ED17C53B
:1041400001001305656897B00100E780C0EC2945C0
:1041500097B00100E78000F197070020239807FA45
:1041600097800000E780408913458400E5BB93F702
:104170000501D1C38545170500200355A5F19760BA
:104180000100E780403E97D501009385E5C017C543
:1041900001001305A54897B00100E780C0E717C5E7
:1041A00001001305A56397B00100E780C0E629452B
:1041B00097B00100E78000EB930730F81707002065
:1041C0002302F7F69707002083D7C7EC17070020D4
:1041D000A30AF7F4170500201305C5F4A1838D4544
:1041E000170700202301F7F497600000E78000C064
:1041F0001345040185BB93F70502D1C797D501008C
:10420000938585B917C501001305454197B0010095
:10421000E78060E017C501001305855E97B00100D7
:10422000E78060DF294597B00100E780A0E39307AE
:1042300040F8170700202307F7EE9707002083D7E1
:10424000A7E317070020A30FF7ECA18317070020AF
:10425000230BF7EC854717070020A306F7EC970719
:104260000020239B07E097500000E780E00D170532
:104270000020130525EB914597600000E78000B70B
:1042800013450402C5B193F70504FDC397D501009A
:10429000938585B017C501001305453897B0010017
:1042A000E78060D717C501001305055797B00100D7
:1042B000E78060D6294597B00100E780A0DA97072C
:1042C000002083C727E61307700A6386E7061307F3
:1042D000800A638CE7081307600A6393E704930777
:1042E00060F817070020230FF7E29707002083D715
:1042F000C7E117070020A307F7E2A18317070020F3
:104300002303F7E2854717070020A302F7E2B14530
:1043100017050020130505E197600000E78000AD58
:1043200097500000E78040021345040497070020DF
:10433000239D07DC05B9930770F8170700202303B6
:10434000F7DE9707002083D747DC17070020A30B71
:10435000F7DCA183170700202307F7DC8547170741
:104360000020A303F7DC994565B7930780F8F1B700
:1043700093F705080145E38707BE97D501009385AC
:10438000A5A117C501001305652997B00100E780B5
:1043900080C817C501001305A54997B00100E78043
:1043A00080C7294597B00100E780C0CB9307A0F8EC
:1043B000170700202308F7D69707002083D787D553
:1043C00017070020A300F7D6A18317070020230CAE
:1043D000F7D4854717070020A307F7D497070020D5
:1043E000239A07D297500000E78000F617050020B7
:1043F000130545D3914597600000E780209F134542
:1044000004088DB6411122C497D501009385859487
:104410002A8417C501001305652006C697B0010060
:10442000E78060BF4C4017D50100130565B497B015
:104430000100E78040BE294597B00100E78080C2B7
:10444000034704009307F00F631FF70297D501009D
:104450009385459017C501001305451C97B00100D1
:10446000E78060BB4C4017D50100130565B197B0DC
:104470000100E78040BA2244B2402945410117B308
:104480000100670023BEB2402244410182804111F5
:1044900022C426C22A84AE8417C50100130505185C
:1044A00097D501009385C58606C697B00100E780C1
:1044B00080B617D501001305A5BC97B00100E780B1
:1044C00080B5294597B00100E780C0B997D50100B4
:1044D0009385058497070020239E87B817C50100A0
:1044E0001305C513054497070020239397B8970732
:1044F0000020239087B8971700202394972297B025
:104500000100E78040B19715002083D5852117D59C
:104510000100130565B797B00100E780C0AF2945DA
:1045200097B00100E78000B4971700202388870E1A
:1045300097F7FF1F938747E8DC4717F5FF1F0345F1
:10454000653203D70700C167FD17631EF700B7E7A1
:10455000040003A387051306000A85452244B240E0
:10456000924441010283B7E7040003A387051306C1
:10457000001493050010DDB7B1C1411122C417C565
:1045800001001305A5092E8497C501009385857741
:1045900006C697B00100E78000A8A28517D50100E4
:1045A000130545AD97B00100E780E0A62244B24074
:1045B0002945410117B301006700C3AA828097F71C
:1045C000FF1F83C7972A17F5FF1F0345252A3D8D37
:1045D000220597F7FF1F83C777293D8D4605458143
:1045E00011C5D1476315F500554582800545828088
:1045F0004111971700202396071297170020238F49
:10460000070006C6170700200347C7B19307F00A43
:104610006315F7029307F0F8894517050020130585
:1046200065B017070020230FF7AE97070020A38B74
:1046300007AE97500000E780607B97600000E7803E
:1046400020A897600000E78060A981453705040035
:104650009707002023AE07AA97070020238907AAFF
:1046600097070020239807A297070020239607A00A
:1046700097070020239B07A897070020239C07A8E3
:1046800097300000E780200D014597500000E7803B
:10469000E07E97000000E780C0F297070020239794
:1046A000A7A6B7E70400BC4F13060014894517F509
:1046B000FF1F0345251B829797C50100938545661B
:1046C00017C50100130585F597B00100E780A09498
:1046D0009705002083D585A317D501001305C59B39
:1046E00097B00100E7802093B2402945410117B3FC
:1046F000010067002397797122D437E404005C5CE1
:1047000006D626D2354697C501009385657517D51F
:1047100001001305654A829711E917C501001305C9
:10472000A5F597B00100E780E0A601A097F7FF1F6D
:10473000938707143ECCB7F50700856793870780FA
:10474000814617F6FF1F13062612E10519453ECED6
:1047500097E0FF1FE780E0087C44194697F5FF1FAC
:10476000938585101705002013050593829734085B
:1047700017F6FF1F1306460F97D50100938585BADC
:1047800017D50100130585BB97700000E780E0EBAB
:10479000AA8421C197C501009385055F17C5010053
:1047A0001305C5E797B00100E780E086A68517C529
:1047B00001001305E56B97B00100E780C08529452E
:1047C00097B00100E780008AB250225492544561AC
:1047D000828097E00000E780005117C501001305B3
:1047E000256097600000E78000E097600100E780A7
:1047F000400A17F5FF1F1305A5B897600100E78071
:10480000E0F217C501001305A55E97600100E7807F
:10481000C00AAA8497600000E780C0469710010094
:10482000E78020E297800100E780407B97800000CE
:10483000E780A0A297700000E780C0BC974001000D
:10484000E78080A397C501009385055417C5010033
:104850001305C5DC99C897A00100E780C07BA68539
:1048600017C5010013050563B9B797A00100E780DC
:10487000807A17C501001305256497A00100E78021
:104880008079294597A00100E780C07D973001001D
:10489000E780607F97000100E780209E6308051491
:1048A00097000000E780E0D197F7FF1F83D747A06C
:1048B000171700202317F7E62A8699C36302F50825
:1048C00097C501009385454C17C50100130505D513
:1048D00032C697A00100E780007432469715002089
:1048E00083D525E417C501001305855E97A0010057
:1048F000E7806072294597A00100E780A0769717AE
:104900000020238D07D097170020239C07E0977085
:104910000000E780600E97C501009385E54617C546
:1049200001001305A5CF97A00100E780C06E17C551
:1049300001001305A56297A00100E780C06D41B595
:1049400085453705040097300000E780C0E097C533
:1049500001009385654317C50100130525CC97A079
:104960000100E780406B17C501001305A55997A00A
:104970000100E780406A294597A00100E780806E2A
:10498000854717170020230BF7C897F7FF1F93875A
:10499000A7A2DC4703D70700C167FD176316F7001E
:1049A00097F0FFFFE780004897700000E780001550
:1049B0008567938707E33E9597700000E780C014F2
:1049C00097200000E780A0BA17150020035565D591
:1049D00097500000E7800017054597500000E780DA
:1049E000E04997500000E780606F35B797000000FE
:1049F000E78020BD97F7FF1F239AA77097C5010096
:104A00009385853817C50100130545C197A001009E
:104A1000E780606017C601001306065197F5FF1F77
:104A200083D5C56E17C501001305855097A00100F9
:104A3000E780605E294597A00100E780A0623C4CBA
:104A40001306000A894517F5FF1F0345A5E1829764
:104A5000014597500000E780604275BD411122C4B6
:104A600037E404008327041A06C682979750000093
:104A7000E78000118327040817F5FFFF130545475A
:104A8000829797F7FF1F238FA7DC17F5FF1F1305EA
:104A9000A59297500000E780E0C12244B240410156
:104AA00017030000670063C5B7E70400FC471171F6
:104AB000A2DDCAD986DFA6DBCED72E8432892E8628
:104AC000AA8517F5FF1F1305E565829717F7FF1FE6
:104AD0001307476583470700930680029387E7071C
:104AE00093F7F70FE3ECF610BA898A0717C70100AE
:104AF000130707BCBA979C43BA9782878D4797C51F
:104B000001009385A52A17C50100130525B1630F80
:104B1000F40097A00100E780005017C501001305BD
:104B2000A5E797A00100E780004FBDA497A0010072
:104B3000E780604E17C50100130585E797A00100C7
:104B4000E780604D294597A00100E780A0519307B9
:104B500020F8114697F5FF1F9385C55C4A8517F726
:104B6000FF1F2301F75C97F7FF1FA38E075A97F0EB
:104B7000FFFFE78060242A841DC997C50100938543
:104B8000E52217C50100130565A997A00100E7807C
:104B90008048A28517C50100130545E597A00100CF
:104BA000E7806047294597A00100E780A04B97C5A3
:104BB00001009385A51F17C50100130525A697A021
:104BC0000100E780404517C50100130565E397A084
:104BD0000100E7804044294597A00100E780804814
:104BE0004165930730FA054697F5FF1F9385855376
:104BF0007D1517F7FF1F2307F75297F0FFFFE78098
:104C0000A01B2A841DC997C501009385251A17C5C5
:104C100001001305A5A097A00100E780C03FA28571
:104C200017C50100130585DC97A00100E780A03EB1
:104C3000294597A00100E780E042B7E70400BC4F98
:104C40000566130606C8A14517F5FF1F034585C174
:104C50008297FE506E54DE544E59BE5911618280C7
:104C600091476303F40297C501009385251417C586
:104C700001001305A59A97A00100E780C03917C568
:104C80000100130525DB71BDB7E70400FC4F91451A
:104C900017F5FF1F034505BD829797C50100938552
:104CA000E51017C501001305659797A00100E7807F
:104CB000803617C501001305A5D997A00100E7802C
:104CC0008035294597A00100E780C0399740000052
:104CD000E7808067914535A485476303F40297C553
:104CE00001009385A50C17C501001305259397A016
:104CF0000100E780403217C501001305E5D615B560
:104D000097F7FF1F23982739B7E704000566BC4FC4
:104D1000130606C8C1450DBF8D476303F40297C54E
:104D200001009385A50817C501001305258F97A0DD
:104D30000100E780402E17C501001305A5D4D5B3A7
:104D4000930740F8114697F5FF1F9385A53D4A85C7
:104D500017F7FF1F2308F73C97F7FF1FA385073CB2
:104D600097F0FFFFE78040052A84E30405EE97C52E
:104D700001009385A50317C501001305258A97A097
:104D80000100E7804029A28517C50100130505C66B
:104D900097A00100E7802028294597A00100E7801F
:104DA000602C45BD9147E31CF4F6B7E70400FC4FC7
:104DB0009305000217F5FF1F0345C5AA829797C503
:104DC00001009385A5FE17C501001305258597A051
:104DD0000100E780402417C50100130525CCF1BD73
:104DE000894763E3870297C50100938525FC17C5B2
:104DF00001001305A58297A00100E780C02117C517
:104E000001001305E5CA31BB97F4FF1F83C4A43129
:104E100097F7FF1F83C7173197C50100938505F9E1
:104E2000A20417B501001305657FDD8C97A0010072
:104E3000E780601EA28517C501001305A5C897A0CD
:104E40000100E780401DC204294597A00100E780CA
:104E50006021C1849305D4FF93960401C1824A86E0
:104E600093F5F50F17F5FF1F1305F52B973000008D
:104E7000E7802092E35F90DC930750F817F7FF1F5D
:104E80002302F72A83C73900228697F5FF1F9385EF
:104E9000652985074A8517F7FF1FA306F72897F0AE
:104EA000FFFFE78060F12A84E30505DA97C501007A
:104EB0009385C5EF17B501001305457697A001004E
:104EC000E7806015A28517C501001305A519C9B5AE
:104ED000894763E3870297C50100938525ED17B5E0
:104EE00001001305A57397A00100E780C01217C544
:104EF00001001305E5BE35B197400000E780C044CE
:104F0000A28517F5FF1F1305E52197500000E780E4
:104F1000E0ED81B38D476303F40297C501009385EB
:104F2000E5E817B501001305656F97A00100E7805C
:104F3000800E17C50100130565BCE5B6B766020013
:104F40000146B7750200054597E0FF1FE7806089BD
:104F5000930760F817F7FF1F2306F71C97F7FF1F4B
:104F6000A383071C9307000617F7FF1F230EF71AEA
:104F7000894717F7FF1FA309F71A97F7FF1F238623
:104F8000071A97F7FF1FA382071AC14717F7FF1FDA
:104F9000230EF718930720F917F7FF1FA308F71838
:104FA000314697F7FF1FA384A71897F5FF1F938536
:104FB00065174A8597F7FF1F238B071697F0FFFFAA
:104FC000E78080DF2A84E30605C897C50100938542
:104FD000E5DD17B501001305656497A00100E780C2
:104FE0008003A28517C501001305C5B255B3B147AB
:104FF0006303F40297C50100938545DB17B50100F3
:105000001305C56197A00100E780E00017C5010006
:10501000130505B239B6B7E70400FC4F9305000449
:1050200017F5FF1F03450584829797400000E7802E
:10503000A031B145F9B5914763E3870297C50100F7
:105040009385C5D617B501001305455D97A00100EE
:10505000E78060FC17C50100130545AFD9B497F48C
:10506000FF1F83C4640C97F7FF1F83C7D70BA204ED
:10507000DD8C8E04B77702006D14BE942286A6855F
:1050800017C501001305C5AD97A00100E780A0F882
:10509000B7E70400FC47228697F5FF1F9385D508E4
:1050A0002800829793160401C1823000A685094525
:1050B00097D0FF1FE780E0722A8409C917C5010055
:1050C0001305C5AB97A00100E780C00C930770F8EB
:1050D000194697F5FF1F9385E5044A8517F7FF1FCB
:1050E0002302F70497F7FF1FA380870497F0FFFFC1
:1050F000E78080CC2A84E30E05B497C50100938530
:10510000E5CA17B501001305655197A00100E780B6
:1051100080F0A28517C50100130545A795B99947E9
:10512000630BF41297C50100938545C817B50100BC
:105130001305C54E97A00100E780E0ED17C50100FB
:10514000130545A6F9BA914763E3870297C50100A5
:105150009385C5C517B501001305454C97A00100FF
:10516000E78060EB17C50100130545A55DBA97F40C
:10517000FF1F83C464FB97F7FF1F83C7D7FAA204FE
:10518000DD8C8E04B77702006D14BE942286A6854E
:1051900017C501001305C5A397A00100E780A0E78C
:1051A000B7E70400FC47228697F5FF1F9385D5F7E4
:1051B0002800829793160401C1823000A6850D4510
:1051C00097D0FF1FE780E0612A8409C917C5010055
:1051D0001305C5A197A00100E780C0FB930780F8E5
:1051E000194697F5FF1F9385E5F34A8517F7FF1FCB
:1051F000230AF7F297F7FF1FA38887F297F0FFFFC4
:10520000E78080BB2A84E30605A497C50100938547
:10521000E5B917B501001305654097A00100E780C7
:1052200080DFA28517C501001305859D95B69947B6
:105230006303F40297C50100938545B717B50100D4
:105240001305C53D97A00100E780E0DC17C501000C
:105250001305859CF9B0B7E70400FC4F93050004E3
:1052600017E5FF1F03450560829797400000E78020
:10527000A00D994579B18D476303F40297C50100EC
:105280009385C5B217B501001305453997A00100F4
:10529000E78060D817C501001305859959B017C577
:1052A00001001305E59997A00100E780A0EE130522
:1052B000C01297D0FF1FE780C008014597E0FFFFAD
:1052C000E78080DD0D4597100000E780C0A32945E9
:1052D00097D0FF1FE780E00697D0FF1FE78040F7D9
:1052E0008DBA99476303F40297C50100938505AC15
:1052F00017B501001305853297A00100E780A0D102
:1053000017C501001305859429B817F7FF1F034738
:10531000B7E197F7FF1F83C727E122075D8F9166EB
:10532000BA96C2061166C1821306F6EF8D47636511
:10533000D60297E7FF1F938727089C4B17F6FF1F9E
:10534000034676DE9386C7002DC203D6070069CADE
:105350008907E39CD7FE89471307A0F8114697F504
:10536000FF1F938525DC4A8597F6FF1F238CE6DA1D
:1053700017F7FF1FA309F7DA97F0FFFFE780C0A335
:105380002A84E308058C97C50100938525A217B5EB
:1053900001001305A52897A00100E780C0C7A285DA
:1053A00017C501001305C58BE5B203D60700630ED0
:1053B000E60A8907E39BF6FE8D4779BF91476304B0
:1053C000F40297C501009385659E17B5010013058A
:1053D000E52497A00100E78000C417C5010013056C
:1053E000A5896FF00FF4B7E70400FC4F93050008A0
:1053F00017E5FF1F034505478297C9B897C5010008
:105400009385C59A17B501001305452197A00100A2
:10541000E78060C017C50100130585876FF06FF046
:105420002390E70017E5FF1F130505F997300100EA
:10543000E780E0EA97C501009385459717B501001D
:105440001305C51D97A00100E780E0BC17C501004A
:105450001305058597A00100E780E0BB294597A0CB
:105460000100E78020C08147C5BD2390070017E5F4
:10547000FF1F130565F497300100E78040E697C5EC
:1054800001009385A59217B501001305251997A072
:105490000100E78040B817C501001305E5815DBF35
:1054A000011122CC06CE26CA4AC8834705002A84A9
:1054B0009DC797C501009385258B17B5010013057E
:1054C000E51597A00100E78000B54C4017C5010025
:1054D000130545C097A00100E780E0B3E1A0584163
:1054E000B707CF009387777D631DF7060359C50083
:1054F000854704450356E5009706002083D66622BB
:1055000063FC270383C7040003C71400A207D98FD5
:10551000C2077177C1871307C755639FE70063050B
:10552000D60C6244F240CA8526854249D2440561C0
:1055300017E3FFFF6700C3CA630AD600CA85268542
:1055400032C697E0FFFFE780A0C932466244F240CE
:10555000CA8526854249D244056117F3FFFF6700DB
:10556000E354B707CC009387777D6317F70497B5AB
:1055700001009385657F17B501001305250A97A0E3
:105580000100E78040A91C448356E4008355C40011
:1055900003C6070017C50100130545B597A0010014
:1055A000E78060A76244F240D24442492945056140
:1055B00017A30100670003ABB707CE009387777D81
:1055C0006304F70297B501009385057A17B50100CA
:1055D0001305C50497A00100E780E0A34C4017C560
:1055E0000100130525A5FDB5F2406244D2444249AD
:1055F00005618280B7E70400FC4741112E8606C68C
:1056000022C426C24AC02E842A89AA8517F5FF1F04
:10561000130545B1829797B501009385E57A17B5D3
:1056200001001305A5FF97A00100E780C09E97F534
:10563000FF1F83C525AF17B501001305E52097A00F
:105640000100E780409D294597A00100E78080A1E7
:1056500097F4FF1F938404AD83C7040041479387E9
:10566000070693F7F70F636FF75A17B70100130791
:10567000670E8A07BA979C43BA9782879D4763074C
:10568000F40297B501009385257417B50100130541
:10569000E5F897A00100E780009817B50100130511
:1056A000251B97A00100E780009795A497F7FF1F9F
:1056B00083C757A7DDCB17F7FF1F0347D7A697F779
:1056C000FF1F83C747A622075D8F97F7FF1F83C77A
:1056D000A7A5C2075D8F97F7FF1F83C7F7A4E2074F
:1056E000D98F17F7FF1F2325F7A283C7640097B54B
:1056F00001009385656D17B50100130525F217F7B5
:10570000FF1F2306F7A097A00100E780C09097F73E
:10571000FF1F9387E79F8C4317F6FF1F0346269FC3
:1057200017B501001305851497A00100E780A08E2E
:10573000294597A00100E780E09297F7FF1FA38318
:10574000079E2244B24092440249930700F817F79B
:10575000FF1F2309F79C9D4517F5FF1F1305859C27
:105760004101174300006700636897600000E7800D
:10577000203897F7FF1F2388A79A9357850017F7BC
:10578000FF1FA302F79A935705012A8417F7FF1FFB
:10579000230CF79893578501014517F7FF1FA305C1
:1057A000F79897600000E780003997F7FF1F238E76
:1057B000A79697B501009385256117B501001305DC
:1057C000E5E597A00100E780008517F6FF1F034677
:1057D000C695A28517B501001305C50AB1B7CD4717
:1057E0006303F40297B501009385055E17B50100C8
:1057F0001305C5E297A00100E780E08117B501001D
:105800001305C50979BD97F7FF1F83C7C79217F71F
:10581000FF1F03473792A207D98FC207C18717F727
:10582000FF1F2315F78E634AF00097F0FFFFE78014
:1058300040D997F7FF1F239BA78CB7E7040003A36A
:1058400087051306000A89452244B2409244024962
:1058500017E5FF1F03450501410102838D476303DF
:10586000F40297B501009385255617B5010013057D
:10587000E5DA97900100E780007A17B5010013057B
:10588000A51105B517F4FF1F0344E48997F7FF1F1F
:1058900083C7578997B5010093850553220417B52F
:1058A00001001305A5D75D8C97900100E780A076D5
:1058B000A28517B501001305E5FF97900100E78069
:1058C0008075294597900100E780C0790D4697F5CE
:1058D000FF1F93852585228597E0FFFFE780C04D58
:1058E000AA8421C197B501009385054E17B5010023
:1058F0001305C5D297900100E780E071A68517B522
:105900000100130565FC97900100E780C0702244F8
:10591000B2409244024929454101179301006700B2
:10592000637497E7FF1F23978776B7E70400116634
:1059300003A38705130606E8914539B78D4763032E
:10594000F40297B501009385254817B501001305AA
:10595000E5CC97900100E780006C17B501001305B6
:10596000651281B317E4FF1F0344E47B97E7FF1F31
:1059700083C7577B97B5010093850545220417B56A
:1059800001001305A5C95D8C97900100E780A06810
:10599000A28517B50100130565F497900100E78013
:1059A0008067294597900100E780C06B0D4697E519
:1059B000FF1F93852577228597E0FFFFE780C03F93
:1059C000AA841DC197B501009385054017B5010054
:1059D0001305C5C497900100E780E063A68517B55D
:1059E00001001305E5F005B797E7FF1F23968768C9
:1059F000B7E70400116603A38705130606E89305BD
:105A0000000299B5894763E3870297B50100938542
:105A1000A53B17B50100130565C097900100E7800D
:105A2000805F17B501001305A508A5B997E4FF1F0E
:105A300083C4646F97E7FF1F83C7D76E97B50100D4
:105A400093858538A20417B50100130525BDDD8CAB
:105A500097900100E780205CA68517B5010013052B
:105A6000A5EA97900100E780005B29459790010027
:105A7000E780405F228697E5FF1F9385A56A26850C
:105A800097E0FFFFE78040332A84630E051A97B53D
:105A900001009385653317B50100130525B897906C
:105AA0000100E7804057A28517B50100130505E7FF
:105AB00099BD854763F98718834519002244B24090
:105AC00092440249B335B00097E7FF1F238EB75CBD
:105AD00017B501001305C5E54101179301006700E3
:105AE0008353A2852244B24092444A85024941012F
:105AF000170300006700632799476303F40297B513
:105B000001009385652C17B50100130525B1979009
:105B10000100E780405017B501001305251351B669
:105B200017E4FF1F0344246097E7FF1F83C7975FB5
:105B300097B5010093854529220417B50100130587
:105B4000E5AD5D8C97900100E780E04CA28517B52C
:105B50000100130565DF97900100E780C04B2945E0
:105B600097900100E7800050194697E5FF1F938545
:105B7000655B228597E0FFFFE7800024AA841DC1B2
:105B800097B501009385452417B50100130505A9B4
:105B900097900100E7802048A68517B501001305FE
:105BA000A5DB95B397E7FF1F23968756B7E7040059
:105BB000116603A38705130606E89305000869B17B
:105BC000854797B501009385252017B5010013057A
:105BD000E5A4630BF40097900100E780C04317B57C
:105BE00001001305A5D875BC97900100E780A0427D
:105BF00017B50100130505D997900100E780A04172
:105C0000294597900100E780E0452244B240924444
:105C1000024997E7FF1F239B074E410117630000CE
:105C2000670083DD97B501009385051A17B501005C
:105C30001305C59E97900100E780E03D17B5010070
:105C400013050505B9BCB240224492440249410102
:105C50008280411106C622C426C239C12A8497E037
:105C60000000E7808061AA8411EDB7E70400BC471B
:105C70004146814522858297B2402244268592443E
:105C80004101828041657D1597E00000E780C05F9B
:105C9000B7E7040001E9BC47414681452285829768
:105CA0008144D9BF0347E501FC479305900819E3F8
:105CB00093050003AA9541462285829785446DBFCE
:105CC000411106C697E0FFFFE780000F0DC197E77F
:105CD000FF1F83D7873D850717E7FF1F2317F73C73
:105CE00097E7FF1F2394A73CB2404101828097E7CA
:105CF000FF1F83D7C73B850717E7FF1F2319F73A15
:105D0000E5B7411122C491462A8417E6FF1F130606
:105D1000664F9D652D4506C697D0FF1FE78060AC96
:105D2000B7F7070003C70701A5476313F70001A0F2
:105D30009306001001469D65254597D0FF1FE7801B
:105D400040AA97E7FF1F238F874A2244B24091461B
:105D500017E6FF1F1306064B9D652945410117D322
:105D6000FF1F670003A81171CED7B7E9040083A70E
:105D7000C904CAD917E9FF1F1309C93AA2DD2E8643
:105D800086DFA6DB2E84AA854A85829797E7FF1FC8
:105D900083C747391307700A6385E710636DF700FF
:105DA0001307600A6385E704FE506E54DE544E59B3
:105DB000BE59116182801307800A6385E7161307B5
:105DC000900AE393E7FE8D476306F41C97B5010044
:105DD0009385453D17B50100130545849790010053
:105DE000E780602317B501001305053925A08D470D
:105DF000630CF40297B501009385C53A17B501000D
:105E00001305C58197900100E780E02017B50100D8
:105E10001305C52F97900100E780E01F2945979053
:105E20000100E780202449B7854717B50100130515
:105E3000A52F17E7FF1F2309F72697900100E7809A
:105E40006035B7750200B76602000146054597D078
:105E5000FF1FE7800099930760F817E7FF1F2303F0
:105E6000F72C97E7FF1FA380072C9307002617E75F
:105E7000FF1F232BF72AE5779387072117E7FF1FDB
:105E80002316F72AB14597E7FF1F2382072A97E7D2
:105E9000FF1FA38EA7284A8597000000E780E01621
:105EA00021B7914763E3870297B501009385852F5A
:105EB00017A501001305857697900100E780A015CE
:105EC00017B5010013054528B1B797E4FF1F83C438
:105ED000A42597E7FF1F83C71725A204DD8C83A79E
:105EE000C9046D14228697E5FF1F9385F5232800CA
:105EF00082978E0493160401B7750200C1823000A8
:105F0000A695094597D0FF1FE780A08D930770F8ED
:105F100017E7FF1F2308F720994597E7FF1FA38581
:105F2000A72095BF914763E3870297B5010093854A
:105F3000652717A501001305656E97900100E7809E
:105F4000800D17B501001305A521E9B597E4FF1FE2
:105F500083C4841D97E7FF1F83C7F71CA204DD8C51
:105F600083A7C9046D14228697E5FF1F9385D51B6F
:105F7000280082978E0493160401B7750200C1822F
:105F80003000A6950D4597D0FF1FE78080859307C9
:105F900080F8BDBF17B501001305451F979001009C
:105FA000E780401F930790F82304F100834719000E
:105FB0008D452800A304F100834729002305F10043
:105FC00097000000E78060041305C01297C0FF1F10
:105FD000E7802037014597D0FFFFE780E00B0D45B4
:105FE00097000000E78020D2294597C0FF1FE78077
:105FF000403597C0FF1FE780A0257DB397E7FF1FBF
:1060000023AAA720828097E7FF1F9387A72003A3D7
:10601000070063030300028317430000670003DDEA
:1060200041114AC097F6FF1F83D6A66F328917D653
:10603000FF1F0356863A22C426C206C62A84AE84AF
:1060400097000000E780E06729C921C8994763F6F7
:1060500097048347140003470400A207D98F1397BE
:106060008700A183D98FC2073167C1831307C75542
:106070006395E70297D7FF1F83D72736A301F40064
:10608000A1832302F40097F7FF1F83D7876991C785
:10609000A302F400A1832303F40097F7FF1F83C733
:1060A000E757A1CB2686A28517D5FF1F0355E532FA
:1060B00097000000E78000C1630F090297F7FF1FF8
:1060C00083C7C7558DEB97E7FF1F83C7E71485C7C5
:1060D0009DC097E7FF1F83C727FD91EF22852244CC
:1060E000B2400249A685924441011743000067006F
:1060F000E3CFE31A09FCB240224492440249410131
:1061000082800145828097A701009387A7419C4325
:1061100001116800914506CE3EC697000000E78059
:10612000C0EEF240056182808D4763F6B708011129
:1061300026CA06CE22CC0344350097E4FF1F83C451
:10614000B40D97B501009385A507B337800017E715
:10615000FF1FA303F70C09C497B50100938505073A
:1061600017B501001305050797900100E780A0EA25
:1061700097E7FF1F83C7570A6386970097000000C1
:10618000E780004397400000E78040F599679387D8
:1061900057EE2316F100680085479145A30781005B
:1061A0002307F10097000000E78020E6F2406244F8
:1061B000D244056182808280894763F7B708011164
:1061C00022CC06CE26CA8344250085472A84639DB7
:1061D000F404914763F5B704034545008347340051
:1061E00022055D8D97D7FF1F2399A71E97000000FA
:1061F000E78000569967938767EE2314F100834781
:10620000340023059100A305F10083474400954520
:1062100028002306F10097000000E78000DFF2402D
:106220006244D24405618280FDF89967938767EEE6
:106230002314F10097D7FF1F83D7271AA305F10076
:1062400023050100A183E1B782800111996722CC67
:10625000D51717F4FF1F1304643C2314F100834780
:10626000040026CA97F4FF1F9384A44B2305F10072
:1062700083D7040028009545A305F100A18306CE2D
:106280002306F10097000000E78020D803D6040021
:106290008345040017B501001305C5F4979001006C
:1062A000E78060D7F2406244D244056182809D67F6
:1062B0007971D9172316F10097F7FF1F93870736D7
:1062C00083C707001305F10006D62307F1009700E6
:1062D0000000E780409809E9B7E70400BC47414661
:1062E00081451305F10082976800CD4597000000B5
:1062F000E780A0D197F5FF1F83C5453217B5010090
:10630000130545F197900100E780E0D0B250456158
:10631000828063080516411126C206C622C44AC0FF
:1063200097E7FF1F83C757EF97F4FF1F83C4042F1E
:1063300099C393E424002A8497100000E780E0F0DA
:1063400019C193E4040137E90400832789042285F5
:106350001306200381458297930750FA2300F40027
:106360009307A005A300F4008D472301F400914793
:10637000A301F4009307D004A302F40097F7FF1FD2
:1063800083D7273A2304F400A183A304F40097D70A
:10639000FF1F83D78704230394002305F40093048D
:1063A000C400A18323020400A305F40026859700FE
:1063B0000000E780408A19E583278904414681452A
:1063C0002685829797D7FF1F83D7C7FE230EF40039
:1063D000A183A30EF40093070002230FF400930798
:1063E00010FAA30FF4009D472300F402A300040257
:1063F000B7E70400FC4713052402194697D5FF1F91
:1064000093858546829797E7FF1F83D747CA230462
:10641000F402A183A304F40297E7FF1F83D7E7C820
:106420002305F402A183A305F40297E7FF1F9387D6
:10643000E7C7839707002285930500032306F4022C
:10644000C207C183A183A306F40297D7FF1F9387D6
:1064500027E7839707002307F402C207C183A183BC
:10646000A307F40297000000E780A0212308A402FC
:106470002181A308A402B24022449244024941016E
:10648000828082805D71E17793C777FF1305E10019
:1064900086C62316F10097000000E780C0E7680079
:1064A0009305400397000000E78020B6B640616185
:1064B00082805DC9411122C426C206C6930750FAE4
:1064C0002300F5009307A005A300F50089472301E9
:1064D000F5009147A301F5009307D004A302F5004E
:1064E00097F7FF1F9387871383C707009304C5009F
:1064F0002A842303F50097E7FF1F9387F7D183C70B
:10650000070023020500A303F50097F7FF1F83D7B9
:1065100047212304F500A183A304F50097D7FF1FAB
:1065200083D7A7EB2305F500A183A305F5002685F6
:1065300097F0FFFFE780207201E9B7E70400BC474E
:1065400041468145268582972285F14597000000C6
:10655000E7802013230EA4002181A30EA400B240E3
:10656000224492444101828082805D710A8586C600
:10657000A2C497000000E78000F437E404007C44E4
:106580008A850810794682973C441305E103094641
:1065900081458297101093050002014597D0FFFFB7
:1065A000E780C015B6402644616182800111B7C7FB
:1065B000A55A22CC9387C73317E4FF1F1304D4C511
:1065C0003EC483470400856601469965254506CE8D
:1065D0003EC697C0FF1FE780C0203000A1469965E6
:1065E000294597C0FF1FE780C01F8345040017B5EA
:1065F00001001305A5CC97900100E780C0A1F240EF
:106600006244056182800111A146300099652D45E3
:1066100022CC06CE97C0FF1FE780A01CA24737C43C
:10662000A55A1304C43363958702B24517B5010018
:10663000130585C0B335B00097E7FF1FA38EB7BC25
:1066400097900100E780209DF240624405618280BE
:106650009165A1463000938505F02D4597C0FF1F39
:10666000E7802018A247E38287FC97E7FF1FA385F6
:1066700007BA814517B50100130545BED1B7C167FB
:1066800069768146FD170506139706014183636409
:10669000B7003E8582803307D50003470700B98FD6
:1066A000214713F81700858363050800B18FC207DF
:1066B000C1837D171377F70F6DF78506F1B741C5D5
:1066C000A547054763F2B708834715000347050050
:1066D0003168A207D98F13978700A183D98FC2078A
:1066E000C1831308C855054763900707411106C6C3
:1066F00022C426C203442500914763F08704930710
:10670000540063ECF502A301C50021822302C500F9
:106710009304340091C6A302D500A1822303D500BF
:106720002A84A68597000000E780A0F52694230020
:10673000A4002181A300A4000147B2402244924456
:106740003A854101828005473A8582800111B7C7A9
:10675000A55A22CC9387E7342A842AC68566014647
:106760009565254506CE3EC497C0FF1FE7806007AC
:106770003000A1469565294597C0FF1FE780600658
:10678000A28517B50100130565B597900100E78054
:10679000808897000000E78080DDF2406244056158
:1067A00082800111A146300095652D4522CC06CE90
:1067B00097C0FF1FE780E002A24737C4A55A130421
:1067C000E43463958702B24517B50100130505ABA4
:1067D00097D7FF1F2393B7C0C205C18197900100CF
:1067E000E7806083F2406244056182809165A14642
:1067F0003000938505EE2D4597C0FF1FE78060FEB2
:10680000A247E38287FCD14717D7FF1F2317F7BCA6
:10681000D14517B50100130565A8C9B721C14111BC
:1068200026C206C622C4AE848DC52A8497100000F5
:10683000E78040A297E7FF1F83C7079E99CB228579
:106840002244B240A68592444101173300006700FC
:10685000E359B24022449244410182808280011176
:106860004EC606CE22CC26CA4AC893F71500AE897A
:106870009DCBAD67371700409387A7AA1CC3B7E726
:106880000400BC4F13060019854517D5FF1F0345AB
:10689000A5B4829713C51900F2406244D24442491C
:1068A000B2490561828093F725000145F5D717F7B6
:1068B000FF1F0357E7E6954763F9E70C014417F616
:1068C000FF1F1306E6D59306300513055004130881
:1068D00010049308B00413039005930764006374D5
:1068E000F7043A847D5997F4FF1F83C464D397F764
:1068F000FF1F83C7F7D2A204DD8CAD679387B7551E
:10690000638BF41463E3970AA9679387A755638E93
:10691000F414A28517F5FF1F130585D0970000001A
:10692000E78000F0E9A0B307860083C50700639AFB
:10693000D50483C517006396A50483C52700639219
:10694000050583C53700639ED50283C54700639A5A
:10695000150383C757006396670222890DE897F5F0
:10696000FF1F83D5E5DBB3852541C20517F5FF1F62
:10697000130505CBC1814A9597000000E78040EAE6
:10698000E1A005044204418089BF3A847D598547CE
:10699000E3EB87F45DC4854517F5FF1F130545C874
:1069A00097000000E780C0E769A8B1679387C755E3
:1069B0006389F404B5679387D755E39CF4F4A28503
:1069C00017F5FF1F1305C5C597300000E78000428B
:1069D0008947630EF4009305E4FFC205C18117F5F2
:1069E000FF1F130505C497100000E780A086A68549
:1069F00017B501001305459097800100E780A0615D
:106A000089A097200000E780C03397100000E7803E
:106A1000C08311C9A28517F5FF1F130565C0971024
:106A20000000E78020830546A28517F5FF1F1305A8
:106A300025BF97F0FFFFE780E05E97200000E7802A
:106A40004030FD57E31DF9F097F7FF1F239A07CC5D
:106A500013C5290091B5A28517F5FF1F130545BC85
:106A600097F0FFFFE780206A59B7A28517F5FF1F4F
:106A7000130505BB97F0FFFFE78020698DBF41112B
:106A800022C437E404005C5C06C6354697A50100C5
:106A90009385053D17B5010013050512829711E98D
:106AA00017B501001305858697800100E780806E89
:106AB00001A08327041C82972A84054597C0000003
:106AC000E780C02197700100E780E0A69760010091
:106AD000E780E07B97B00000E78040332285B2403A
:106AE0002244410182804111054506C622C426C2C6
:106AF00097C0FFFFE78020441305A00497B0FF1F55
:106B0000E780E05A757585457D1597C0FFFFE780E2
:106B1000C02D7D7585451305F53697C0FFFFE780CD
:106B20002037371400408327840A8D451305002041
:106B300093E707202324F40A97C0FFFFE780E02AA9
:106B4000B7E4040097C0FFFFE7800070C858978043
:106B50000100E780206417B501001305E505978063
:106B60000100E78020638327840C8545414593E736
:106B700007082324F40C97C0FFFFE78060318D45A0
:106B80001305000897C0FFFFE780803097C0FFFF24
:106B9000E780605D37A507001305051297C0FFFF6A
:106BA000E7800059014597C0FFFFE780205F9545CA
:106BB0000545894717F7FF1F2306F7B697C0FFFF64
:106BC000E780605FB7E700E013070006238DE7402A
:106BD0003707000423A0E71097D0FFFFE780E0E02D
:106BE00097D0FFFFE780E0F297000000E78060E9C0
:106BF00097000000E78060A197000000E780A0BA3E
:106C000097E0FFFFE780C0E597000000E780C065E0
:106C100097000000E780801083A704081705000094
:106C2000130525C4829797C7FF1F2387A77ABC4CFB
:106C3000130600648545829797B0FF1FE780407B6D
:106C400001458280AD67371700409387A7AA1CC310
:106C5000B7E700E03707400023A0E7180100010074
:106C6000B7F7070003C70701A5476316F700939717
:106C7000450191C301A04111AE860146AA85254573
:106C800006C697C0FF1FE780C0B5B240B7E700E077
:106C90003707400023A0E710410182804111B286EE
:106CA0002E86AA852D4506C697C0FF1FE78060B3D4
:106CB000B2400145410182809307000463ECC704A0
:106CC0001D71A2CC2A840808A6CACAC886CE32C6BC
:106CD00097800100E780C028AD6737170040938791
:106CE000A7AA1CC3B7E400E03709400023A0241979
:106CF00001000100B2461008A285294597C0FF1F78
:106D0000E78020AEF640664423A02411D6444649CD
:106D1000256182803955828041110D658D4506C6F9
:106D200097C0FFFFE780600CB71700408D6623A671
:106D3000D70A17F5FF1F1305259F1387C70A9387E7
:106D4000870A1CC15CC5856689675CC958C114C5C2
:106D500018C9B7E70400B24003A3871E41010283AC
:106D60008145B307B5008387070089E71723000033
:106D70006700C3038505C205C181E5B7411106C699
:106D8000B94763EEB70017A501001305656F9700BB
:106D90000000E78020FDB240054541018280834725
:106DA000E500130710036390E702854717F7FF1FFD
:106DB000230EF7A617A501001305C56E97F7FF1F51
:106DC000239507A6E9B713070003E39EE7FA97F7B1
:106DD000FF1F238D07A497F7FF1F239807A417A56C
:106DE00001001305A56D65B7411126C2E97797F437
:106DF000FF1F9384E4A322C49387A7552E84238185
:106E0000B4002E86AA8517F5FF1F1305A5A206C696
:106E10002390F400A381040097800100E7804014D0
:106E200093052400C205C18117F5FF1F130565A056
:106E300097000000E780E084B38784002382A700E6
:106E40002181A382A700930564002244B2402685D5
:106E50009244C205C181410117230000670003F578
:106E600009C99307000463E6B70017030000670031
:106E7000E3F782809306F00F0307060019E79307F4
:106E8000F00F63F0B7022E85828093871500C2074A
:106E9000C183E3E6F6FEAA952380E5000506BE85DC
:106EA000E1BF2E9523000500F9BF01111C08B6971C
:106EB00006CE238A07FE5C00BE9617A801001308C1
:106EC000686B1377F600429703470700FD1611829F
:106ED0002380E600E397D7FE3E8697000000E78018
:106EE000A0F9F240056182800111580006CE230707
:106EF0000100A947BA8829482543B3760603FD1740
:106F000093F7F70F93860603A304D700B35606033F
:106F10006375C3007D173686EDF33386F80097005E
:106F20000000E78060F5F24005618280397117A6A4
:106F300001001306265D06DE22DC26DA2A844AD802
:106F40004ED697000000E78020F3AA8517E6FF1FC2
:106F50000356267D9146228597000000E78020F5A4
:106F600097E7FF1F83C7876BAA8517A60100130643
:106F7000E65689C717A601001306C6552285970055
:106F80000000E78060EFAA8517A601001306C65728
:106F9000228597000000E78020EEAA8517A6010051
:106FA00013060657228597000000E780E0ECAA85CB
:106FB0001146228597000000E78040F3AA8517B6A6
:106FC0000100130666B3228597000000E780C0EA3F
:106FD000AA8517A6010013062654228597000000F3
:106FE000E78080E9AA8517B601001306E6B022857E
:106FF00097000000E78040E8AA851306D0042285A8
:1070000097000000E78080EE97D7FF1F83C7D72047
:10701000AA8517A601001306E64C89E717A601000A
:107020001306C64C228597000000E780E0E4AA859D
:1070300017A601001306864E228597000000E78000
:10704000A0E337A60700AA8513060612228597003B
:107050000000E780A0E9AA8517A601001306864C68
:10706000228597000000E78020E197E7FF1F83C794
:10707000276DAA8517A601001306C64789E717A63C
:1070800001001306A647228597000000E780C0DEB6
:10709000AA8517A601001306A649228597000000BD
:1070A000E78080DDAA8517A601001306E648228541
:1070B00097000000E78040DCAA8517A601001306B0
:1070C0002648228597000000E78000DB9146AA85CC
:1070D00017C6FF1F0356062E228597000000E78083
:1070E00000DDAA8517A601001306C6452285970074
:1070F0000000E78060D89146AA8517C6FF1F035697
:10710000C62D228597000000E78060DAAA8517A6C1
:1071100001001306A643228597000000E780C0D532
:107120009146AA8517D6FF1F035666F82285970059
:107130000000E780C0D7AA8517A601001306864184
:10714000228597000000E78020D39146AA8517D6B4
:10715000FF1F035686F5228597000000E78020D5A3
:10716000AA8517A601001306663F22859700000036
:10717000E78080D09146AA8517D6FF1F035606F3F5
:10718000228597000000E78080D2AA8517A601001B
:107190001306063D228597000000E780E0CDAA8512
:1071A000914617C6FF1F0356A611228597000000BF
:1071B000E780E0CFAA8517A601001306E63A2285EC
:1071C00097000000E78040CBAA85814497C9FF1F44
:1071D000938989691949B387340103C60700894631
:1071E000228597000000E78080CC8504AA85E3947F
:1071F00024FF17A601001306A6372285970000007A
:10720000E78080C72AC6080897F0FFFFE780A0A4A0
:10721000B24504081309010283C7040003C6140021
:107220009146A2075D8E228597000000E78020C866
:107230008904AA85E31299FEF2506254D25442594D
:10724000B2592161828017E5FF1F0345654F828097
:1072500097E7FF1F83C7875D89E717230000670053
:10726000E3B4828097E7FF1F83C7E76099EF41117E
:1072700006C697200000E78040ABB240854717E77D
:10728000FF1F230AF75E4101828082806302054C62
:107290006380054C2971B7064000232E1112232C60
:1072A0008112232A91122328211323263113232408
:1072B00041132322511323206113232E7111232CF8
:1072C0008111232A91112328A1112326B1110147ED
:1072D0005948A5069319070193D9090163F1B90229
:1072E000B307E50083C70700D91793F7F70F636863
:1072F000F800B3D7F600858B13061700A1E3B38916
:107300003541C20993D90901B9472E89AA8463F985
:1073100037033304E500394697A501009385C50579
:10732000228597800100E78040C119E9CE8522853A
:1073300097000000E780C0A425E5F1A4328759BF7B
:1073400097E7FF1F83C7874E638F0724BD6A396C99
:10735000014A17EBFF1F130BEB3E938BFA55938CEF
:10736000FA66130DEC5505A8B387440183C60700E0
:1073700097E7FF1F83D7674BA5E39307A005639BA0
:10738000F600854717E7FF1F2311F74A97E7FF1F0E
:10739000238AD73A050A93170A01C183E3E627FD3A
:1073A0008320C11303248113832441130329011370
:1073B0008329C112032A8112832A4112032B01124D
:1073C000832BC111032C8111832C4111032D011139
:1073D000832DC11031618280854D639BB703930774
:1073E000500A639EF600894717E7FF1F231FF742E5
:1073F000930750FA17E7FF1FA306F73461BF9307FF
:10740000A005E389F6F897E7FF1F2390074259B7D5
:10741000138717004207DA9741832380D70017E6C6
:10742000FF1F2314E6408D47E3F6E7F617E4FF1F3E
:107430000344743197E7FF1F83C7E73022045D8C54
:107440009307F4FFC207C1839306F00DE3EDF6FA4C
:1074500093076400C207C183E31EF7F2930524007B
:10746000C205C18117E5FF1F1305E52D97F0FFFF4A
:10747000E780202133078B008347570003474700ED
:10748000A207D98F17E7FF1F2311073A6312F510E0
:107490008149630DB40197E9FF1F83C9E92AA20955
:1074A00097E7FF1F83C7572AB3E9F90017050000C4
:1074B0001305459B97F0FFFFE78080B4638579094A
:1074C00063EF3B036388A9059307EC656383F906C3
:1074D00097E7FF1F83C7472705476380E70881CBEE
:1074E0001387A7051377F70F8D4663F9E60813078F
:1074F000F0072300E100A300F100894595A8638906
:1075000099059387FA77E395F9FC97F0FFFFE780F9
:10751000A0F711A8A28517E5FF1F1305E52297F034
:10752000FFFFE780A0C0014597F0FFFFE78040AD77
:1075300095B5A28517E5FF1F1305052197F0FFFFFD
:10754000E780C0C7CDB797F0FFFFE78040D0E1BF2D
:1075500097F0FFFFE780E0D5F9B7930710F8130520
:1075600011002300F10097F0FFFFE780C0F4FD4514
:107570000A8597000000E780608775B7A28517E548
:10758000FF1F1305651C97E0FFFFE780007E61BFCA
:107590009307F00789450A852310F1009700000042
:1075A000E780C084C5BB15476375270503C6040083
:1075B0009306500B0147631FD60203C614009306BF
:1075C000B0053E876318D602CA85268597F0FFFF6F
:1075D000E78060B311C917A501001305E5DA97F03C
:1075E000FFFFE78020786DBB17A50100130505DBC1
:1075F000FDB70147B70640005946A5061314070119
:10760000418063692401CA85268597C0FFFFE78012
:1076100020BD79B3B389E40083C70900D91793F774
:10762000F70F6367F600B3D7F600858B0507F9F708
:107630003304894042044180BD4763FD87064146CB
:1076400097A50100938585D74E8597800100E78037
:10765000C08E17A601001306A6D705C13D4697A503
:107660000100938525D84E8597800100E780E08C46
:1076700039E517A601001306E6D781450A8597F07C
:10768000FFFFE780607FAA850A8597000000E780FA
:10769000208AAA8517960100130606550A8597F0D9
:1076A000FFFFE780607DAA850A8597100000E780CC
:1076B000E06FFDB1E304F4FAB947E316F4F4394698
:1076C00097A50100938545CB4E8597800100E78003
:1076D000C08601E5A2854E85A1B9394697A501006E
:1076E000938585D24E8597800100E780008501DD76
:1076F000C147E3FA87F0414697A501009385C5D1BC
:107700004E8597800100E7804083E31E05EE83C726
:10771000090113071003639CE700854717E7FF1F64
:107720002300F70217A50100130545D04DBD13072F
:10773000000317A50100130565D2E392E7EA97E776
:10774000FF1F238F07FE17A501001305A5CF41BD1D
:107750008280411126C2AE848D4522C406C62A8489
:1077600097B0FFFFE780C072B717004099C803A524
:10777000C70C418D23A6A70CB2402244924441017C
:10778000828003A5870C418D23A4A70CF5B78347FE
:10779000050003471500A207D98FC2076177C1878B
:1077A00013072720639AE700834525003705040067
:1077B00017030000670023FA828017E6FF1F1306F5
:1077C000E60B8147B2861303F00FA9483308F60091
:1077D0000348080013F7F70F6307A80C6306680057
:1077E0008507E39517FF2947B387E6002380A700A5
:1077F00097E7FF1F938747095DA8411113D76500DD
:107800001347170006C693F63500058B954791CAB6
:10781000054699476387C60009469D476383C600AE
:10782000A14713F645003336C00093F685030506DD
:1078300085C2A145638BB604E145638AB60493050E
:1078400080026388B604930580036393B600914673
:1078500097E5FF1F238FF52897E5FF1F238AC5288B
:1078600097E5FF1FA386D528BE8517A50100130540
:1078700065D497700100E780007AB240854717E72A
:10788000FF1FA308F726410182808546D1B78946AC
:10789000C1B78D4675BF17A50100130525D4177311
:1078A00001006700437717E7FF1F1307E7FDBA974B
:1078B0002380B700E147E302F5F493077002E30C7D
:1078C000F5FC82802A8723800500814717E5FF1F8A
:1078D0001305C5FA1308F00F2946B306F50083C651
:1078E00006006396E60297E6FF1F9386E6F9B697D1
:1078F00083C7070005452380F5009947636EF702AB
:107900009D4763FDE700E147630DF70082806385D3
:1079100006018507E393C7FC0145C5B72380050031
:107920008280B737004003C7370083C7050093F74D
:107930000704D98F2380F50082805D7152DC56DA0E
:107940005ED6716A97EBFF1F938BCB2B8D6AA6C215
:107950004EDE62D486C6A2C4CAC05AD866D26AD0E5
:107960006ECEC1495E8C97E4FF1F9384A4F2130A84
:107970000A20938A7ADC17E9FF1F0349A92BB387F2
:107980002B0183C7070093F7F70FC9EFB7870040B4
:1079900003C76700058BE310077C03C76700118BE3
:1079A000E30D077E83C75700918B99E36F10200387
:1079B00017E7FF1F0347272885476304F7006F1069
:1079C000400197E7FF1FA386E71297E7FF1F238376
:1079D00007F897E7FF1F2381070497E7FF1F238F0F
:1079E000070E97E7FF1F238C070E97E7FF1FA38360
:1079F00007F697E7FF1FA381070297E7FF1FA38FF3
:107A0000070C97E7FF1FA38C070C97E7FF1FA383C3
:107A1000070E97E7FF1FA3800722B7870040114793
:107A20006F0070779307190093F7F70F3D47636472
:107A3000F70617E7FF1F230FF71E97E7FF1F938730
:107A4000671ECA9783C707001307100293F7F7034F
:107A5000638EE71E6366F70405446385871CE38C29
:107A600007620947638EE71013070002E384E74EBD
:107A7000B7E700E03707400023A0E7180100010046
:107A8000629923000900FD1923A0E71093F9F90F6B
:107A9000E39309EEE5BD97E7FF1F238D071871BF3C
:107AA000130730026388E70C63E8E7161307400208
:107AB000638CE70A13070003E39CE7FA97E7FF1FCD
:107AC00093874715CA9703C70700A1471377F70F96
:107AD000E31BF71483C7640097E6FF1F2382F600B9
:107AE00097E7FF1F83C777DB91C7FD5797E6FF1F17
:107AF0002388F6FE97E5FF1F83C5D5D997E7FF1FBB
:107B0000A380B7FE97E7FF1F83C7C7D813FB0708FB
:107B10009306000493F70706639FD74C9307A009C9
:107B2000638DF51663EAB7129307F0056386F54A8D
:107B3000930750096384F52A014497E7FF1F83C721
:107B400037FA1547E392E736B7E700E0370740001A
:107B500023A0E71801000100B786004023808602B9
:107B6000130680FC6F00500EFD5717E7FF1F230818
:107B7000F7F6FDBDFD5717E7FF1F2301F7F6CDBD53
:107B800017A50100130505B797700100E780806015
:107B900097E7FF1F93870708CA9703C40700014BA5
:107BA00097ECFF1F938C8CE71374F40F17AD010053
:107BB000130DCDB463478B04294597700100E7800E
:107BC000604A854717E7FF1FA308F7E417E7FF1F81
:107BD000230587E417E7FF1F230EF7F037E700E0E0
:107BE000B70640002320D718010001003786004067
:107BF0008347A60293F7370F2305F6022320D710F9
:107C000085BDB3876C0183C507006A85050B977036
:107C10000100E780404079BF854717E7FF1F230D2C
:107C2000F7DEB9B517E7FF1F1307C7FE4A970347EB
:107C3000070097E6FF1FA38FF6D097E6FF1F238C60
:107C4000E6D017E7FF1F2307F7EA1DB5854717E7BB
:107C5000FF1F2301F7D029BD9307400A6389F5343C
:107C60009307200B6384F5369307100AE396F5EC2F
:107C7000838724000144E3D207EC97E7FF1F83C703
:107C800097C193F63700638A061A0546638AC622AF
:107C900009466395C61A1D4755A217E5FF1F034500
:107CA00085BFC94797ECFF1F83CCFCBE97E5FF1F3C
:107CB00083C585BE17E4FF1F034414BE6315F5108A
:107CC000CD476392FC1093077008639CF50213077D
:107CD000300FB7170E006308E4001307900DB7B715
:107CE00004006314E40817E7FF1F2321F7E0BE85B3
:107CF00017A50100130505A197700100E780A031C9
:107D000025BD93078008639DF500B307804013F4F9
:107D1000F70FB7774600938787CDB3D78702E1B7D0
:107D200093079008639AF500B307804013F4F70FA8
:107D300091679387C766D5B79307A008639BF50043
:107D4000B307804013F4F70FB7173D0093870790F0
:107D5000E9B79307B008639AF500B307804013F4BE
:107D6000F70F9167938797D04DBF93F5F5078D4730
:107D7000639BF500B307804013F4F70FB7975B00E0
:107D8000938707D859BF8947639BF500B3078040A5
:107D900013F4F70FB7770B009387071BBDBF854719
:107DA000639AF500B307804013F4F70FDD679387FC
:107DB00067E3A5B7D28785F9B307804093F7F70F3C
:107DC000B3D7FA020DB797000000E780409FA28565
:107DD000668597000000E780809EB9BB930561002F
:107DE00017E5FF1F034525AB17E4FF1F0344B4AAA3
:107DF00097000000E78040AD930571002285970051
:107E00000000E78060AC3C0017E7FF1F232AF7DE85
:107E1000834761002304F10083477100A304F1004C
:107E2000894717E7FF1F230DF7CA8357810017E71C
:107E3000FF1F2311F7A6094409B3154793F647001E
:107E4000B336D00093F78703850685C32146638B3D
:107E5000C7066146638AC706130680026388C706A1
:107E6000130680036393C700914717E6FF1F2301A2
:107E7000D6C897E6FF1FA38DF6C697E7FF1F238A94
:107E8000E7C617E7FF1F034727A19376070497E785
:107E9000FF1F83C777A08DEE1377770C93067008CA
:107EA000630CD7021377F7078D466312D70CB3071D
:107EB000F040B7955B0093F7F70F938505D849A875
:107EC0001947ADBF854755B7894745B78D4771BF3E
:107ED000930670086311D7021307300FB7150E0011
:107EE0006389E7021307900DB7B504006383E702C7
:107EF0001307700845BF9306800C6311D702B307C0
:107F0000F040B775460013F7F70F938785CDB3D5CB
:107F1000E70297E7FF1F23ABB7BCD9BB9306900CD2
:107F2000631CD700B307F04093F5F70F9167938771
:107F3000C766B3D5B702F1BF9306A00C631DD70087
:107F4000B307F040B7153D0093F7F70F9385059001
:107F5000B3D5F5027DBF9306B00CE315D7F4B30794
:107F6000F04093F5F70F9167938797D0D9B789467B
:107F7000631BD700B307F040B7750B0093F7F70FFB
:107F80009385051BF1B78546631AD700B307F04008
:107F9000DD6593F7F70F938565E35DBFD28535FB0C
:107FA000B305F04093F5F50FB3D5BA029DB783C77B
:107FB0002400C18B99C7854717E7FF1F2305F7B238
:107FC000A5BE97E7FF1F238007B2BDB6854717E719
:107FD000FF1FA300F7B28DB63C0017E7FF1F232158
:107FE000F7C20947930700032314F10097E6FF1F28
:107FF0002388E6AE2DBD63940756A94763E5B742D3
:1080000017970100130747588A05BA959C41BA97FC
:10801000828717E4FF1F03441488894C6306940D7C
:1080200063E68C0685476303F4089307F00F17E7B0
:10803000FF1F0347E7AA63F6E70017E7FF1F2301C7
:10804000F7AA97ECFF1F83CCACA99307000413F4A5
:10805000FC0F63F497011304000497E7FF1F938755
:1080600027BA03AD070022862685EA85B38C8C40AB
:10807000229D97700100E780A0EE97E7FF1F238104
:1080800097A797E7FF1F23ADA7B745BC8D47630CA4
:10809000F40A9947E31BF4F8979701009387475533
:1080A00017E7FF1F232EF7B4A94751B717E7FF1FA4
:1080B000034767B897E7FF1F938787A449469795BB
:1080C00001009385E55B6306870097950100938522
:1080D00025573E8597700100E78080E817E7FF1F6E
:1080E0002320A7B2C947A1B797E6FF1F83C6A6B44E
:1080F000054797E7FF1F9387A7A06394E6023E8595
:10810000130670029795010093850555977001003D
:10811000E78000E517E7FF1F2324A7AE930770024F
:1081200039B73E8513063004979501009385054DB8
:1081300097700100E780C0E217E7FF1F2322A7AC7A
:1081400093073004EDB597D5FF1F83C5C574179508
:1081500001001305655C97700100E780C0EB054DD9
:1081600097EDFF1F83CD2DAD97D5FF1F83C5A5725A
:10817000179501001305455A6398AD0B97700100E0
:10818000E78060E997D7FF1F83C7E770B5CBE36E41
:10819000F4E8179401001304E452638CB7011794B8
:1081A00001001304A452638697011794010013047D
:1081B0006453228597700100E78000FF1375F50F67
:1081C00093071500860717E7FF1F230BF7928D47CC
:1081D00017E7FF1FA306F79297E7FF1F93874792C2
:1081E0000147BE861376F70F89076365A60297E7F6
:1081F000FF1F23A7D7A097E7FF1F83C7679005BD81
:10820000979701009387074517E7FF1F232AF79EDB
:10821000914731BD3306E40003460600A380070002
:1082200005072380C7007DBF97700100E780A0DEAF
:1082300097D7FF1F83C72766E1D7E368F4DE17945B
:10824000010013042445638CA70117940100130453
:10825000E44463869701179401001304A445228522
:1082600097700100E78040F41375F50F9307150030
:10827000860717E7FF1F2305F7888D4717E7FF1FBE
:10828000A300F78897E7FF1F938787870147BE867C
:108290001376F70F8907E37CA6F43306E400034660
:1082A0000600A380070005072380C700D5B797D530
:1082B000FF1F83C5455E179501001305A5469770FE
:1082C0000100E78040D597E7FF1F83C7378393E717
:1082D000470017E7FF1FA303F78283C7240017E7B0
:1082E000FF1FA30BF78089B8179501001305C5443C
:1082F00097700100E78000EA97D7FF1F9387C77F39
:1083000083C7070017D7FF1F2306F75817D4FF1F8F
:108310000344047D333480000DB01795010013052C
:10832000E54297700100E780E0E697D7FF1F83C71B
:10833000F77C93E7070117D7FF1FA301F77C83C7DB
:10834000240017D7FF1F2309F77A6FF0EFFE179568
:1083500001001305E54097700100E780A0E303C723
:1083600004007D8B51EFB787004003C76702137786
:10837000C70B136727002383E70203C7A7021377FE
:10838000C70B136727002385E70203C7E7021377AC
:10839000C70B136727002387E70203C72703137759
:1083A000C70B136727002389E702854717D7FF1FED
:1083B0002302F75A17D7FF1F2300F76617D7FF1FAF
:1083C000230EF77017D7FF1F230BF77097D7FF1FE8
:1083D000A382075897D7FF1FA380076497D7FF1F73
:1083E000A38E076E97D7FF1FA38B076E97D7FF1F2C
:1083F000A382077097E7FF1FA38F07826FF0CFF369
:1084000089476312F70297D7FF1F83C7E748914652
:10841000638CD70863E0F604638EE70C6369F70AA0
:1084200005476380E70EFD5717D7FF1FA30AF76ABA
:1084300037074000B7E700E023A0E718010001007C
:10844000B78600401306F0FC2381C60223A0E71084
:108450006FF00FE2130720086382E7086362F702F8
:1084600013071008E391E7FC378700408347670252
:1084700093F7C70B93E727002303F7026FF0CFEBC7
:10848000130730086389E70213074008E39DE7F804
:10849000378700408347270393F7C70B93E72700ED
:1084A0002309F7026FF04FE937870040834727031E
:1084B00093F73707F5B7378700408347E70293F70D
:1084C000C70B93E727002307F7026FF0EFE6378724
:1084D00000408347E70293F73707F5B73787004037
:1084E0008347A70293F7C70B93E727002305F702FB
:1084F0006FF08FE4378700408347A70293F7370771
:10850000F5B7378700408347670293F73707ADB762
:10851000179501001305C52597700100E78080C7F6
:1085200097D7FF1F23880736D5B31795010013058A
:10853000252597700100E780E0C597D7FF1F239B93
:10854000073497D7FF1F9387A75903C407008947AC
:1085500063F3870009441374F40F6FF00FDE130701
:108560000002E392E7EC631B0B0A638FF5009307AD
:1085700020026383F508179501001305E523977022
:108580000100E78040A945B51795010013050520B6
:1085900097700100E78000C00144179D0100130D92
:1085A0002D20A14CB387840083C507006A8505048C
:1085B00097700100E78020A6E31694FF178501005D
:1085C0001305856897700100E780C0BC17D4FF1FB2
:1085D0000344842C01E897D7FF1F238F0728014B02
:1085E0006FF0AFD58947E310F4E4854717D7FF1F35
:1085F0002304F7286FF04FD417D6FF1F0346B62980
:1086000097D5FF1F83C52529179501001305C519A7
:1086100097700100E78020A06FF00FD26380F5060D
:1086200093071002E399F5F497D5FF1F83C5C5267C
:10863000179501001305451997700100E780A09D6B
:1086400097D7FF1F23AE975A97D7FF1F9387074AE5
:10865000944383D7470017D7FF1F0347874917D68F
:10866000FF1F2329D6221D4497D6FF1F2396F622EB
:1086700097D7FF1F2383E7226FF02FCC97D5FF1FDB
:1086800083C5852117950100130585159770010095
:10869000E780609897D7FF1F2380071E97D7FF1F9B
:1086A000239A071E6FF02FF92547638FE7C8994675
:1086B000378700406394D70223008702B7E700E0C2
:1086C000B706400023A0D71801000100130600FCE4
:1086D0002301C70223A0D7106FF08FB99306100AA9
:1086E000639FD70023008702B7E700E0B70640008A
:1086F00023A0D71801000100130680FCD1BF930608
:10870000A009E381D7FE9306400AE38DD7FC9306C8
:108710002002639DD700B7E700E0B706400023A022
:10872000D7180100010023008702F9B78546E384CA
:10873000D7FE93070008E300FBFEB7E700E0B706AB
:10874000400023A0D71801000100130620FC2300DD
:108750008702BDBF17D7FF1F034797386302F71E75
:1087600063E7E70295476300F7109947630AF70448
:10877000B786004023800602B7E700E037074000D5
:1087800023A0E718010001001306A0FC75B99307A8
:10879000F005630AF700930750096306F700930793
:1087A0001002E317F7FCB7E700E03707400023A00B
:1087B000E71801000100B7860040130620FC69B1EC
:1087C00017DBFF1F034BCB31930700045A8D63F473
:1087D0006701130D000497D7FF1F9387674283AC8F
:1087E00007001374FD0F2286E68526859760010039
:1087F000E7800077B3078B40669417D7FF1F2301EC
:10880000F72E97D7FF1F23AD873EB7870040630C35
:108810000B022380A703B7E600E03706400023A041
:10882000C6180100010003C727021347070423816C
:10883000E70203C727021377C70F2381E70223A0AC
:10884000C6106FF0EFA22380070237E700E0B706FB
:1088500040002320D71801000100130620FC2381CB
:10886000C7026FF0AFB9378700408347370097D60C
:10887000FF1F83C6762893F70708D58FA301F7005B
:10888000B7064000B7E700E023A0D71801000100B9
:108890001306A0FC35BD97D7FF1F9387A737CA974C
:1088A00083C7070093F7F70FC1CF97D7FF1F83C781
:1088B0008738D9E717D7FF1F03479722930700028E
:1088C0006310F70883AD040017DDFF1F034DCDFCD7
:1088D00097DCFF1F83CC5CFC17DBFF1F034BEBFB1C
:1088E000E6876A87DA866E8697D5FF1F83C5C5F847
:1088F00017950100130545F097600100E780A0710E
:1089000097D7FF1F23A4B71F97D7FF1F2382A71F47
:1089100097D7FF1FA38E971D97D7FF1F238B671D28
:1089200097D7FF1FA38987F4B7E700E03707400018
:1089300023A0E71801000100B78600406FF04FA2A6
:10894000B7E700E03707400023A0E7180100010067
:10895000B786004015BD97D6FF1F83C6C62D0547B5
:10896000639CE60429472381E70209472383E70242
:108970002385E70297D7FF1FA38E071697D7FF1F00
:10898000A38B072AB7870040A381070017D7FF1FD3
:10899000A304071605472383E700B6402644964400
:1089A0000649F259625AD25A425BB25B225C925C2F
:1089B000025DF24D6161828029472381E702094708
:1089C0002383E7022385E7022387E7022389E7025F
:1089D00055B717D7FF1FA300F7EA6FE01FFF8547C2
:1089E00017D7FF1F2308F7F617D7FF1F2306F70235
:1089F00017D7FF1F2304F70E17D7FF1F2301F70E0A
:108A00006FE0BFFE854717D7FF1F2305F7F417D781
:108A1000FF1F2303F70017D7FF1F2301F70C17D7FA
:108A2000FF1F230EF70A17D7FF1FA30507F217D75B
:108A3000FF1FA30307FE17D7FF1FA301070A97D73E
:108A4000FF1FA38E07088280411106C69700000011
:108A5000E78080FBB787004023800700130740FCB6
:108A60002386E7001307C004A386E70017D7FF1F7C
:108A7000130747E22398E70017D7FF1F130787E57F
:108A8000239AE70017D7FF1F130707F1239CE7007E
:108A900017D7FF1F130787FC239EE7002947238171
:108AA000E70209472383E7022385E7022387E702DA
:108AB0002389E702A3810700930600F8A380D7006B
:108AC000930690022380D700FD562383D70023818D
:108AD000E7009306000537E700E0230BD740B70611
:108AE00040002320D71003C7170013671700A38087
:108AF000E700B24097D7FF1F239007004101828013
:108B0000411106C697000000E78000F0B7870040DB
:108B100023800700130700FC2386E7003147A38664
:108B2000E70017D7FF1F1307E7D62398E70017D7EB
:108B3000FF1F130727DA239AE70017D7FF1F130732
:108B4000A7E5239CE70029472381E7020947238300
:108B5000E7022385E702A3810700930600F8A380BC
:108B6000D700930690022380D700FD562383D700B9
:108B70002381E7009306000537E700E0230BD74089
:108B8000B70640002320D71003C71700136717004C
:108B9000A380E700B24097D7FF1F239F07F441014E
:108BA0008280F1679387072017D7FF1F2320F7F4F0
:108BB000854717D7FF1F231DF7F2A14717D7FF1FC0
:108BC0002309F7F297D7FF1FA38507F297D7FF1F57
:108BD000238207F297D7FF1F238007CA97D7FF1F6B
:108BE000A38B07C8814717D5FF1F130525C9FD555E
:108BF00017D6FF1F130646C92947B306F500238081
:108C0000B600B306F600238006008507E397E7FE6B
:108C100097D7FF1FA38707EC97D7FF1FA38507EC04
:108C200097D7FF1F238007EC97D7FF1F238B07EAF7
:108C300097D7FF1F238A07EA97D7FF1FA38407EA66
:108C400097D7FF1F238107EA814717D6FF1F130617
:108C500066FB4147B306F600238006008507E39BC9
:108C6000E7FE828017D7FF1F0347E7FC854763169F
:108C7000F700170300006700E3E817030000670030
:108C8000E3DC411122C406C617D7FF1F0347A7FA2A
:108C900085472E8613F4F50FAA856317F70417D5B9
:108CA000FF1F130565D397600100E780602B97D7FE
:108CB000FF1F238307D6B787004023848702B7E6C8
:108CC00000E03706400023A0C6180100010003C7DA
:108CD000A7021377C70F2385E702B240224423A0DF
:108CE000C61001454101828017D5FF1F130585C2BB
:108CF00097600100E780C02697D7FF1F238C07C429
:108D0000B787004023828702B7E600E037064000BD
:108D100023A0C6180100010003C767021377C70F1D
:108D20002383E7025DBF411106C697000000E7807C
:108D300080E7B2404101170300006700E3F24111F0
:108D400006C697F0FFFFE78080BF97D7FF1F83C756
:108D500077C0A1CB97D5FF1F83C5E5BF89C917D5BC
:108D6000FF1F130565BF97E0FFFFE780605297D7AD
:108D7000FF1FA38107BE97D7FF1F238D07D637E7B5
:108D800000E0B70640002320D71801000100378615
:108D900000408347660293F7370F2303F602232030
:108DA000D710B2404101828041C9D9C597D7FF1F72
:108DB00083C787D4D1C3011122CC4AC84EC656C23C
:108DC0005AC006CE26CA52C42E89AA890144930AE3
:108DD0000004371B030063772403B3078940C207ED
:108DE000C183BE8463F4FA0093040004C204C1800A
:108DF000130A1BD497D7FF1F83C7C7B59DE37D1AFE
:108E0000631C0A00F2406244D2444249B249224AF9
:108E1000924A024B0561828097F0FFFFE78020B203
:108E2000D1BF338589002694A685420497000000AF
:108E3000E78060E5418045B7828097D7FF1F938721
:108E4000E7F118429C4383D645000345070083C5DC
:108E5000C700035646006396A50083D5E700638DDF
:108E6000D502011106CE2386A7002397D700B705A8
:108E7000CF00DC4B9385757D05077D162EC2230040
:108E800001003AC42316C1002317D10099C30A85F3
:108E90008297F240056182808280411122C417A42A
:108EA000FF1F1304E4555C4C06C691CBC84B01C9A7
:108EB000B7E70400BC5782975C4C23AA0700B24076
:108EC000224441018280DC4DDC4B81CFB7E70400B6
:108ED000904503A38705914517D5FF1F034545E836
:108EE00002838280B7E7040003A30705A14517D5D5
:108EF000FF1F0345E5E602836D713C083EC6B707D8
:108F0000E500232291103EC8AA843C08328523261E
:108F100011103ECA23248110232021112E8997305D
:108F20000000E780605A2A84979501009385459058
:108F3000177501001305856E97600100E780A00D8D
:108F4000A285179501001305659B97600100E780D6
:108F5000800C294597600100E780C010B705CB0061
:108F60009385757D680097100000E780E05FA2851B
:108F7000680097300000E780804701478146700015
:108F8000CA85268597200000E780608305CD2A8466
:108F9000979501009385C58917750100130505682C
:108FA00097600100E7802007A2851795010013054F
:108FB000A59597600100E7800006294597600100AC
:108FC000E780400A8320C1100324811083244110CC
:108FD000032901105161828097D7FF1F938707D81B
:108FE00018429C43797122D406D60348070083C8EF
:108FF00007012A8483D6450003554600639608017D
:1090000083D82701638DD802238807010507239998
:10901000D7003708CC00DC4B1308787D3ACC130717
:10902000F5FF42CA23080100231EE100231FD100DF
:1090300099C7080832C62EC482973246A2452285B7
:1090400097000000E78080EBB25022544561828097
:1090500079713146977501009385054D280006D634
:1090600097600100E780C0EF97A7FF1F83D74739BC
:10907000231B0100231C0100231D0100231E0100EE
:10908000231F010099E3C167FD17231AF10097A779
:10909000FF1F83D7073791EB97D7FF1F938707CC25
:1090A0009C439C43DC4783D7070097A6FF1F93860A
:1090B0002635231BF100D84E83D74600231CF10030
:1090C0005C4B91CB97A7FF1F83C7F73381EB9700CA
:1090D0000000E780C0DCB25045618280FD1717A612
:1090E000FF1FA302F6320356070183C706014C4750
:1090F0002800230FF10097300000E780602C97D7FD
:10910000FF1F9387A7C59C4301479786010093865D
:10911000A67B884330004C0897100000E780206A47
:109120005DD975B799C9B7E7040003A30705A14541
:1091300017D5FF1F0345C5C2028382805C4EDC4BFE
:10914000B9CFB1CD411122C4177501001305054DEA
:109150002E84978501009385E57206C6976001000D
:10916000E78060EBA285178501001305E573976022
:109170000100E78040EA294597600100E78080EE22
:10918000B7E704002244B24003A3870517D5FF1FA9
:10919000034505BD130640069145410102838280C7
:1091A000411122C417A4FF1F130444231C4C06C6FC
:1091B00089C7DC4399C34C488297584CB7E70400F1
:1091C000BC57484B82975C4CB240224423AA07000C
:1091D0004101828017A7FF1F13074722834707001B
:1091E0009306F00B850793F7F70F63E9F60097A650
:1091F000FF1F2385F620034507008280930700F8B0
:10920000FDB78357450099E37D558280011122CC3B
:1092100017A4FF1F1304C41E5C4C4AC84EC6DC4B87
:1092200052C406CE26CA56C2B2892E8A2A898DC752
:10923000B7E70400FC5F829797D7FF1F938707B0BB
:109240009C431307301FB307F54071556375F7064C
:1092500097000000E780A0C49307D00D7D5563EC14
:109260003705B7E4040093878900B858832AC401FE
:10927000139507014181029723AAAA00484C584937
:1092800021E7978501009385E55D177501001305BA
:10929000E53897600100E78000D8178501001305C5
:1092A000656997600100E78000D729459760010054
:1092B000E78040DB5D55F2406244D2444249B24906
:1092C000224A924A0561828013874900B705CF0080
:1092D0002319E5009385757D310597100000E7801F
:1092E000A028484C83456900310597300000E7808D
:1092F0000010484C4E86D285310597300000E7803B
:10930000200C7146CA8517A5FF1F1305650F9760CE
:109310000100E780E0C4FC5C82970326C90097D770
:10932000FF1F23ADA7A011CABC4C854517D5FF1F51
:10933000034505A382970145BDBF97000000E78064
:1093400060D1D5BF411106C622C426C217D4FF1F63
:10935000130404A197000000E78060B4B7E40400A0
:10936000FC4C0345040085458297034504002244D4
:1093700003A3C405B2409244A145410102834111B7
:1093800026C297D4FF1F9384649D9C4006C622C4C6
:109390004AC0D5C3DC43C5C35CC12300B5002A84E1
:1093A000978501009385454717750100130505272B
:1093B00097600100E78020C6294597600100E7809B
:1093C00060CA9C4023A4070023A2070097A7FF1FA1
:1093D0009387C700DC4FDC4B91C7295597000000ED
:1093E000E78040DC97A7FF1F93878701DC4FDC4BAA
:1093F00089C797000000E78020F537E9040083273C
:10940000C905894517D5FF1F034585958297832791
:10941000C905914517D5FF1F0345859482979C4048
:1094200003A347016309030022852244B24092440A
:10943000024941010283B24022449244024941015F
:1094400082800111328506CE22CC26CA2E84973026
:109450000000E7806007AA84978501009385053F97
:10946000177501001305851B97600100E780A0BAFE
:10947000030784000356640083554400A6861785BD
:1094800001001305E54497600100E780C0B8294555
:1094900097600100E78000BD97A7FF1F83C767F4AF
:1094A000639D9700014597000000E780A0CF8145AC
:1094B0000A8597000000E780C0ECF2406244D24485
:1094C000056182806D7123248110232611102322CF
:1094D000911093F745002E84638707143C083EC023
:1094E000B707E5003EC23C083EC42317010023181D
:1094F000010023190100231A0100231B010097A773
:10950000FF1F83D7A7ED99E3C167FD172316F1006D
:1095100097A7FF1F83D7A7EC91EB97D7FF1F9387E0
:10952000E7839C439C43DC4783D7070017A7FF1FB3
:109530001307C7EA2317F100544F83574700231836
:10954000F100DC4AA1E79785010093856534177522
:1095500001001305A50C97600100E780C0AB1785DB
:1095600001001305A54397600100E780C0AA2945C3
:1095700097600100E78000AF134544008320C110CD
:1095800003248110832441105161828097A7FF1F1B
:1095900083C737E52555D9C3FD1717A6FF1FA302BB
:1095A000F6E403D6060183470701CC460A85230B60
:1095B000F10097300000E780A0E097C7FF1F938776
:1095C000E7799C4317A7FF1F130747E19786010020
:1095D0009386062D88430A866C0097100000E7806A
:1095E000001EAA8451D9978501009385652A1775B5
:1095F00001001305A50297600100E780C0A1A685C0
:10960000178501001305453A97600100E780A0A087
:10961000294597600100E780E0A4268597000000B7
:10962000E78040B891BF93F725009DC7B7E70400D6
:10963000BC47414681452808829725559700000080
:10964000E78040B628089305F00F97000000E780F8
:1096500040D3134524001DB793F7150081CB970025
:109660000000E780209F1345140009BF93F7850091
:10967000014589D717A7FF1F0347F7D897A7FF1FF3
:10968000938707D80DC3D84F584B11CF37E7040045
:10969000384F9047854517C5FF1F0345656C0297F6
:1096A00013458400E1BD97F0FFFFE780407FCDBF09
:1096B0005C4D411106C688C317C7FF1F2320F76AF8
:1096C000B7E7040083A70708170500001305C5DFE7
:1096D0008297B24097C7FF1F2384A76801454101C5
:1096E000828001113335A000A307A100B7E7040071
:1096F00083A7471706CE1306F100854513055030A2
:109700008297F240056182808280411122C406C6A0
:1097100097B7FF1F83C757B0054489EF97C7FF1F4F
:1097200083C7C7EF014499E717B4FF1F0344C4AED2
:1097300013441400228597000000E780C0FA1785C3
:1097400001001305252D09E4178501001305852D5A
:109750002244B2404101176301006700C38B797155
:1097600022D4A30F010037E404008327841726D2F4
:109770004AD006D6AA842E89130550309305F101EC
:1097800032C6829732468347F10193150601C181A3
:1097900085CB01452EC697000000E780C0F48327E3
:1097A0004417B2454A8626858297054597000000F2
:1097B000E78060F3B250225492540259456182808E
:1097C000832744174A8626858297EDB741119397E0
:1097D000050122C406C626C2C1872E8463D40702AF
:1097E000B7E40400FC5417A5FF1F034565C4829726
:1097F00019C1BC5482972165218DB2402244924404
:109800004101828093F715008DC7B7E7040083A755
:10981000471A17A6FF1F1306A6C097C5FF1F9385FB
:10982000E55417A5FF1F0345A5C0829713451400F3
:10983000E9B793F725000145E9D397C7FF1F83C711
:10984000675485E7B7E7040003A8871A1307401F8A
:1098500097A7FF1F83C7C7BD8146130640069945DA
:1098600017C5FF1F0355855102981345240071B792
:1098700097C7FF1F83D787506398A70217C7FF1F9B
:10988000231FB74E17C7FF1F231CC74E17C7FF1F45
:109890002319D74E2E86178501001305251FBE8577
:1098A0001753010067002377178501001305851FF3
:1098B000176301006700038E0357450097C7FF1F1A
:1098C00083D7C74B6318F702C167F91717C7FF1F84
:1098D0002326F74A97C7FF1F23A4074A97C7FF1FEE
:1098E000238C074897C7FF1F238E074817030000E4
:1098F0006700E3E1178501001305C51A176301002E
:10990000670043897D15954763E2A71C178701000F
:109910001307C70E0A053A951C41011122CC06CE49
:10992000BA972E8482871785010013052518976042
:109930000100E7802086A1A203C725009947631193
:10994000F7022E8597000000E78040F7834564000A
:10995000178501001305851697500100E780A06B5D
:1099600097B7FF1F238A078A178501001305C516BD
:109970007DBF03C7250095476319F702C16717C765
:10998000FF1F0357A73FF91703D5A5006309F70287
:10999000B7E7040083A7C71782971785010013054F
:1099A000A51497500100E780E07E854717B7FF1F99
:1099B0002304F78617850100130585158DBF97C70A
:1099C000FF1F239DA73A83D7E50097C6FF1F239863
:1099D000F63A83D7050197C6FF1F2393F63A83D73C
:1099E000250197C6FF1F239EF63897C7FF1F2385C3
:1099F0000738631BE502B7E70400BC4F096613068E
:109A00000690894517A5FF1F034585A28297035637
:109A1000E4008355A400178501001305250E975017
:109A20000100E780405F51B79307700F2316F100E4
:109A3000B7E7040083A7870D17A6FF1F0346469FBD
:109A40006C0082974DF9854717C7FF1F2306F73231
:109A50005DB7178501001305650CD1BD83C52500D1
:109A600091476392F502178501001305A50C9750E5
:109A70000100E780207297000000E78040C9F240B3
:109A800062440561828099476392F50222859700BE
:109A90000000E780A0E283456400178501001305FC
:109AA000E50197500100E7800057D1BF9547639AC1
:109AB000F50083471400E1F3178501001305C5097C
:109AC000BDB5178501001305A509E1BF8280375791
:109AD000315F97A7FF1F9387E796130777D598C342
:109AE0009356C50017870100130707F7BA9683C579
:109AF000060093568500BD8ABA9603C606009356A3
:109B00004500BD8A3D89BA962A9783C60600034759
:109B10000700238407002383D700A383E700238261
:109B2000B700A382C70097A7FF1F9387A79223833D
:109B3000B700A383C7002384D700A384E7008280F3
:109B4000411106C697000000E780A0F8B7E70400BF
:109B500083A7871417A6FF1F1306C68ED545014598
:109B60008297B2404D4697A5FF1F9385A58E13059A
:109B700070304101170300006700A3BE6171232408
:109B8000811A37E40400832704082326111A2322AC
:109B9000911A2320211B232E3119170500001305CC
:109BA00025C3829717A9FF1F130989889947854400
:109BB0002300A900231CF100978501009385C5E8C7
:109BC0009307400617750100130545A5231CF108EE
:109BD0002308910097C9FF1F9389A9B497500100EA
:109BE000E780604383D50900178501001305C5E4AC
:109BF00097500100E7802042294597500100E780F7
:109C0000604603D5090097000000E78080EC8327B9
:109C10004417100885451305503082978327441751
:109C200017A6FF1F13060683CD45130570308297D4
:109C3000832744171796FF1F1306C67FB5451305E4
:109C40006030829783274417300889451305103107
:109C5000829783274417300989451305203182975D
:109C6000832744159305000A0D45829783274415E1
:109C70009305000A11458297A305910023069100E0
:109C800002CD23080100230C01008327841630092C
:109C90009145130570408297832784161306B100FF
:109CA00085451305004082978327841670008545FB
:109CB00013051040829783278416300885451305C5
:109CC000204082978327841610088545130550404D
:109CD0008297832704157D558297832744137D55EA
:109CE00082977D5597A0FFFFE780209A8327440C39
:109CF00082979790FFFFE7808075832784141796DB
:109D0000FF1F13062674D545014582978947130620
:109D1000700F814528092306F1009780FFFFE78037
:109D2000003F8D471306000881452808230CF108E1
:109D30009780FFFFE780A03D9147230CF1009767D4
:109D400001009387277F984383C747003AC8230AB7
:109D5000F10097D0FFFFE7808081700085450545C1
:109D600097A0FFFFE780809930099305700F0945A0
:109D700097A0FFFFE78080983008930500080D4505
:109D800097A0FFFFE780809710089545114597A0A1
:109D9000FFFFE780A096C16717C7FF1F130707FEE5
:109DA000F9171CC3232207001795FF1F1305056829
:109DB00097A0FFFFE78060938327C41D17C5FF1F8F
:109DC000130545FA82973C4803450900854582976B
:109DD0008320C11A0324811A8324411A0329011AFA
:109DE0008329C1195D618280C16717C8FF1F0358AD
:109DF000E8F8F9176301F8083DCDB5CD011126CA81
:109E0000B7E4040083A7841222CC2E862315B10068
:109E100006CE2A8401478146ED45428582972AC6AF
:109E200011ED17850100130565C497500100E78007
:109E30006036F2406244D24405618280FC4403569D
:109E4000A100A28582972C0017C5FF1F035505F3BB
:109E500097A0FFFFE780209669DD178501001305B5
:109E600025C297500100E780E03283A7C412ED4578
:109E7000280082977DBF82800DC585471797FF1FF9
:109E8000A30FF75A9797FF1F238C075A35469795CC
:109E9000FF1F9385255A13056030170300006700E4
:109EA000438C9797FF1FA38C0758E9BF97C7FF1FE5
:109EB00083C747EDA9EFC16717C7FF1F035707EC1B
:109EC000F9176306F7044111854722C417C7FF1F1E
:109ED000230AF7EA37E404007C4C06C68945179547
:109EE000FF1F0345E55482970323841A2244B2409E
:109EF0009797FF1F83C7C75317C5FF1F035505E873
:109F00001307401F814631469945410102838280F3
:109F10006D71232481102326111023229110328485
:109F200001CD8947630AF5028320C1100324811003
:109F3000832441105161828017850100130505C3F8
:109F4000AE8497500100E780E024A285268597B073
:109F5000FFFFE780606AC9BFB7E70400FC4728003D
:109F6000829717850100130525C197500100E780EE
:109F700060228347810039C41307000B6380E70226
:109F80001387A7051377F70F8D4663EDE602A285C9
:109F9000280097C0FFFFE78040DD79B78547E3F5EC
:109FA00087F8834591001775010013056598B3354F
:109FB000B00097A7FF1F2389B70E97500100E780D5
:109FC00080059DB703479100A207B966D98F138713
:109FD000E6556384E70C636DF7042D671307B755E7
:109FE000638FE708636AF70029671307A755638F34
:109FF000E708A2852800A1BF31671307C75563880A
:10A00000E70635671307D755E395E7FE8947E3FD74
:10A0100087F097000000E780A0E99305E4FFC20500
:10A02000C1811305A1009790FFFFE780601BEDBD84
:10A030003D671306F7556389C706636DF60093867F
:10A04000E665E398D7FAA285280097C0FFFFE7806E
:10A05000E016D9BD9306F766638DD7041307F7772B
:10A06000E399E7F897C0FFFFE780004275BD01461E
:10A07000A285280097C0FFFFE780C0FA75B5A285CA
:10A08000280097C0FFFFE780000879BDA28528005F
:10A0900097C0FFFFE780600741BDA285280097C0F9
:10A0A000FFFFE780A00849B597C0FFFFE780201AAF
:10A0B000A5BD97C0FFFFE780C01FBDB5C16717C52D
:10A0C000FF1F0355A5CBF9176307F500B7E7040099
:10A0D00003A3C7170283828017F3FFFF6700236380
:10A0E0001783FFFFE70203FE2A8408452E89B28901
:10A0F00019C900C1971500009385A58661059730A1
:10A100000100E780600481447D5A97100000E780D9
:10A11000E03963C7A404814497100000E780003A47
:10A1200063C8A40497C7FF1F938707C69C43DC47F7
:10A13000B307F94091872302F4006383090483275E
:10A14000C900B307F4409587A302F4001C4C89C7EB
:10A150009C4799C3228582971783FFFF6700C3F945
:10A160005C44139714008504BA972390470171BF8C
:10A170001C48139714008504BA972390070069BF01
:10A18000832789000547B307F4409587A302F400AD
:10A1900083570400638EE7028DC309476384E70495
:10A1A0000D47E395E7FA978701009387A7EF1CCC4B
:10A1B00097870100938707F011A89787010093877D
:10A1C000E7B51CCC97870100938747B65CC8BDBF35
:10A1D00097870100938787A11CCC978701009387FD
:10A1E000E7A1EDB797870100938787F01CCC97878D
:10A1F00001009387E7F0D9BF95E51783FFFFE702DA
:10A2000003EE004618448347940075839D8B6317C3
:10A21000F70097100000E78060B448C41783FFFF81
:10A22000670023EE82801783FFFFE702A3E913890B
:10A230003500C16442094111AA890144F11413593E
:10A240000901054A2EC697100000E7802026B24576
:10A250006348A400014541011783FFFF6700C3E97C
:10A2600083A7090013171400BA9783D707006388E0
:10A27000B7006394970063742A010504E1B70545AC
:10A28000D9BF1783FFFFE70203E3AA892E89328B28
:10A29000B6843A8ABE8A97A00000E78000FE71C9A2
:10A2A000268597200000E780C00C8D4763E7A70054
:10A2B0007D551783FFFF670083E383DB440097101E
:10A2C0000000E780A0242A8497100000E780402542
:10A2D0009307740031443305850263CDA7029710BC
:10A2E0000000E780A02297100000E78020222A8447
:10A2F00097100000E780C0229307740031443305B3
:10A30000850263C3A70497100000E780202093070D
:10A31000450029A897100000E780802033058502BA
:10A320001307F0179307C017E35FA7FA2D55E3C291
:10A3300077F963040B02D6865286A6854A85972054
:10A340000100E78000BDB5B797100000E780401D11
:10A35000330585029307C5FFD1BF832749001385C5
:10A36000C90083D5270097000000E78000EC61F565
:10A3700081B769553DBF97C7FF1F2399A7A097C70E
:10A38000FF1F938767A0904381470C463307F50072
:10A39000420741836393B700828054461398470075
:10A3A0008507C2962390E600D5B797C7FF1F93870E
:10A3B000A79D9C4303C58700828017C5FF1F0355D7
:10A3C000E59C82801783FFFFE70263D1C167138793
:10A3D000D7FF630BE502636AA700F1176300F5027C
:10A3E00001451783FFFF6700C3D11387E7FF6302AF
:10A3F000E502FD171D8D13351500E5B797500000D8
:10A40000E780A0297D15C5BF97500000E78020FE9A
:10A41000D5BF97500000E78040FCEDB71783FFFFE2
:10A42000E702E3CB4111AA8401442EC69710000035
:10A43000E780C008B2456348A40001454101178385
:10A44000FFFF670003CC9C48131514003E9583570B
:10A450000500E385B7FE0504C9BF034855008146E2
:10A4600093F7F60F63E5070181473E8582805845E3
:10A4700093975600BA9703D727006316B70003D700
:10A480000700E304C7FE8506E1BF83464500014798
:10A490009377F70F63E4D700814711A81C45131683
:10A4A00057000507B29703D60700E313B6FE3E85B3
:10A4B00082801783FFFFE702E3C093170501C1877E
:10A4C00097CAFF1F938A4A8C635BF00883A70A0030
:10A4D000C0479C4703570400198D420541816368BA
:10A4E000F500014422851783FFFF6700E3C01205D2
:10A4F0002A94CDBFDC4713944900014A3E94834718
:10A5000044006341FA02014A834754006349FA0256
:10A510008509C20993D9090183A70A009847E3EB8B
:10A52000E9FCC1B71C4413195A00A6853E994A8517
:10A5300097000000E780C0EE05E1050AC9B75C445A
:10A5400013195A00A6853E994A8597000000E780B6
:10A5500020ED19E1050A4DBFE30C09FA61B7AA84A1
:10A5600081495DBF1783FFFFE70263B71C452A845B
:10A5700081E79307C5001CC51C44231204001CC0BE
:10A580009307F00F63EDB70093F5F50F2285972041
:10A590000000E780C0E51783FFFF670083B6939450
:10A5A0000501C167C18063F9F500A6852285972062
:10A5B0000000E780E0E8C5B7C18193F5F50F22857B
:10A5C00097200000E780A0E2A68522859720000062
:10A5D000E780E0E3C9B797B7FF1F9387E77A88431F
:10A5E00082801C4599C797B7FF1F23AFA778014505
:10A5F00082807D55828097B7FF1F9387E7789843C5
:10A6000083474500484792073E9582801783FFFFA6
:10A61000E702E3AC617100451C183EC6B707800134
:10A620003EC81C183ECA8357440002CE02D002CC5A
:10A63000231EF100834784002A8902D22301F102FC
:10A640003C083ED402D697000000E78000FB835709
:10A6500005002316F10297500000E78040C723074A
:10A66000A1025C4003556400F18313F71700834790
:10A67000F10252055181F99BD98FA307F10297107E
:10A680000100E780607839CDAA840355050097A0C2
:10A690000000E78060BF83D704002AD26800231C33
:10A6A000F10083D72400231DF1001C4803D6470086
:10A6B0008C4397200000E780A0D08347B400CA866F
:10A6C000177601001306064C8117A305F4006C00F1
:10A6D000481097200100E780C0835D611783FFFF6A
:10A6E000670023A22155D5BF1C45B1CF03C5A700E4
:10A6F000894613576500630BD7028D46630ED70258
:10A7000085466300D702130740063305E50203C7F9
:10A71000B700418B15CB83C7B700BD8B3355F540D0
:10A7200082801375F5031307803EC5B7096713755B
:10A73000F50313070771D1BF372709001375F50318
:10A740001307077CD9B7014582801783FFFFE70213
:10A75000039903A98500630C09048347B900AE84FB
:10A7600093F7070E85C303459900930520030D81D8
:10A770000505B305B5028844610597300100E780FF
:10A78000C0AC35A02E8597000000E78020F62A8413
:10A7900019CD97000000E780605C8325C900B307EE
:10A7A000B54063FA87002E94B305A440E9F51783FA
:10A7B000FFFF6700039585457DBF1783FFFFE70215
:10A7C00003922A8403D50500011132C636C43AC269
:10A7D0002EC002CA02CC02CE97A00000E780C0AA19
:10A7E00082452ACA22852ECC97000000E780E0E04F
:10A7F00003570500231EE10097500000E78020ADBD
:10A80000A24632469247230FA10036874C08B286F3
:10A810002285014697000000E780E0A605611783C6
:10A82000FFFF6700038E1783FFFFE702438B617111
:10A830001C183EC6B70780013EC81C183ECA3C081B
:10A8400000453ED4AA8402CC02CE02D002D202D667
:10A8500097000000E78060DA83570500355923161A
:10A86000F10297500000E78080A62307A10209C4E7
:10A870008357440081EB21594A855D611783FFFFAF
:10A880006700238803556400520551819710010029
:10A89000E78080572A8965D18347B40093F7070E74
:10A8A00099C71305840197300100E780409C8357C6
:10A8B0004400231EF100834784002301F1025C4021
:10A8C00003550900D98313F7070883471102231C96
:10A8D000A10093F7F707D98FA300F102835729004E
:10A8E000231DF1005C40F18313F717008347F10249
:10A8F000F99BD98FA307F10297A00000E780C098C9
:10A900002AD235D9834794006800139757008347AC
:10A91000B400FD8BD98FA305F4001C4803D6470073
:10A920008C4397200000E780A0A9A6871777010035
:10A9300013074725740005464C1026859700000034
:10A94000E78060942A890DD98347B400A685FD8BE2
:10A95000A305F40097000000E78060DF31BF1773A4
:10A96000FFFFE702C377832485FE2A8441112685F1
:10A9700097000000E78080D7834734FF93F7070EE6
:10A980008DCB2AC6268597000000E78060C809CDD8
:10A99000834734FFB245FD8BA309F4FE91C52285A0
:10A9A00097300100E780608A41011773FFFF67005D
:10A9B00043757DD98327C4FF2685829775F5834724
:10A9C00034FF93F7070E91C7228597300100E78087
:10A9D000008A032584FE97000000E78000E5E9B7C0
:10A9E0001773FFFFE702A36C9C4141112A8903C73B
:10A9F000070089472E84935667006380F6040D464E
:10AA00006388C6049307F0076304F7022E85972036
:10AA10000000E78060ABAA848149C16B130C490038
:10AA200097B7FF1F938747369C43984763E4E90431
:10AA300041011773FFFF6700436B03D7450085474C
:10AA4000E3F8E7FE2E8597200000E78040ADE1B7F0
:10AA500003D74500E3FEE7FC2E8597200000E78042
:10AA6000A0A6AA84228597200000E78000A8C2043F
:10AA7000C98C5DB7DC470355A900139A49003E9A7B
:10AA800093170501C187635DF00083570A00639740
:10AA9000A70263E774038327CA00034D5A002DA061
:10AAA000A1672167A98F1307F7EFE374F7FE639798
:10AAB000090097000000E780209161FD85098DB7AE
:10AAC00083278A00034D4A00835DA900035769006C
:10AAD000216A138BC7003AC6814A33CA4D01631EEF
:10AAE0005D0197B7FF1F9387A72A9C43E1DBA286EE
:10AAF0006286814526858297D1B7A1679387F7EF54
:10AB0000930C4BFF63F24703B2455A8597F0FFFF62
:10AB1000E780A0710DC103278B00104709CE1043B9
:10AB20006382C4023107D5BFEE85668597000000B9
:10AB3000E780008F71F993861A0093FAF60F130BD2
:10AB40000B0271BF835644005C43E3E9F6F62285AD
:10AB50003AC697200000E7802081A1679387D70439
:10AB60002A8A035D4400324763E897008347D9008F
:10AB700093E707F8A306F9001C4766852286E2855D
:10AB80008297C1670844FD17337AFA00529508C0CE
:10AB90002312A40125B797B7FF1F9387E71E984399
:10ABA000814715C31447814763FFD500939745003C
:10ABB0004C47BE9519C903C7550081476375E60028
:10ABC000DC451606B2973E85828003C74500814763
:10ABD000E37BE6FE16069C45F5B71773FFFFE70219
:10ABE000634EAA892E8A814497BAFF1F938ACA1995
:10ABF00083A70A00984763E6E4001773FFFF670026
:10AC0000A34FDC471394440001493E9413BB140046
:10AC100083474400634BF900014913BB1400834789
:10AC20005400634FF9008504E1B7084493175900B5
:10AC30005287DA860146A2853E9582990509C9BFE9
:10AC40004844931759005287DA860546A2853E95F7
:10AC500082990509E9B71773FFFFE7024348814569
:10AC600017F5FFFF1305054897B7FF1F239007123D
:10AC700097000000E780A0F61773FFFF67006348A6
:10AC800097B7FF1F938747109C4395C31773FFFF28
:10AC9000E702E344814517F5FFFF1305A54497003C
:10ACA0000000E780C0F31773FFFF670083458280D1
:10ACB0001773FFFFE702034137E404008327841280
:10ACC00041112315E100AE893289368A3A868146E0
:10ACD0000147ED45AA8482972AC621C90356A100DF
:10ACE000D28597400100E780A0278327C413CE8533
:10ACF00026858297058905C98327440D23142101E0
:10AD000001462C00268582972A8401C9B7E70400F2
:10AD100083A7C712ED45280082972285410117734A
:10AD2000FFFF6700633D4944D5B76554FDB75C41FB
:10AD3000FD175CC182801773FFFFE702433AB7E754
:10AD40000400FC5F829795473305F50281450D812C
:10AD50001773FFFF6700E33A1773FFFFE70223381B
:10AD6000B7E70400FC5F829795473305F5020D8134
:10AD70001773FFFF6700E3381773FFFFE7022336FF
:10AD8000B7E7040083A7870B035505008297177365
:10AD9000FFFF670003371773FFFFE70243340355D4
:10ADA00005003287AE861786FF1F0356C67097B51B
:10ADB000FF1F938525FE97000000E780A0EF177323
:10ADC000FFFF670003341773FFFFE7024331B7E764
:10ADD000040083A7C71782971773FFFF67006332CA
:10ADE0001773FFFFE702A32FB7E7040083A78713BA
:10ADF00097B5FF1F938505FA829701451773FFFFEB
:10AE0000670023301773FFFFE702632DB7E70400E5
:10AE100083A7C71F81451785FF1F0355C565829707
:10AE20001773FFFF6700E32D1773FFFFE702232B64
:10AE3000B7E7040083A7871397B5FF1F938585F6AF
:10AE4000829701451773FFFF6700A32B1773FFFF5E
:10AE5000E702E328B7E7040083A7C71F81451785EA
:10AE6000FF1F0355456782971773FFFF670063292C
:10AE70001773FFFFE702A3262E8597800000E78067
:10AE8000C0B297800000E780C0EF1773FFFF670034
:10AE900043271773FFFFE702832497800000E780B2
:10AEA000C0F91773FFFF6700C3255C49E1175CC950
:10AEB0005CC583572501A1072319F50083570501B8
:10AEC000A1072318F5008280F1473305F50297B7F3
:10AED000FF1F938727EF9C433E9582808D47631524
:10AEE000F60803D74600854763F0E7081773FFFFAE
:10AEF000E702E31E368536842E8997100000E7802E
:10AF0000A05C29C98357440093140501C18063E301
:10AF10009704228597100000E780005BFD14231240
:10AF200094009307A0026300F5029307B002630741
:10AF3000F50293079002631FF50022859700010038
:10AF4000E780A08801A80146CA85228597A0000055
:10AF5000E78040B31773FFFF6700A31A228597109D
:10AF60000000E7806007FDB7828097B6FF1F9386D9
:10AF7000A6E59C42014599CF9843D44217B6FF1FDE
:10AF80002324E6E46396D70097B6FF1F23A0E6E4E8
:10AF90001385C7FE82801773FFFFE70243149700F3
:10AFA0000000E780A04B71443305850291459790DE
:10AFB0000000E78000EC11E565551773FFFF67009F
:10AFC000431497B7FF1F23ADA7DE97000000E7806B
:10AFD000E04833058502914597900000E78060E9DD
:10AFE00061DD97B7FF1F23AFA7DC97000000E78064
:10AFF000E04697B7FF1F239FA7DA97000000E7807E
:10B00000E04597B7FF1F2398A7DA9777010093874A
:10B01000A7BC17B7FF1F2323F7DA97070000938712
:10B0200007E917B7FF1F2329F7D8014579B7177329
:10B03000FFFFE702C30AAA8517B5FF1F130585D7CF
:10B0400097100000E780605F1773FFFF6700630BD6
:10B050001773FFFFE702A30897000000E78060FD79
:10B0600097100000E780E05E97B7FF1F9387C7D572
:10B070009C4391CF1387C7FE19CB83D5C7FF17B564
:10B08000FF1F1305E5D497200100E780001C17730C
:10B09000FFFF670003071773FFFFE70243049700F2
:10B0A0000000E780C0EC09CD834785002A8493F730
:10B0B000070499EB0355E50097000000E78080F94D
:10B0C0001773FFFF6700E3038347C500930445013F
:10B0D00017B9FF1F130949CF85E3832709005CC90E
:10B0E00097B7FF1F23A297CE83274900F1FB97B79D
:10B0F000FF1F23AD97CCE9B7FD172306F5006105C7
:10B1000097800000E780A0D98307840063CB070401
:10B110008347840093E707F82304F400B7E70400AB
:10B120009C5F82974205A94741813375F5028347A9
:10B13000840093F707FCC98F2304F4008347D400ED
:10B140003E951C402318A40089CF984319CB834710
:10B15000C4005040814585073305F5024205418111
:10B160000297832709005CC897B7FF1F23AE97C4D7
:10B170008327490089E797B7FF1F23A997C483470F
:10B18000C4009DDF8355040117B5FF1F130545C497
:10B1900097200100E780600B25B71773FFFFE702D8
:10B1A00003F497B7FF1F9387E7E79C470144858324
:10B1B000858B85E3AE84B2853A8697100000E780E0
:10B1C000204F2A8419C597100000E78060458294BB
:10B1D00008CC22851773FFFF6700A3F21773FFFFE8
:10B1E000E70243EE41112E8932C6AA89970000007A
:10B1F000E780C031324713060502CA869705000072
:10B200009385C5CC17B5FF1F1305C5BA970000007D
:10B21000E780E0F82A8425C99304C5009700000060
:10B22000E780E0411946AA85268597100000E7804F
:10B2300020198545268597100000E78000151775B1
:10B240000100130525974E95834505002685971027
:10B250000000E780C0195C4831468145A1075CC801
:10B260005CC483572401E1172319F40083570401B8
:10B27000E1172318F4001C4C3E859770FFFFE78010
:10B2800000E9A3042501228541011773FFFF670030
:10B29000A3E61773FFFFE70283E44111AA842EC6D9
:10B2A00032C497100000E780003A004DB2452246B4
:10B2B000834784000CC050C093F7F70393E707045B
:10B2C0002304F40023180400268597100000E7806B
:10B2D000203583479400A9462317A40013D73700CD
:10B2E00005073307D7029D8B85072306F400A306C5
:10B2F000E40083C70401D8488507230FF7FE17B77A
:10B30000FF1F130767AC5843232A04009307440127
:10B3100029E317B7FF1F232BF7AA17B7FF1F232512
:10B32000F7AA17B4FF1F1304A4AA228597200100CF
:10B33000E780E0E31C44858B5D8D19E5814522851E
:10B3400097200100E78060F041011773FFFF67005D
:10B3500043DB1CC317B7FF1F232AF7A6D9B7177300
:10B36000FFFFE702C3D797050000938565B7014546
:10B3700097000000E78000B001451773FFFF6700EA
:10B3800043D81773FFFFE70283D597000000E780DB
:10B3900080B01773FFFF6700C3D68347C500A5E3DE
:10B3A0001773FFFFE702A3D32A840355E500970034
:10B3B0000000E78000C821C18347840093F7F7FBB2
:10B3C0002304F4001C4091C7DC4381C74C40014575
:10B3D000829797000000E78080B917B5FF1F13051B
:10B3E000259F97200100E78080E80355E40097003F
:10B3F0000000E78020C61773FFFF670083D08280BC
:10B400001773FFFFE702A3CD97B7FF1F9387C79B73
:10B4100097050000938565C817B5FF1F1305459B69
:10B4200023A0070023A2070097200100E780C0D1D6
:10B430001773FFFF6700E3CC1C4D91CFDC4381CF36
:10B440001773FFFFE702A3C98345070082971773AD
:10B45000FFFF670003CB828097B7FF1F9387879911
:10B460009C4303C50700828097B7FF1F9387879887
:10B470009C4303C51700828097B7FF1F9387879768
:10B480009C4303C52700828097B7FF1F9387879649
:10B490009C4303C54700828097B7FF1F938787951A
:10B4A0009C4303C53700828097B7FF1F938787941B
:10B4B0009C4303C55700828097B7FF1F93878793EC
:10B4C0009C4303C56700828097B7FF1F93878792CD
:10B4D0009C4303C57700828097B7FF1F93878791AE
:10B4E0009C4303C58700828097B7FF1F938787908F
:10B4F0009C4303C59700828097B7FF1F9387878F70
:10B500009C4303C5A700828097B7FF1F9387878E50
:10B510009C4303C5B70011E11D45828097B7FF1F0B
:10B520009387478D9C4303C5C700828097B7FF1F51
:10B530009387478C9C4303C5D700828097B7FF1F32
:10B540009387478B9C4303C5E700828097B7FF1F13
:10B550009387478A9C4303D50701828097B7FF1FD3
:10B56000938747899C4303C52701828097B7FF1FB4
:10B57000938747889C4303D54701828097B7FF1F75
:10B58000938747879C4303D56701828097B7FF1F46
:10B59000938747869C4303D58701828097B7FF1F17
:10B5A000938747859C4303C5A701828097B7FF1FF8
:10B5B000938747849C4303C5B701828097B7FF1FD9
:10B5C000938747839C4303C5C701828097B7FF1FBA
:10B5D000938747829C4303C5D701828097B7FF1F9B
:10B5E000938747819C438857828097B7FF1F938733
:10B5F00067809C4303D5C702828097A7FF1F93876C
:10B60000677F9C4303D5E70219E11305800C828014
:10B6100097A7FF1F9387077E9C4303C5070382807C
:10B6200097A7FF1F9387077D9C43C85B828097A7DE
:10B63000FF1F9387A77B8843828097A7FF1F93876D
:10B64000277B8843828019E17D558280F5DE984210
:10B6500065DFFDD917B7FF1F1307C79C1847AA87D7
:10B660007155058B631D072403C507001547E37D4E
:10B67000A7FC03C737001305F0057D171377F70FF5
:10B68000E364E5FC03C35700E30003FC83C86700E1
:10B69000E38C08FA03C77700494579171377F70F4A
:10B6A000E364E5FA03C7A70011481305F7FF137514
:10B6B000F50FE36BA8F803CE97000D481305FEFFC6
:10B6C0001375F50FE362A8F803C8B7006309080013
:10B6D00065181378F80F1305600DE36705F703C5C8
:10B6E000C700794879151375F50FE36FA8F403C8FF
:10B6F000D7000D457D181378F80FE36705F503D8DB
:10B700000701930E40175118420813580801E3ED42
:10B710000EF303C8E7007D181378F80FE36605F30E
:10B7200003C827017D181378F80FE36F05F103C8EC
:10B730008700C54E75181378F80FE3E70EF103D8AC
:10B740006701856E938EBEE06D184208135808019C
:10B75000E3EC0EEF03D847016D18420813580801B7
:10B76000E3E40EEF03D88701791842081358080163
:10B77000E36C05ED03C8A7017D181378F80FE365A6
:10B7800005ED03C5B7011D487D151375F50FE36D74
:10B79000A8EA03C5D701714879151375F50FE3655C
:10B7A000A8EA03D5E7011308E00F7D1542054181A2
:10B7B000E36CA8E803C50702494879151375F50F2E
:10B7C000E364A8E8C85301C937C834005915130801
:10B7D00058BFE36BA8E603A8870237C534001305FA
:10B7E00055BF5918E36205E717A5FF1F2322C5605F
:10B7F00003C6050117A5FF1F232EF55E0545E3755A
:10B80000C5E403D82501D04933760603E31E06E2DA
:10B8100003C61501E30A06E217A6FF1F2328B65C3C
:10B8200083C5270001466387A50003C61700F145BD
:10B830003306B60283C707039305C00272971A073F
:10B840001307C70516031A9796084697B387B702DA
:10B8500041553E973297420741836362E80617736A
:10B86000FFFFE702C387368597800000E780806B83
:10B8700097000100E780004B2A8497A00000E78032
:10B88000605D2A9497F00000E78040292A94979001
:10B890000000E78080842A9497F0FFFFE780E06F44
:10B8A0002A9497400000E78000972A949770000040
:10B8B000E780809F22951773FFFF67008384828053
:10B8C0001773FFFFE702A3814111A307A10097A00F
:10B8D0000000E78080C89305F100170500001305FC
:10B8E000E5B597F0FFFFE780802F01454101177311
:10B8F000FFFF670003811763FFFFE702C37B17A405
:10B90000FF1F1304247203288400795993681800D8
:10B9100097A4FF1F23AC147113781800631008025A
:10B92000BA84BE89368B328A2E89AA8A97F0FFFFA5
:10B93000E780E0A77D15269519E531594A851763FB
:10B94000FFFF6700C37A97F0FFFFE78040A67D15F1
:10B950002695A167E353F5FE97B7FF1F938787A34B
:10B9600098433E8C814B01CB014597F00000E78066
:10B970000047933B15004A85DA865686D285979014
:10B980000000E780A0502A8911CD1C44F99B17A71D
:10B99000FF1F232DF76883270C00CDD3E3800BFA1C
:10B9A000829769BF268597A7FF1F23AF076697F089
:10B9B000FFFFE780809C4146CE8517A5FF1F13053A
:10B9C000E56F97300100E780A05997D00000E7802D
:10B9D000209C0325040B97D00000E780E09F0545DD
:10B9E00097D00000E780E0A6054597000000E780BB
:10B9F00060EDA9B797A7FF1F9387C7629C47858B08
:10BA0000EDC71763FFFFE702836D17A5FF1F13053F
:10BA1000256997A7FF1F23A7076097A7FF1F23A5E7
:10BA2000076097A7FF1F23A3076097200100E78007
:10BA3000008497500000E780C0F897100100E7806D
:10BA4000804F97100100E780805597A7FF1F9387CD
:10BA5000E75B9C4391C7054597800000E780202362
:10BA600097A7FF1F938747449C4399C741657D155E
:10BA700097700000E78020A597F00000E780C040A5
:10BA800097D00000E780609297A7FF1F9387876E8B
:10BA90009C43139717016356070097F00000E78057
:10BAA000E0AF97A7FF1F23AB076097A7FF1F23A94E
:10BAB000076097A7FF1F23A7076097A7FF1F23A56E
:10BAC000076097000000E780008C97000000E78087
:10BAD000A07597F0FFFFE780401897F00000E7801F
:10BAE00020D91763FFFF6700C361828097A7FF1FFC
:10BAF000938747538843828097A7FF1F9387875276
:10BB0000C8438280B7E7B0009387075063E1A7027C
:10BB100097A7FF1F93870751D843FD576367E50039
:10BB200097A7FF1F23A2A75081473E858280B95760
:10BB3000EDBF1763FFFFE702835A97800000E7809D
:10BB4000A07497800000E78000771763FFFF67000D
:10BB5000435B1763FFFFE702E3562A849304140252
:10BB600001112E85B289A685214636C63A899730BD
:10BB70000100E780803C0DE9B24638082686CE8574
:10BB80001305940497500000E780A04021462C083C
:10BB90004A8597300100E780403A1335150005616A
:10BBA0001763FFFF670043550145D5BF1763FFFFCC
:10BBB000E702E3529305450617A5FF1F1305C523AA
:10BBC00097100100E78060681763FFFF6700635309
:10BBD0001763FFFFE702A35041112EC697F0FFFF46
:10BBE000E780C017B24588C141011763FFFF6700B6
:10BBF00043511763FFFFE702E34CAA842E8497802A
:10BC00000000E780406BAA898545228597000000E7
:10BC1000E780E07D83C7E4011389940899E31389E1
:10BC20000403CE85228597000000E780407C2146F2
:10BC300093051902228597000000E780607897A796
:10BC4000FF1F9387273E8C43228597100000E780D3
:10BC5000C082214693858402228597000000E780F8
:10BC600020761763FFFF670023491763FFFFE70292
:10BC70008344397197F00000E78020B493054006B3
:10BC800061E997800000E780405F6302051497A791
:10BC9000FF1F83C7271813B7170097A6FF1F238B13
:10BCA000E616014499CFC16417A9FF1F130989370C
:10BCB0009309400EFD1497000000E7802083634243
:10BCC000A40A97F0FFFFE78060094169B7290900DE
:10BCD000096AFD7A2A8B81447D199389F97B130ABD
:10BCE0000A71938A8AC797000000E780208063D793
:10BCF000A4041304400EB387840217A7FF1F130781
:10BD000067320324070B3E948357C4016382270BD9
:10BD100018403307EB4063EAE90083474400850796
:10BD2000B3874703D6976365F70801468145094500
:10BD300097F0FFFFE780C04AAA8B29E597400000F3
:10BD4000E780C08285476317F5068965938505718D
:10BD500017A5FF1F1305450A97100100E780E04E65
:10BD600095A0B30734030327090BBA9703D7C7017C
:10BD70006308970003C75700A38207002382E700E8
:10BD8000050415BF9305C500228597000000E780D4
:10BD900080E65E852286976501009385E5E297F04F
:10BDA000FFFFE780404F5E8597100000E780608AC4
:10BDB000850415BF97A7FF1F9387C7269C478D83D0
:10BDC000858BC1F721611763FFFF6700433201468E
:10BDD0008545094502D002D202D402D697F0FFFF72
:10BDE000E7800040AA8479DD97F00000E780209C7E
:10BDF0001389C4002A8481454A8597000000E780A2
:10BE0000005F0C4041464A8597000000E780405B98
:10BE1000832944006385090C4E8502D802DA02DCCE
:10BE200002DE97300100E78020382ACE1410054644
:10BE30002C0808184ECC97500000E780200A137594
:10BE4000F50F51ED8355840093E525004A85970051
:10BE50000000E780E05E11460C104A859700000064
:10BE6000E7800056014697650100938565D62685D3
:10BE700097F0FFFFE7802042268597000000E780CB
:10BE8000407D5C40A1D3014685450D4597F0FFFFFD
:10BE9000E7800035AA841DD548401389C400973037
:10BEA0000100E78060302AC64A8597000000E780DD
:10BEB000404C3246636FC5004C404A8597000000F5
:10BEC000E780005001468145268597F0FFFFE78017
:10BED000803C268597000000E780A077E5B5835574
:10BEE0008400ADB71763FFFFE702631F97A7FF1F2B
:10BEF000938747139C471DC193E7870017A5FF1F32
:10BF0000130585EF17A7FF1F2322F71297100100D3
:10BF1000E78080311763FFFF6700A31EDD9B17A733
:10BF2000FF1F2325F71097300000E78020647DF184
:10BF300017A5FF1F130545EC97100100E78020337C
:10BF4000D1BF1763FFFFE70203174169AA892E8A51
:10BF5000B28A368BBA8B814417ACFF1F130C8C0C42
:10BF6000930C400E7D1997F0FFFFE780205863C4C3
:10BF7000A40001443DA03384940383270C0B3E941A
:10BF80008357C401638627055A87D6865286CE8595
:10BF90001305040397000000E780E0BB01C923807C
:10BFA0000B0022851763FFFF670063148347F401CA
:10BFB00085C35A87D6865286CE8513059408970086
:10BFC0000000E78040B909C585472380FB00D1BF49
:10BFD000850451BF835745006380071E1763FFFF29
:10BFE000E702430E01112A8497000000E780C04D4C
:10BFF00009C985476309F50605611763FFFF6700F7
:10C00000A30F97E00000E780407B7DF58357440055
:10C010004947ED9BE392E7FEC1452285970000006A
:10C02000E7804033AA84228597000000E780204FF4
:10C030000357440002CE91472A89631AF7002285EC
:10C0400097000000E780A0513C082ACC3ECE97E044
:10C050000000E780C0755C55C5D374084A86A68584
:10C060000545829751BF03574400D147E3F6E7F8EF
:10C07000032A0400C169014997AAFF1F938A8AFA1B
:10C08000130B400EFD1997F0FFFFE7802046634F2A
:10C09000A90E2285032A040097000000E780C04211
:10C0A000A1452A89228597000000E780A02AAA845A
:10C0B000228597000000E780804A14402A86AA89DA
:10C0C00078082685CA8597000000E780C0E7AA8423
:10C0D00005D503C7F40189476315F7008347C101FC
:10C0E00081DF5546D2851385640097300100E780D3
:10C0F00020E7014597800000E780001901C583D73C
:10C10000C401A5E797A7FF1F9387C7F19C479355E5
:10C110001900858913D73700058B01CF8983858B5B
:10C120006399B70001452EC697000000E780C0DB89
:10C13000B2454E8597800000E780A01E0346C101EE
:10C140002A8493751900268597900000E78020398E
:10C1500035C1268597800000E7802018268511C00C
:10C16000014597800000E780404B97300000E78052
:10C17000E03F8547E312F5E883C754001307F00F4B
:10C18000E38CE7E68507A382F400BDB5B304690339
:10C1900083A70A0BBE9483D7C401638B370155462E
:10C1A000D2851385640097300100E78000D955DD02
:10C1B0000509D1BD5DD86DB782801763FFFFE70227
:10C1C00063F097800000E780400B05C1C164014423
:10C1D00017A9FF1F130909E59309400EFD1497F0F5
:10C1E000FFFFE780A030634EA40017A5FF1F1305D3
:10C1F000A5C097100100E78020031763FFFF6700C9
:10C20000A3EF330534038327090B3E958357C501FC
:10C21000638897002312050097800000E780E00BF9
:10C22000050475BF97A7FF1F9387C7DF9C478D83C2
:10C23000858B8DE31763FFFFE70263EA17A5FF1FF6
:10C24000130585BB97100100E78060021763FFFFAD
:10C25000670023EB82801763FFFFE70243E897053F
:10C2600000009385C5A017A5FF1F1305E5B897101B
:10C270000100E78060ED1763FFFF670083E8176345
:10C28000FFFFE702C3E58841B7E70400BC5B050593
:10C2900042054181829709C585472300F5000505C0
:10C2A0001763FFFF6700E3E583C7F5FF2E8585076A
:10C2B000A38FF5FE828083C7F5FFFD1793F7F70F75
:10C2C000A38FF5FE99EF1763FFFFE70243E1B7E79E
:10C2D0000400BC571385F5FF82971763FFFF6700C3
:10C2E00043E282801C41035745008D8FBA951CC1E3
:10C2F0002312B5003E85828093D78500A2051441A4
:10C30000DD8D835745001387E6FF18C18907231287
:10C31000F50013D685004111238FB6FEA38FC6FE0C
:10C320004101828018419307F7FF1CC183574500E4
:10C3300085072312F500A30FB7FE828083574500BF
:10C340008D8F2312F5001C41BE950CC12E85828075
:10C35000AA8703D7470008410D8FAA952392E700CB
:10C360008CC38280184108453305A74082808357DB
:10C370004500035765001D8F1C4108453385A740C4
:10C380003305A74082801763FFFFE70243D54111C1
:10C390002EC62A8497000000E780A0FDB245637393
:10C3A000B50001A0835744000840BE952312B40095
:10C3B0003E9541011763FFFF6700A3D41763FFFF9A
:10C3C000E702E3D141112E84B28532C69700000006
:10C3D000E780A0FB3246A28597300100E78040B895
:10C3E00041011763FFFF6700C3D11763FFFFE70237
:10C3F00003CF2E84854597000000E78000F92300D5
:10C4000085001763FFFF6700C3CF1763FFFFE702D5
:10C4100003CD41112317B100894597000000E78043
:10C42000C0F68347E1002300F5008347F100A30035
:10C43000F50041011763FFFF6700A3CC1763FFFFFF
:10C44000E702E3C993D78500A2054111DD8D2317CB
:10C45000B100894597000000E78020F38347E100A1
:10C460002300F5008347F100A300F50041011763A5
:10C47000FFFF670003C91763FFFFE70243C6139777
:10C48000850193D78501C166938606F0D98F13D7AE
:10C490008500758FD98FA2053707FF00F98D4111EF
:10C4A000DD8D2EC6914597000000E78000EE6C0000
:10C4B000114697300100E780A0AA41011763FFFFF2
:10C4C000670023C41763FFFFE70263C11C41854572
:10C4D00003C4070097000000E78080E62285176309
:10C4E000FFFF670003C21763FFFFE70243BF1C4162
:10C4F0004111894503C7070083C717002307E100DF
:10C50000A307F10097000000E78080E30355E100F6
:10C5100041011763FFFF6700C3BE1763FFFFE70218
:10C5200003BC1C414111894503C7070083C717009D
:10C530002307E100A307F10097000000E78040E037
:10C540008357E100410113D58700A2075D8D4205A5
:10C5500041811763FFFF6700C3BA1763FFFFE7025C
:10C5600003B80C4141112A8411466800973001003C
:10C57000E780009F9145228597000000E78040DC1E
:10C58000B247C166938606F01397870113D58701DA
:10C59000598D13D78700758F598DA2073707FF0074
:10C5A000F98F5D8D41011763FFFF670083B51C455F
:10C5B000BE950CC18280AE87944391E6584101EF4D
:10C5C0000CC15CC1828003C7570013671700A382A8
:10C5D000E700B687D5B70CC3EDB7AA87084119CDD8
:10C5E0001841D44398C36313D500D8C32A870346A0
:10C5F00057009376160081E623200700828094433B
:10C6000081CA8C4203A847008CC363930601CCC344
:10C61000799A14C3A302C7003687D1BF1C45DC47F3
:10C620001D8DB777DBB6938777DB09853305F50278
:10C63000420541818280F147B385F50248452E9538
:10C6400082808347450085072302F50082801763B7
:10C65000FFFFE702C3A82A8409E41763FFFF67000E
:10C6600043AA83474400F5DBFD1793F7F70F230236
:10C67000F400E5F71C4403D7270005072391E700E2
:10C68000DC4399C3228582974C4889CD8347540067
:10C69000898B99E71C4422859C479C439C47829741
:10C6A000232A04000040232004007DB71763FFFF06
:10C6B000E702E3A28357250041112EC681EB014416
:10C6C000228541011763FFFF6700A3A303570500FD
:10C6D0008147F146E305F7FEB385D702404585075C
:10C6E0002E948345440008C4F5F5B247AA8481E737
:10C6F000232A040009A81C456C0022859C439C4306
:10C70000829748C84DDD85472312F400B2472320A5
:10C710000400231804002319F4005C485CC483D788
:10C720002400FD172391F40061BF1763FFFFE702A8
:10C73000039B9797FF1F9387276E88432326050047
:10C7400023240500410597100100E78040B21763DC
:10C75000FFFF6700039B1763FFFFE70243981794EF
:10C76000FF1F1304646B1C40411199CF9C472300A9
:10C77000B5002AC65CC197000000E78040FB1C4062
:10C78000DC4399C33245829741011763FFFF67007D
:10C7900043970347450029E3584DAA877D551DCF90
:10C7A0001763FFFFE702A3931CC3DC479796FF1FA5
:10C7B00023A4E666F156130507012390D7009705D9
:10C7C00000009385050297100100E780E09701457E
:10C7D0001763FFFF6700E3927D55828082801763B5
:10C7E000FFFFE702C38F0111614681452800976072
:10C7F000FFFFE780C0919797FF1F9387E7619C43F6
:10C8000028009305F00FDC473EC697000000E78044
:10C81000C0F405611763FFFF6700A38E9797FF1FA2
:10C820009387875F9C43D847A1679387C702631E9E
:10C83000F70A397106DE22DC26DA80004AD84ED6A5
:10C8400052D456D23285B28497000000E780C0C728
:10C85000AA89268597000000E78020C92318A4FC38
:10C86000268597000000E78040C82319A4FC268590
:10C8700097000000E78060C783D744000A8A231A24
:10C88000A4FC858393F7F70F230EF4FC8607BD07FE
:10C8900093F7073F3301F1408A8A01498347C4FD7A
:10C8A0006367F902CE85130584FC232C54FD9700A1
:10C8B0000000E78080EA5281130104FCF2506254C8
:10C8C000D2544259B259225A925A21618280268505
:10C8D00097000000E78060C193171900D6970509FB
:10C8E0002390A7001379F90F55BF82809797FF1FF8
:10C8F000938787529C43D847A1679387A702631AFF
:10C90000F70A397106DE22DC26DA80004AD84ED6D4
:10C9100052D456D23285B28497000000E780C0BA64
:10C92000AA89268597000000E78020BCFD572318C0
:10C93000A4FC26852319F4FC97000000E780E0BAE8
:10C9400083D744000A8A231AA4FC858393F7F70F40
:10C95000230EF4FC8607BD0793F7073F3301F14030
:10C960008A8A01498347C4FD6367F902CE851305AE
:10C9700084FC232C54FD97000000E78000DE5281E8
:10C98000130104FCF2506254D2544259B259225A53
:10C99000925A21618280268597000000E780E0B4EA
:10C9A00093171900D69705092390A7001379F90F5B
:10C9B00055BF82809797FF1F938707469C43D847B0
:10C9C000A16789076310F70A397106DE22DC26DACF
:10C9D00080004AD84ED652D456D23285328997003A
:10C9E0000000E78060AEAA894A8597000000E780D2
:10C9F000C0AF835749000A8A2318A4FC858393F7A4
:10CA0000F70F230CF4FC8607BD0793F7073F3301AC
:10CA1000F1408A8A8144834784FD63E7F402CE852E
:10CA2000130584FC232A54FD97000000E780E0D220
:10CA30005281130104FCF2506254D2544259B2594B
:10CA4000225A925A216182804A8597000000E7802D
:10CA5000C0A993971400D69785042390A70093F458
:10CA6000F40F55BF82809797FF1F9387E73A9C4347
:10CA7000D847A1679387E704631EF70A397106DE7A
:10CA800022DC26DA80004AD84ED652D456D23285DD
:10CA9000B28497000000E78020A3AA89268597002A
:10CAA0000000E78080A42318A4FC268597000000DE
:10CAB000E780A0A3231AA4FC268597000000E78046
:10CAC000C0A283D744000A8A2319A4FC858393F764
:10CAD000F70F230EF4FC8607BD0793F7073F3301DA
:10CAE000F1408A8A01498347C4FD6367F902CE8514
:10CAF000130584FC232C54FD97000000E780E0C55B
:10CB00005281130104FCF2506254D2544259B2597A
:10CB1000225A925A21618280268597000000E78080
:10CB2000C09C93171900D69705092390A700137985
:10CB3000F90F55BF82809797FF1F9387E72D9C437E
:10CB4000D847A1679387C704631AF70A397106DECD
:10CB500022DC26DA80004AD84ED652D456D232850C
:10CB6000B28497000000E7802096AA892685970066
:10CB70000000E7808097FD572318A4FC2685231A20
:10CB8000F4FC97000000E780409683D744000A8AAF
:10CB90002319A4FC858393F7F70F230EF4FC860773
:10CBA000BD0793F7073F3301F1408A8A0149834764
:10CBB000C4FD6367F902CE85130584FC232C54FD64
:10CBC00097000000E78060B95281130104FCF25025
:10CBD0006254D2544259B259225A925A21618280E7
:10CBE000268597000000E780409093171900D6979C
:10CBF00005092390A7001379F90F55BF82809797F5
:10CC0000FF1F938767219C43D847A167DD07631700
:10CC1000F7041753FFFFE702834C797132853284A2
:10CC200097000000E780408A2AC62285970000000E
:10CC3000E780A08B2311A102228597000000E780E6
:10CC4000A088B2452300A102280897000000E780D1
:10CC5000C0B045611753FFFF6700A34A82809797D2
:10CC6000FF1F9387671B9C43D847A167938787045F
:10CC70006317F7041753FFFFE702634679713285A4
:10CC8000328497000000E78020842AC6228597001E
:10CC90000000E78080852311A10222859700000013
:10CCA000E7808082B2452300A10228089700000097
:10CCB000E780A0AA45611753FFFF67008344828085
:10CCC0009797FF1F938747159C43D847A167938782
:10CCD000A7046312F7021753FFFFE7024340011155
:10CCE0002800814597000000E78020A705611753C1
:10CCF000FFFF6700034182809797FF1F9387C7114B
:10CD00009C43D847A167938757026319F7021753CB
:10CD1000FFFFE702C33C0111328597F0FFFFE78078
:10CD2000A07A2308A1008145280097000000E78031
:10CD3000C0A205611753FFFF6700A33C828097974D
:10CD4000FF1F9387670D9C43D847A1679387E7022E
:10CD5000631BF7041753FFFFE702633801113285A5
:10CD6000328497F0FFFFE7804078AA84228597F00D
:10CD7000FFFFE7808077854709E9228597F0FFFF6D
:10CD8000E78080744205B337A0002800814523184E
:10CD900091003ECA97000000E780209C0561175370
:10CDA000FFFF6700033682809797FF1F9387C706B0
:10CDB0009C43D84799476313F7081753FFFFE702CF
:10CDC000033279713285328497F0FFFFE780C06FBC
:10CDD0002AC6228597F0FFFFE78020712310A10269
:10CDE000228597F0FFFFE780206E2301A1022285B4
:10CDF00097F0FFFFE780406DA301A102228597F025
:10CE0000FFFFE780606C2302A102228597F0FFFFFD
:10CE1000E780806B2313A102228597F0FFFFE78054
:10CE2000A06AB2452314A102280897000000E780F9
:10CE3000C09245611753FFFF6700A32C828097972C
:10CE4000FF1F938767FD9C43D847A1679387C7035C
:10CE50006313F7081753FFFFE702632879713285E0
:10CE6000328497F0FFFFE78020662AC6228597F07C
:10CE7000FFFFE78080672310A102228597F0FFFF64
:10CE8000E780A0662311A102228597F0FFFFE780CB
:10CE9000A0632302A102228597F0FFFFE780C06212
:10CEA000A302A102228597F0FFFFE780E061230340
:10CEB000A102228597F0FFFFE7800061B245A3033E
:10CEC000A102280897000000E780208945611753D8
:10CED000FFFF6700032382801753FFFFE702232031
:10CEE00001112A8497F0FFFFE780005EAA84228563
:10CEF00097F0FFFFE780605F228597F0FFFFE780F4
:10CF0000C05E035744008D4763F7E700228597F022
:10CF1000FFFFE780805D228597F0FFFFE780E05C00
:10CF20002800A68597000000E7802083056117533D
:10CF3000FFFF6700031D9797FF1F9387E7ED9C4353
:10CF4000D847A167FD07631FF7001753FFFFE702EC
:10CF50000319328597000000E78040F81753FFFF60
:10CF60006700231A82809797FF1F9387E7EA9C4305
:10CF7000D847A167E5076315F7081753FFFFE702D6
:10CF8000031679713285328497F0FFFFE780C05332
:10CF90002AC6228597F0FFFFE7802055228597F06B
:10CFA000FFFFE78080542310A102228597F0FFFF46
:10CFB000E780A053520551812311A102228523024B
:10CFC000010297F0FFFFE7802050A302A102228513
:10CFD00097F0FFFFE780404F2303A102228597F0DF
:10CFE000FFFFE780604EB245A303A102280897F037
:10CFF000FFFFE780807645611753FFFF67006310EE
:10D0000082809797FF1F938727E19C43D847A167AA
:10D010009387E703631FF7001753FFFFE702230C13
:10D02000328597000000E78060EB1753FFFF670031
:10D03000430D82809797FF1F938707DE9C43D84755
:10D04000A16793874704631EF7021753FFFFE702A8
:10D05000030979713285328497F0FFFFE780C0467B
:10D060002AC6228597F0FFFFE7802048B2452808AE
:10D0700097F0FFFFE780606E45611753FFFF670081
:10D08000430882809797FF1F938707D99C43D8470F
:10D09000A167938787026310F7041753FFFFE70226
:10D0A000030479713285328497F0FFFFE780C04135
:10D0B0002AC6228597F0FFFFE7800041B245230092
:10D0C000A102280897F0FFFFE78020694561175308
:10D0D000FFFF6700030382801753FFFFE70223006F
:10D0E000011197F0FFFFE780203EAA85280097F006
:10D0F000FFFFE780806605611753FFFF670063004D
:10D100009797FF1F938747D19C43D847A167D107C3
:10D11000631FF7001753FFFFE70263FC3285970098
:10D120000000E780A0FB1753FFFF670083FD8280AC
:10D130009797FF1F938747CE9C43D847A167C507A2
:10D14000631FF7001753FFFFE70263F9328597006B
:10D150000000E780A0F81753FFFF670083FA828082
:10D160009797FF1F938747CB9C43D847A167B90781
:10D17000631FF7001753FFFFE70263F6328597003E
:10D180000000E780A0F51753FFFF670083F7828058
:10D190009797FF1F938747C89C43D847A167AD0760
:10D1A000631FF7001753FFFFE70263F33285970011
:10D1B0000000E780A0F21753FFFF670083F482802E
:10D1C0009797FF1F938747C59C43D84789476318A4
:10D1D000F7021753FFFFE70283F00111328532C8CF
:10D1E00097F0FFFFE780402EAA85280097F0FFFF09
:10D1F000E780A05605611753FFFF670083F0828028
:10D200009797FF1F938747C19C43D847A1678D0716
:10D210006311F7041753FFFFE70263EC0111328536
:10D22000328497F0FFFFE780202A13066100AA846A
:10D230004C00228597300000E78000232800A68557
:10D2400097F0FFFFE780605105611753FFFF67000C
:10D2500043EB82809797FF1F938747BC9C4381CF06
:10D26000DC4391CB1753FFFFE70263E78297175325
:10D27000FFFF670003E982801753FFFFE70223E601
:10D2800079713C08AE843ED2A165B7070A002A84B2
:10D290003ED448103C08DD053ED636C432C63AC2FC
:10D2A00097D0FFFFE780402C12474810BA8597F0CF
:10D2B000FFFFE780C01332464810B28597F0FFFFAA
:10D2C000E780E014A2464810B68597F0FFFFE7809C
:10D2D0000012501001478146A685228597D0FFFF96
:10D2E000E780E04D45611753FFFF670083E1175367
:10D2F000FFFFE702C3DE01117C000329C501AE84F4
:10D300003ECAA165B70707002A843ECC48087C00C6
:10D31000C5053ECE97D0FFFFE78000258345D900A5
:10D32000480897F0FFFFE780800C500801478146CE
:10D33000A685228597D0FFFFE780604805611753D7
:10D34000FFFF670003DC1753FFFFE70243D983C7E2
:10D35000950093F7F707A384F50097000000E78096
:10D3600040F91753FFFF6700C3D91753FFFFE702C8
:10D3700003D779713C08AE843ED2A165B707090096
:10D380002A843ED448103C08938545043ED632C6D4
:10D3900036C497D0FFFFE780201DA2464810B6850F
:10D3A00097F0FFFFE780A00432464810B28597F05F
:10D3B000FFFFE780C005501001478146A685228502
:10D3C00097D0FFFFE780A03F45611753FFFF67003D
:10D3D00043D31753FFFFE70283D083C79500411162
:10D3E0002A8493F7F707A384F50032852EC697F0B9
:10D3F000FFFFE780800F85672AC46370F50297708E
:10D400000000E78060E82246B24509ED11478146F9
:10D41000228597000000E78060E641011753FFFF77
:10D42000670023CE01478346F501DDB71753FFFFA1
:10D43000E70243C901113C003ECAB7070A003ECCCF
:10D440003C003ECE83C79500AA89328593F7F70743
:10D45000A384F5002E8497F0FFFFE780000985671D
:10D46000637DF504A165AA8493858504480897D057
:10D47000FFFFE780600F268597700000E780C0E01F
:10D480002A8929E19145480897F0FFFFE78020F6B7
:10D49000A685480897F0FFFFE78060F7CA8548082F
:10D4A00097F0FFFFE780A0F4014781465008A2856E
:10D4B0004E8597D0FFFFE780803005611753FFFF4F
:10D4C000670083C38145480897F0FFFFE78020F29B
:10D4D0000349090275BF1753FFFFE702A3BE797125
:10D4E0001C103ECAB7070F003ECC404D1C10AA844A
:10D4F000AE894808994532C636893ECE97D0FFFF9F
:10D50000E780800632464808B28597F0FFFFE78043
:10D5100000EE630C0902A545480897F0FFFFE7807D
:10D52000C0E62546CA8597200100E78060A3500821
:10D5300001478146CE85268597D0FFFFE7802028CA
:10D5400045611753FFFF670023BB8355C40248089A
:10D5500097F0FFFFE780A0EB0355E402814505C586
:10D56000854785456301F502C167FD179305F00FF7
:10D57000630BF5007D1597700000E780608D9305C3
:10D58000150093F5F50F480897F0FFFFE78020E6B8
:10D5900083450403480897F0FFFFE78040E5834593
:10D5A0001403480897F0FFFFE78060E483552403E5
:10D5B000480897F0FFFFE78080E58355440348085B
:10D5C00097F0FFFFE780A0E49DB71753FFFFE70246
:10D5D00003B183C795008146014693F7F707A384FB
:10D5E000F50097000000E78040EF1753FFFF67004A
:10D5F00043B11753FFFFE70283AE79713E841C10DD
:10D600003ECA2E89B7070F00A1653ECCFD051C1050
:10D61000AA84480842C03AC23ECE36C432C697D029
:10D62000FFFFE78060F432464808B28597F0FFFFBD
:10D63000E780E0DBA2464808B68597F0FFFFE78069
:10D6400000DD12474808BA8597F0FFFFE78020DC2D
:10D650000248630C08029145480897F0FFFFE780F5
:10D66000C0D21146A28597200100E780608F500844
:10D6700001478146CA85268597D0FFFFE7802014A1
:10D6800045611753FFFF6700C3A78945480897F016
:10D69000FFFFE78080CF834704002300F500834726
:10D6A0001400A300F500E1B71753FFFFE70283A1C1
:10D6B00083C7950001112A8A93F7F707A384F50021
:10D6C0003285AE8432C697F0FFFFE78000E2324633
:10D6D0002A89328597F0FFFFE78000DF8567637353
:10D6E000F902AA894A8597700000E780E0B92A8488
:10D6F00019ED114781464A86A6855285970000009C
:10D70000E780C0B705611753FFFF6700E39E93876B
:10D71000E9FF93F7F70F0547E366F7FE8347F50147
:10D7200095EB8947E380F9FE8346F4015285014772
:10D730004A86A68597000000E78040B4A167D90714
:10D7400048083ECC230A010002CE97000000E78083
:10D75000A0B04DBF639EE7008947639EF900930721
:10D760001020231FF50097700000E78000B76DBF01
:10D770000947E39BE7FA8D47E398F9FA228597700A
:10D780000000E780C0DE9797FF1F938727889C43A0
:10D7900099E79787FF1F938727719C4399C703D504
:10D7A000040097800000E780E0CD231F040022855D
:10D7B0005DBF1753FFFFE702839201113C003ECA91
:10D7C000B7070B003ECC3C003ECE83C795002A89AC
:10D7D000328593F7F707A384F500AE8497F0FFFF37
:10D7E000E780A0D093170501C187635AF006A165B1
:10D7F0002A849385E502480897D0FFFFE780C0D6CA
:10D80000A285480897F0FFFFE78060C09787FF1F59
:10D81000938787699C43A9EB01449375F40F4808EB
:10D8200097F0FFFFE780A0BC9355844093F5F50F78
:10D83000480897F0FFFFE78080BB9355044193F5BC
:10D84000F50F480897F0FFFFE78060BA014781466F
:10D850005008A6854A8597D0FFFFE78040F605610E
:10D860001753FFFF6700E389416585460546A2859A
:10D870007D1597500000E780A0BC59DD5105970049
:10D880000100E780C08E130440063344850271B75F
:10D890001753FFFFE702A3840111B70706003EC636
:10D8A00083C7950021642A8993F7F707A384F500BD
:10D8B000AE8428009305A4040AC40AC897D0FFFFC9
:10D8C000E78080CA300001478146A6854A8597D007
:10D8D000FFFFE780C0EE97E0FFFFE780E011130451
:10D8E0009404480822CC230A010002CE97000000CD
:10D8F000E780809605611753FFFF67008380174319
:10D90000FFFFE702237CC1642A8901449789FF1F36
:10D9100093894971130A8002FD1497E0FFFFE780A5
:10D92000E0BD6347A40001451743FFFF6700C37CC8
:10D93000B307440303A7C90ABA9703D707006306CE
:10D94000970083D72700638427010504F9B70545AD
:10D95000E1BF1743FFFFE702E3762A8A2E8999C1C8
:10D9600023A0050081498144978AFF1F938A4A4B6F
:10D97000614B97E0FFFFE780A0BE63C7A4004E8520
:10D980001743FFFF670043773384640383A70A00CC
:10D990003E948357040099E763040900232089001B
:10D9A0008504C1BF4146D28513054400971001008C
:10D9B000E780A05875F5A289E5B71743FFFFE70296
:10D9C000637039717C083ED4B7070A003ED67C08E4
:10D9D0003ED883C795002A8A328593F7F707A38438
:10D9E000F5002E8932C697F0FFFFE78000B085670B
:10D9F0006373F5083246AA84328597F0FFFFE7800B
:10DA0000A0AC8547AA8963E8A706A165938585042C
:10DA1000281097D0FFFFE78020B52685977000007B
:10DA2000E78080862A8429ED9145281097F0FFFF32
:10DA3000E780E09BA685281097F0FFFFE780209DF8
:10DA4000CE85281097F0FFFFE780609A0147814656
:10DA50003010CA85528597D0FFFFE78040D6A16776
:10DA60009387770448183EDC230A010202DE97F010
:10DA7000FFFFE780607E21611743FFFF6700C367F8
:10DA80008145281097F0FFFFE7806096A685281053
:10DA900097F0FFFFE780A0979797FF1F9387478F27
:10DAA0009C4381CB22856389090097D00000E780E1
:10DAB00080238345040271B797D00000E7800022DD
:10DAC000CDBF1743FFFFE702E35F83C79500411116
:10DAD000AA8993F7F707A384F5003285AE84328ACA
:10DAE00097F0FFFFE78060A08567637FF5022A89D2
:10DAF00097600000E78040792A84914631C58347CA
:10DB0000F50105476387E70291C70D476366F70490
:10DB1000AD461DA89305050303250A00414697104D
:10DB20000100E78080410DE941011743FFFF6700D5
:10DB3000A35C9305950803250A0041469710010050
:10DB4000E780A03F814669F54A86A6854E85970005
:10DB50000000E780C081C9BF83250A00130594082F
:10DB600097700000E780E02819C1C146F1BF978790
:10DB7000FF1F9387A7499C4399E79787FF1F9387C8
:10DB8000A7329C4399C7228597800000E78060896F
:10DB900069FD8547A30FF400228597B00000E78058
:10DBA000A083228597600000E78020734E85814620
:10DBB0004A86A68597F0FFFFE780607BA167938781
:10DBC000570448003EC42302010002C697F0FFFF3D
:10DBD000E780806891BF1743FFFFE702C34D83C70B
:10DBE00095004111AA8993F7F707A384F5003285C0
:10DBF0002E89B28A97F0FFFFE780208F85676374D4
:10DC0000F50EAA8497600000E78000682A840DED75
:10DC1000416B014A978BFF1F938BCB40130C400E37
:10DC20007D1B19A833048A0383A70B0B3E948357EB
:10DC3000C40163836705050A97E0FFFFE780008B57
:10DC4000E342AAFE95460DA08357C501639697024D
:10DC50009305050303A50A00414697100100E780DC
:10DC6000C02D994611E181462686CA854E8597F0DA
:10DC7000FFFFE780C06F85A883A50A001305040392
:10DC800097700000E780E016C14679FD2285231ECB
:10DC9000940097A00000E780207422859760000020
:10DCA000E780A0639787FF1F9387876E9C43A9C374
:10DCB00023000402228597D00000E78080EF4E8584
:10DCC00081462686CA8597F0FFFFE780406AA167F4
:10DCD0009387070448003EC42302010002C697F060
:10DCE000FFFFE780605741011743FFFF67002340B4
:10DCF00089472300F402E1B7397106DE22DC4AD8F5
:10DD0000800052D456D25AD026DA4ED65ECE2E8A13
:10DD100032892A8B97D0FFFFE780407A060571058C
:10DD200041998A8A3301A140232224FC231404FC54
:10DD300097D0FFFFE780807883479A000605350576
:10DD400093F7F7072315A4FCA304FA004A852326BA
:10DD500024FC97E0FFFFE780407993170501C18716
:10DD60006340F0025681130104FCF2506254D25415
:10DD70004259B259225A925A025BF24B2161828077
:10DD8000AA844A8597E0FFFFE7802076AA894A8522
:10DD900097E0FFFFE7806075A1659385C5022A893A
:10DDA000130544FC97C0FFFFE780007C268597C0E1
:10DDB000FFFFE7804070854511C94A86CE8597C030
:10DDC000FFFFE780C069AA8B21E98945130544FC60
:10DDD00097E0FFFFE780A061A685130544FC97E06C
:10DDE000FFFFE780C062CE85130544FC97E0FFFF8C
:10DDF000E780E061CA85130544FC97E0FFFFE780F8
:10DE0000006101478146130644FCD2855A8597D0AC
:10DE1000FFFFE780C09AB9B78145130544FC97E03E
:10DE2000FFFFE780C05CA685130544FC97E0FFFF79
:10DE3000E780E05DCE85130544FC97E0FFFFE780B7
:10DE4000005DCA85130544FC97E0FFFFE780205C76
:10DE5000814497D0FFFFE7806066E3D4A4FA83A7EC
:10DE60000B0113971400BA9783D5070099C51305C2
:10DE700044FC97E0FFFFE78080598504D9BF7971A2
:10DE800006D622D44AD000184ECE52CC56CA26D23C
:10DE90005AC8AE893289AA8A97D0FFFFE78000620C
:10DEA0000605690541990A8A3301A140232A24FC09
:10DEB000231C04FC97D0FFFFE780406083C79900D4
:10DEC00006052D0593F7F707231DA4FCA384F9008D
:10DED0004A85232E24FC97E0FFFFE780006193171B
:10DEE0000501C187634FF0005281130104FDB25058
:10DEF000225492540259F249624AD24A424B456135
:10DF00008280AA844A8597E0FFFFE780005EA165D2
:10DF10009385A5022A89130544FD97C0FFFFE7807A
:10DF2000A064268597C0FFFFE780E058854509C9B2
:10DF3000CA8597C0FFFFE78080552A8B29E1894574
:10DF4000130544FD97E0FFFFE780604AA6851305AF
:10DF500044FD97E0FFFFE780804BCA85130544FD31
:10DF600097E0FFFFE780A04A01478146130644FD82
:10DF7000CE85568597D0FFFFE7806084B5B7814591
:10DF8000130544FD97E0FFFFE7806046A685130573
:10DF900044FD97E0FFFFE7808047CA85130544FDF5
:10DFA00097E0FFFFE780A046814497D0FFFFE7801E
:10DFB000E050E3DBA4FA83270B0113971400BA9710
:10DFC00083D5070099C5130544FD97E0FFFFE7805F
:10DFD00000448504D9BF1743FFFFE702431083477E
:10DFE0004500404DD5EFFD575DC483469400094779
:10DFF0006363D70A0346B400854663EEC60883060A
:10E00000E40063CA06085C45F9562390D700978759
:10E01000FF1F83C727E199E3A304E4009787FF1F4D
:10E02000938787E89C4381E78947A306F400978795
:10E03000FF1F9387E7359C4381E789472306F40058
:10E040009705000093854506AA841305040197F0FF
:10E050000000E780600FFD57231AF40281471CDCA3
:10E0600001489787FF1F23AB87DA9787FF1F9387A6
:10E0700027DB232E040304C0804397D0FFFFE780F3
:10E08000204E61463306C502814522859740FFFF39
:10E09000E780E00781473E851743FFFF670063067F
:10E0A000FD57D5BF1743FFFFE70263032A840355DB
:10E0B000450297600000E780201D19E5231E04003B
:10E0C0001743FFFF6700E3038357E401F5DB930584
:10E0D00004FF17450100130565E997E00000E7809C
:10E0E0002014F9BF1743FFFFE70263FF2E89A165E4
:10E0F00041119385E5032A8436C432C6BE843AC2F0
:10E1000097C0FFFFE780404612472285BA8597E017
:10E11000FFFFE780C02D32462285B28597E0FFFFE2
:10E12000E780E02EA2462285B68597E0FFFFE780D4
:10E13000002E630309029145228597E0FFFFE780E7
:10E14000C0241146A68597100100E78060E14101D7
:10E150001743FFFF6700E3FA8945228597E0FFFF39
:10E16000E780A02283C704002300F50083C71400C2
:10E17000A300F500E9BF1743FFFFE70243F683C79B
:10E180009500444D054793F7F707A384F5001C421B
:10E19000411183C707006367F7062E842A89B1C03F
:10E1A00003C7D400630FF7021787FF1F1307C7CFFA
:10E1B000184305C3A386F40097A00000E7808049B8
:10E1C00083C7D40099E741657D1597400000E7803B
:10E1D000802F83D72403918B89C797E00000E780C5
:10E1E00000134A85A28597F0FFFFE7808010A167A2
:10E1F000C10748003EC42302010002C697F0FFFF9A
:10E20000E780800541011743FFFF670083EF174355
:10E21000FFFFE702C3EC03D745008D47AA844111F5
:10E220002E8432892E8563E3E70297E0FFFFE780C3
:10E23000C02BAA8523000900268597C0FFFFE78031
:10E24000002541011743FFFF6700A3EB97E0FFFFA5
:10E25000E780A0292AC6228597E0FFFFE780E02813
:10E26000B24585472A862300F900268597C0FFFF1F
:10E27000E780E01EF9B7397106DE22DC26DA80007D
:10E280004ED652D456D24AD85AD05ECEAE89B28437
:10E29000AA8A97D0FFFFE7806021060513052502B3
:10E2A00041990A8A3301A140232224FC231404FC4F
:10E2B00097D0FFFFE780801F83C7990006054D05B3
:10E2C00093F7F7072315A4FCA384F90026852326DA
:10E2D00024FC97E0FFFFE780402193170501C187E9
:10E2E0006340F0025281130104FCF2506254D25494
:10E2F0004259B259225A925A025BF24B21618280F2
:10E30000AA8B03AB040097C0FFFFE780C01A51E55A
:10E3100083D7440001498544F11793B71700A3013F
:10E32000F4FC834734FCA165C9C79385E504130554
:10E3300044FC97C0FFFFE7802023A685130544FC1B
:10E3400097E0FFFFE780A00ADE85130544FC97E015
:10E35000FFFFE780C00B834734FC114691E3094679
:10E36000DA85130544FC97E0FFFFE78060058144F0
:10E37000630A0900416B7D1B97D0FFFFE780001304
:10E3800063CCA40201478146130644FCCE85568522
:10E3900097C0FFFFE780A042B1B7A685130634FC03
:10E3A00097000000E780E0E6933415002A89860490
:10E3B0008DBF9385C504A5BF8327C900139714009B
:10E3C000BA9783D5070063886501130544FC97E07D
:10E3D000FFFFE780C003850445B71743FFFFE7024F
:10E3E00083CD79711C103EC4B7070F003EC61C10C8
:10E3F0003EC883C79500AA8A328593F7F707A3849E
:10E40000F500AE89328497E0FFFFE780000E931796
:10E410000501C187635AF0062A8A228597E0FFFF2B
:10E42000E780A00C2A895285032B040097C0FFFFC8
:10E43000E780600839ED8357440081440544F117B3
:10E4400093B71700A303F10083457100DA87228791
:10E45000CA865286280097000000E780E0C801477E
:10E4600081463000CE85568597C0FFFFE780203576
:10E47000A1679387D70348083ECC230A810026CEA4
:10E4800097F0FFFFE78040DD45611743FFFF67001E
:10E4900003C6A2851306710097000000E78060D7CD
:10E4A000AA84094455D13544E30055FB4A8597F0C9
:10E4B000FFFFE78000450D4441D9014497D0FFFF9D
:10E4C000E780C0FE634DA400C16B0144FD1B97D0E3
:10E4D000FFFFE780A0FD634EA4001544B5B7DC4400
:10E4E00013171400BA9783D7070063832703050423
:10E4F000F1B7D84493171400BA9703D70700631BEA
:10E50000770123902701268597A00000E780C0DAD5
:10E5100001441DBF050465BF1743FFFFE70283BA2F
:10E5200083C7950041112A8A93F7F707A384F50062
:10E5300032852E89328497E0FFFFE78000FB931736
:10E540000501C1876353F006AA89228597E0FFFF82
:10E55000E780A0F92311A1004E85832A040097C00B
:10E56000FFFFE78040F539E58357440085440144C7
:10E57000F11793B71700A300F100034811000357E8
:10E580002100D6875285CE862686CA8597F0FFFF62
:10E59000E7806006A167F10748003EC423029100AE
:10E5A00022C697F0FFFFE78020CB41011743FFFF12
:10E5B000670083B4A2851306110097000000E7806E
:10E5C00040C52A84894455D9835721001167854461
:10E5D000BA97C2071167C1831307F7EFE36FF7F824
:10E5E0009787FF1F938787A29C4381CB854513059F
:10E5F000210097500000E780607483552100228538
:10E60000814497C0FFFFE780A0E125D923100500D2
:10E61000228597A00000E78080CC85B71743FFFFD5
:10E62000E70263A983C7950041112A8B93F7F70787
:10E63000A384F50032852E8A328497E0FFFFE780BD
:10E64000C0EA93170501C1876351F006AA8A2285A3
:10E6500097E0FFFFE78060E92A895685832B040055
:10E6600097C0FFFFE78020E531E5835744008144F0
:10E670000544F11793B71700A301F10003483100D7
:10E68000DE875A854A87D6862286D28597F0FFFF95
:10E69000E78060F6A167ED0748003EC423028100D1
:10E6A00026C697F0FFFFE78020BB41011743FFFF1D
:10E6B0006700E3A3A2851306310097000000E780FE
:10E6C00040B5AA8409445DD99167CA97C20711670A
:10E6D000C1831307F7EF0544E362F7FACA8597C0D1
:10E6E000FFFFE780E0D3014451F9814997D0FFFF54
:10E6F000E780C0DC63DBA900984893971900BA97BC
:10E7000003D7070005EF2390270197D0FFFFE7808D
:10E71000E0DA1544E384A9F6268597A00000E78097
:10E7200000BC9787FF1F9387678E9C430144B9D72E
:10E730004A8597500000E780005889B785097DB762
:10E740001743FFFFE702039879713E847C083EC8B7
:10E750002E8AB7071400A1653ECAE5057C08AA8980
:10E76000080836C4428932C6BA8AC6843ECC97C0ED
:10E77000FFFFE78060DFCA85080897E0FFFFE780BA
:10E7800000C732460808B28597E0FFFFE78020C83F
:10E79000A246630A09049D45080897E0FFFFE78049
:10E7A000C0BE1D4681459740FFFFE78040966389C4
:10E7B0000A089145080897E0FFFFE78000BD114671
:10E7C000A68597000100E780A079100801478146DF
:10E7D000D2854E8597C0FFFFE78060FE45611743F5
:10E7E000FFFF67006391B685080897E0FFFFE780A9
:10E7F00000C21C400808D8439355C70185891207F9
:10E800005183B205D98D97E0FFFFE78040C01C40DF
:10E81000080883C5870097E0FFFFE78040BD1C40E4
:10E82000080883C5A70097E0FFFFE78040BC1C40B5
:10E83000080883C5970097E0FFFFE78040BB85BFCE
:10E840008945080897E0FFFFE78020B483C70400EC
:10E850002300F50083C71400A300F500BDB71743DC
:10E86000FFFFE702238683C795004111AA8993F72A
:10E87000F707A384F5003285AE84328497E0FFFF6A
:10E88000E780A0C693170501C187635DF0042A895C
:10E89000032A040097C0FFFFE780E0C119E983570E
:10E8A00044000548F11793B71700A307F10081460C
:10E8B00031A81306F100A28597000000E78060955B
:10E8C0001DC51C459DC783D6470001480347F1007D
:10E8D00093078500D2884A86A6854E85970000005A
:10E8E000E78040E641011743FFFF6700E3800948E6
:10E8F0007DBF1D486DBF1733FFFFE702A37C657125
:10E900005C083EC4B7077B013EC65C083EC883C7AF
:10E9100095002A8A328593F7F707A384F500AE891C
:10E9200097E0FFFFE78040BA8357E100E1C78945E0
:10E93000280097C0FFFFE78020C38145280097E0AB
:10E94000FFFFE780C0AA97C0FFFFE78000C9978755
:10E95000FF1F9387E7A39C431774FF1F0344844C56
:10E96000AA843334800099C3136424009777FF1F6F
:10E97000938787539C4399C3136444009777FF1F81
:10E980009387C7689C4399C31364840083D50400AC
:10E990002800014997E0FFFFE78060A783D52400A6
:10E9A000280097E0FFFFE78080A683D54400280079
:10E9B00097E0FFFFE780A0A597D0FFFFE78000ABBF
:10E9C00093150501C181280097E0FFFFE78020A48F
:10E9D000A285280097E0FFFFE78060A39C44636066
:10E9E000F902014781463000CE85528597C0FFFF6E
:10E9F000E780E0DC59611733FFFF6700E36FDC4419
:10EA00001314490028003E9497E0FFFFE7806096CA
:10EA1000834744000347540089070607BA978607CF
:10EA2000E36AF5FC835524002800814A97E0FFFF44
:10EA3000E780E09D83454400280097E0FFFFE780E2
:10EA4000009B83455400280097E0FFFFE780209A51
:10EA50008347440063C9FA00814A8347540063C175
:10EA6000FA020509A5BF1C4413975A002800BA975B
:10EA700083D50700850A97E0FFFFE7804099C9BF6B
:10EA8000032BC40093975A0028003E9B83552B000C
:10EA9000850A97E0FFFFE780809783550B002800E9
:10EAA00097E0FFFFE780A0964DBF1733FFFFE70217
:10EAB00003635C4993E717005CC997A00000E780F7
:10EAC00060B51733FFFF6700C3631733FFFFE7022B
:10EAD00003612E84814597F0FFFFE780C0E705C5FD
:10EAE00083570500FD172310F50009C4835725003F
:10EAF0002310F40097000000E78060FB0145173306
:10EB0000FFFF6700036031457DD823100400C5BFB7
:10EB10001733FFFFE702035B83C7950041112A8A81
:10EB200093F7F707A384F50032852E89328497E0A6
:10EB3000FFFFE780809B93170501C1876356F006AE
:10EB4000AA89C145228597E0FFFFE780A0802A8B34
:10EB50004E85832A040097C0FFFFE780C09531E906
:10EB600083574400231101000544F11793B71700A0
:10EB7000A300F10081440348110003572100D68708
:10EB80005285CE862286CA8597F0FFFFE780A0A631
:10EB9000A1679387170248003EC42302810026C65E
:10EBA00097E0FFFFE780406B41011733FFFF6700ED
:10EBB000A35413061100A28597F0FFFFE78060655C
:10EBC000AA8409E523110100094475B793052100C2
:10EBD0005A8597000000E78080EF835721002A8440
:10EBE000D9DB9777FF1F938767429C4381CB85458D
:10EBF0001305210097500000E78040148355210041
:10EC00002685314497C0FFFFE78080812DD52310F2
:10EC10000500268597900000E780606C0144A1BF45
:10EC20001733FFFFE702A34B41112E896C00AA8422
:10EC300002C697F0FFFFE78000D20DC10357050021
:10EC400005072310E50097000000E78040E68147B4
:10EC50003E8541011733FFFF6700A34A32479547BE
:10EC600065DBCA85268597300000E780800CC147A8
:10EC7000E34005FE3244854741462310F4008357A4
:10EC80000900A685130544002311F4009700010034
:10EC9000E780002D228545BF1733FFFFE70283423F
:10ECA00083C795004111AA8A93F7F707A384F5005B
:10ECB0003285AE89328497E0FFFFE78000839317A7
:10ECC0000501C1876356F0062A8AC145228597D07F
:10ECD000FFFFE7802068AA845285032B040097B0C9
:10ECE000FFFFE780407D31E9835744002311010095
:10ECF0008544F11793B71700A300F10001440348BE
:10ED0000110003572100DA875685D2862686CE85E4
:10ED100097F0FFFFE780208EA167938707024800E6
:10ED20003EC42302910022C697E0FFFFE780C05255
:10ED300041011733FFFF6700233CA2851306110032
:10ED400097F0FFFFE780E04C2A8409E523110100DA
:10ED5000894475B726859305210097000000E78058
:10ED600060ECAA8449FD83552100228597B0FFFFFE
:10ED7000E780006B49F5014997C0FFFFE780007409
:10ED8000635DA900184893171900BA9703D70700C5
:10ED90000DEF035721002390E70097C0FFFFE780A6
:10EDA000E071630625039777FF1F938727269C430F
:10EDB00099C70355210097500000E780C0EF2285D6
:10EDC00097900000E780A0511DBF050975B79544D5
:10EDD0003DB705C19307F00F630FF500C547630CFE
:10EDE000F5009307F5FF05453315F5004205418110
:10EDF00082800145828041657D158280B9E91733A3
:10EE0000FFFFE702C32D034506033284970000008D
:10EE1000E78060FC9305803EB305B502C205C18161
:10EE200081CD0357E402854763F8E7001305040129
:10EE300097E00000E78060418357E40241677D1757
:10EE40006385E700FD172317F4021733FFFF670000
:10EE5000432B82801733FFFFE702E325004283C77D
:10EE60009500444D0349140093F7F707A384F50078
:10EE700083470400220911673369F900A167B3478A
:10EE8000F90041112A8BAE8A63ECE70E8347240018
:10EE90001307C00EB91793F7F70F6373F710034703
:10EEA0003400C14763EEE70E834744001307E007D1
:10EEB00093C707086371F70C834984008347740084
:10EEC000A209B3E9F900856763F7F90A034A640008
:10EED000834754004E85220A336AFA009750000097
:10EEE000E780803A61C123962403834B3400137A70
:10EEF000FA00239A340323887403239944039389E3
:10EF00000401631C090023A60402239804024E8511
:10EF100097E00000E780A0353DA0034924004A8522
:10EF200097000000E78020EB2397A402834744006A
:10EF30004E85A388F402E38D0BFCE30B09FC97E0FC
:10EF40000000E780602E97900000E78040728146C5
:10EF50000146D6855A8597E0FFFFE7800058A167F4
:10EF6000938797033EC423020100480002C697E03E
:10EF7000FFFFE780602E41011733FFFF6700231773
:10EF80008544A2862686D6855A8597E0FFFFE780CE
:10EF9000C054A167938797033EC423029100F1B741
:10EFA000BD44C5B79144F1BF1733FFFFE70283119A
:10EFB00001111C08404D3EC2B7070F003EC41C089B
:10EFC0003EC62A89AE8997C0FFFFE78000D7585C0C
:10EFD0001C5C6346B70E6394E50063E2A70E3385BD
:10EFE000A740B3B7A700B305B7401306803E8146DC
:10EFF0009D8D97000100E780C0B693140501C18084
:10F00000A1659385C503480097B0FFFFE780C05511
:10F010008145480097D0FFFFE780603D8355040499
:10F02000480097D0FFFFE780803E835524044800C6
:10F0300097D0FFFFE780A03D814589CCC167FD17D0
:10F040009305F00F6388F400268597500000E78051
:10F0500020E0AA85480097D0FFFFE780403903559C
:10F060004404814501CDC167FD179305F00F630787
:10F07000F50097500000E780A0DDAA85480097D0F2
:10F08000FFFFE780C03683456404480097D0FFFF48
:10F09000E780E03583457404480097D0FFFFE780A0
:10F0A0000035500001478146CE854A8597B0FFFF65
:10F0B000E780E07005611733FFFF6700E3038144D9
:10F0C00081B71733FFFFE702830183C7950093F7EA
:10F0D000F707A384F50097000000E78020ED1733C1
:10F0E000FFFF670003021733FFFFE702A3FD83C79B
:10F0F00095004111404D93F7F707A384F5002A8A44
:10F100003285B284AE8997D0FFFFE780003E2A8B1C
:10F11000268597D0FFFFE780403D2A89268597D036
:10F12000FFFFE780603A93170B0163CA0702E1779C
:10F13000CA97C207C183116763E3E7029307091007
:10F14000C207C1831307B00F637BF7009317090150
:10F15000C187AA8A634AF000C54763FE570141018F
:10F160001733FFFF670043F997B0FFFFE7802025C3
:10F17000E31725FFD5B763080B0263060902814434
:10F1800063890A02B7077F00231064052311240551
:10F190007CC0568597000000E780E0C39304803E62
:10F1A000B304950239A0B7077F00232004047CC074
:10F1B00081440355240497E00000E780E0A2A1C445
:10F1C00097C0FFFFE78060B7269593D7F4413337A8
:10F1D0009500AE97BA9708DC5CDCCE855285970027
:10F1E0000000E780A0DC99E023220404A167938754
:10F1F000B70348003EC42302010002C697E0FFFFA8
:10F20000E7808005A9BF814701481CDC232E040349
:10F21000E9B71733FFFFE70283EC97C0FFFFE780F2
:10F220002034E1473305F502914597500000E7800F
:10F2300040C4E55711C59777FF1F23A3A7BE814799
:10F240003E851733FFFF6700C3EB1733FFFFE7026D
:10F2500003E99777FF1F938767BC80433DC08357BF
:10F2600004046390A70683572404639CB70436897B
:10F27000B28497C0FFFFE78040AC5C5C63C3B70417
:10F280006395B7001C5C63EEA7028347640463F3D5
:10F29000F400A6872303F4048347740463F3970000
:10F2A000A687A303F4048357440441677D1763854D
:10F2B000E70085072312F4043C4481C7CA852685EC
:10F2C00082971733FFFF6700C3E39777FF1F93878A
:10F2D000E7B49C43014599C303C587008280173377
:10F2E000FFFFE702C3DF0111B70707003EC683C770
:10F2F0009500584D0AC493F7F7070AC8A384F50090
:10F300002A89AE8411CB1C4283C707002304F7006F
:10F3100097900000E7800034216493055402280090
:10F3200097B0FFFFE780402497000000E78020FAB5
:10F33000AA85280097D0FFFFE780600B30000147C7
:10F340008146A6854A8597B0FFFFE78040471304B2
:10F350004402480822CC230A010002CE97E0FFFFB6
:10F36000E78080EF05611733FFFF670083D917330C
:10F37000FFFFE702C3D601117C003ECAB7070700B2
:10F380003ECC7C003ECE83C795002E84AA8493F7A2
:10F39000F707A384F500A16593855502480897B047
:10F3A000FFFFE780601C97000000E78040F2AA851D
:10F3B000480897D0FFFFE780800350080147814647
:10F3C000A285268597B0FFFFE780603F0561173370
:10F3D000FFFF670003D39777FF1F938727A49C4302
:10F3E000094599C303C5970082809777FF1F9387CC
:10F3F000E7A29C43094599C303C5D700828097774C
:10F40000FF1F9387A7A19C43014599C303C5A7008C
:10F4100082801733FFFFE702E3CA0111B707080034
:10F420003EC683C79500404D0AC493F7F7070AC844
:10F43000A384F5002A89AE8429C41442854703C7F2
:10F44000060063E0E70A8347940009468149638028
:10F45000C702B307F740A304E400B339F00083C741
:10F4600016002305F40097900000E780A01E0357C4
:10F470002403058B19C76386090097D00000E78035
:10F4800000E9216493058402280097B0FFFFE7801C
:10F49000A00D97000000E78040F4AA85280097D0CF
:10F4A000FFFFE780C0F497000000E78080F5AA85A1
:10F4B000280097D0FFFFE78080F3014781463000A6
:10F4C000A6854A8597B0FFFFE780602F130474027A
:10F4D000480822CC230A010002CE97E0FFFFE78014
:10F4E000A0D705611733FFFF670003C11733FFFF84
:10F4F000E702E3BE01117C003ECAB70708003ECC1C
:10F500007C003ECE83C795002E84AA8493F7F7072C
:10F51000A384F500A16593858502480897B0FFFF95
:10F52000E780800497000000E78020EBAA85480868
:10F5300097D0FFFFE780A0EB97000000E78060EC2A
:10F54000AA85480897D0FFFFE78060EA5008014786
:10F550008146A285268597B0FFFFE780402605619A
:10F560001733FFFF6700E3B99777FF1F9387078B78
:10F570009C43014599C303C5B70082801733FFFF41
:10F58000E702E3B50111B70707003EC683C7950040
:10F59000404D0AC493F7F7070AC8A384F5002A89E7
:10F5A000AE8405C81C42054783C707006368F70699
:10F5B0000347B400630FF700A305F4009790000021
:10F5C000E78040098347B400B9CF97D0FFFFE780B9
:10F5D00000BF21649305B400280097B0FFFFE780C7
:10F5E000A0F897000000E78060F8AA85280097D06F
:10F5F000FFFFE780C0DF014781463000A6854A85CE
:10F6000097B0FFFFE780A01B2904480822CC230AFB
:10F61000010002CE97E0FFFFE78000C405611733C9
:10F62000FFFF670003AE97D0FFFFE780E0BF55B74D
:10F630001733FFFFE702A3AA01117C003ECAB707F8
:10F6400007003ECC7C003ECE83C795002E84AA8462
:10F6500093F7F707A384F500A165AD05480897B0B7
:10F66000FFFFE78060F097000000E78020F0AA85A8
:10F67000480897D0FFFFE78080D7500801478146B0
:10F68000A285268597B0FFFFE780601305611733D9
:10F69000FFFF670003A79767FF1F938727789C43A7
:10F6A000094599C303C5C70082801733FFFFE702EE
:10F6B00003A301117C00AE843ECAA165B707070011
:10F6C0002A843ECCD1057C0048083ECE97B0FFFF8F
:10F6D000E78080E997000000E78020FCAA854808C1
:10F6E00097D0FFFFE780A0D0500801478146A6854C
:10F6F000228597B0FFFFE780800C05611733FFFF7D
:10F70000670023A01733FFFFE702639D83C79500BF
:10F7100093F7F707A384F50097000000E78020F92E
:10F720001733FFFF6700E39D1733FFFFE70283995D
:10F7300083C795000329C501411193F7F707A384F7
:10F74000F5001C4283C90700854763E637079777B2
:10F75000FF1F9387E7C39C432E84AA8485CF97001D
:10F760000000E78080F389476306F502630409021D
:10F770008347C9006380370323063901979000004F
:10F78000E78040ED83572903898B89C797D0000014
:10F79000E780E0B72685A28597000000E78020F18A
:10F7A000A167CD0748003EC42302010002C697E0CE
:10F7B000FFFFE78060AA41011733FFFF6700C39393
:10F7C0009767FF1F938787659C431D4599C303C5B2
:10F7D000E70082801733FFFFE70263900111B7074C
:10F7E00007003EC683C79500584D0AC493F7F70734
:10F7F0000AC8A384F5002A89AE8415C71C4283C7B2
:10F80000070093968701E18663C4060685466381F7
:10F81000D7068346E7006388F6002307F700979032
:10F820000000E78020E321649305E400280097B0FE
:10F83000FFFFE78060D397000000E780A0F8AA856B
:10F84000280097D0FFFFE78080BA0147814630004B
:10F85000A6854A8597B0FFFFE78060F63504480823
:10F8600022CC230A010002CE97E0FFFFE780C09E72
:10F8700005611733FFFF6700C3881733FFFFE702F7
:10F88000038601117C003ECAB70707003ECC7C000E
:10F890003ECE83C795002E84AA8493F7F707A384EE
:10F8A000F500A165B905480897B0FFFFE780C0CB18
:10F8B00097000000E78000F1AA85480897D0FFFF75
:10F8C000E780E0B2500801478146A285268597B0BF
:10F8D000FFFFE780C0EE05611733FFFF670063821B
:10F8E0001723FFFFE702037EAA8401441769FF1F65
:10F8F00013090953E14997C0FFFFE78060C66344DD
:10F90000A400014519A833053403832709003E9557
:10F91000835725006397970011051723FFFF6700A2
:10F92000A37D0504C9BF032E8500630A0E12176369
:10F93000FF1F1303A36D0323030063150300294373
:10F940006390061203234E01631503001D43639960
:10F9500007101723FFFFE7020376C689428A3E8914
:10F96000BA8AB684328BAE8B2A84B5E103554E0039
:10F9700019E501431A851723FFFF67004377A16745
:10F98000A98F116763FBE70097000000E78080F50F
:10F99000814597F0FFFFE78080130844B70700E038
:10F9A0005841F98F18455CC1B707001FF98F1CC576
:10F9B0005C4991C7610597E00000E780408BE38ACE
:10F9C00009FA228597900000E78060C65DB732850E
:10F9D00097C00000E78040430D4349DD1C44116798
:10F9E00003D54700A167A98F63FBE70097000000DC
:10F9F000E78040EF814597F0FFFFE780400D03234C
:10FA0000840093164B01D1828347B30003566300F1
:10FA10008588FD8BA305F300FD777D8E558EFD76E1
:10FA2000FD16B204F18E83274301C58E23127301A4
:10FA30002313D3002304530123052301A30443010B
:10FA4000BDDF228597B0FFFFE78040CAAA85084442
:10FA5000B5D1610597D00000E780207F8DB71D43A9
:10FA60001A8582801723FFFFE702C3650569AA8410
:10FA7000AE89328A0144FD5A7D1997C0FFFFE780A5
:10FA8000E0A26347A40001451723FFFF6700C36698
:10FA9000D84493171400BA9703D70700631F37039E
:10FAA0002390570163070A00268597900000E7809E
:10FAB000A0809C449DC383D76700B3F72701639E52
:10FAC0003701D28801488147014781460146814577
:10FAD000268597000000E78040E5050479BF1723DD
:10FAE000FFFFE702235E79711C103EC4B7070F00C9
:10FAF0003EC61C103EC883C79500AA8A328593F77C
:10FB0000F707A384F5002E89328497D0FFFFE780A2
:10FB1000C09D93170501C187635AF006AA89228503
:10FB200097D0FFFFE780609C2A8A4E85032B040054
:10FB300097B0FFFFE780209839ED83574400814458
:10FB40000544F11793B71700A303F1008345710033
:10FB5000DA872287D2864E86280097E0FFFFE7806B
:10FB6000A058014781463000CA85568597B0FFFFEF
:10FB7000E780E0C4A1679387F70348083ECC230AD7
:10FB8000810026CE97D0FFFFE780006D45611723E7
:10FB9000FFFF67006356A2851306710097E0FFFF21
:10FBA000E7802067AA84094455D1528597E0FFFF7A
:10FBB000E78020D50D4459D90546D2852685970082
:10FBC0000000E78060EA2A8451B71723FFFFE702AD
:10FBD0000351835507000346270041112A842E85CF
:10FBE00032C62EC497E0FFFFE780A0D101C932469C
:10FBF000A245228597000000E78000E74101172316
:10FC0000FFFF670003501723FFFFE702C34A83C7C4
:10FC100095004111AA8A93F7F707A384F50032856E
:10FC2000AE89328497D0FFFFE780208C93170501BF
:10FC3000C1876357F00AC1452A8A228597C0FFFF12
:10FC4000E78040712A8D228597D0FFFFE780E08909
:10FC50002A89228597D0FFFFE7800087930705F860
:10FC600093F7F70F1307E007AA8B637BF70622854C
:10FC700097D0FFFFE78040852A8C228597D0FFFF31
:10FC8000E7808084AA8C5285032B040097B0FFFF85
:10FC9000E780608239E983574400231101008144E1
:10FCA000F11793B71700A300F100054403471100B3
:10FCB00083562100938784005685DA8822885286ED
:10FCC000CE8597F0FFFFE780E0A7A167E90748002E
:10FCD0003EC42302810026C697D0FFFFE780C057AD
:10FCE00041011723FFFF6700834013061100A2851F
:10FCF00097E0FFFFE780E051AA8409E523110100A6
:10FD000009446DB7930521006A8597F0FFFFE780EE
:10FD100060F12A8441FD835521009356C9001316D2
:10FD2000490185486688E2875E87858A51822685F3
:10FD300097000000E78060BF2A848DBF1723FFFF74
:10FD4000E702633783C7950041112A8B93F7F707C2
:10FD5000A384F5003285AE89328497C0FFFFE78027
:10FD6000C07893170501C1876352F00A2A8A228559
:10FD700097C0FFFFE7806077AA8A228597C0FFFFC0
:10FD8000E780A0762A89228597C0FFFFE780C073AD
:10FD9000930705F893F7F70F1307E0072A8C6377AB
:10FDA000F706228597C0FFFFE7800072AA8C2285A4
:10FDB00097C0FFFFE78040712A8D5285832B040096
:10FDC00097A0FFFFE780206F39E583574400854403
:10FDD0000144F11793B71700A301F1000347310065
:10FDE000930784005A85DE882688D6865286CE857B
:10FDF00097F0FFFFE78000958D4748003EC423023F
:10FE0000910022C697D0FFFFE780004541011723EC
:10FE1000FFFF6700C32DA2851306310097E0FFFFA7
:10FE2000E780203F2A84894455D99356C900131688
:10FE3000490185486A88E6876287858A5182D68526
:10FE400097000000E78060AEAA8449BF1723FFFF38
:10FE5000E70243272A8981440144617A916A176B3A
:10FE6000FF1F130BAB1A97B0FFFFE780206563C736
:10FE7000A40022851723FFFF6700032883270900BA
:10FE800093991400CE9703D5070033074501420725
:10FE900041836364570305C103270B0019C78545D8
:10FEA0003E8597400000E78060E98327090005044C
:10FEB000CE972390070085047DB797000000E78068
:10FEC00060A2832709000504CE972390070065D51B
:10FED000814597F0FFFFE78080BFF1BF1723FFFF49
:10FEE000E702431E83C7950041112A8A93F7F7075B
:10FEF000A384F50032852E89328497C0FFFFE78006
:10FF0000C05E93170501C187635AF004AA89832A4A
:10FF1000040097A0FFFFE780005A31E583574400B3
:10FF200085440144F11793B71700A301F10003487A
:10FF30003100D68752850147CE862686CA8597D05E
:10FF4000FFFFE780406BA167F50748003EC423022E
:10FF5000910022C697D0FFFFE780003041011723B0
:10FF6000FFFF67006319A2851306310097E0FFFFCA
:10FF7000E780202A2A8489445DD99767FF1F9387E9
:10FF8000E7089C4381CF044997B0FFFFE780005307
:10FF9000AA85268597400000E78040DA1305040112
:10FFA00097000000E780C0EA228597800000E78084
:10FFB00000338144ADBF1723FFFFE702C30F83C7A0
:10FFC00095004111AA8A93F7F707A384F5003285BB
:10FFD000AE8932842311010097C0FFFFE780E05013
:10FFE00093170501C1876354F0062A8AC14522850B
:10FFF00097C0FFFFE7800036AA8B5285032B0400D1
:020000040001F9
:1000000097A0FFFFE780204B21E9835744008544F8
:100010000144F11793B71700A300F1000348110042
:1000200003572100DA875685D2862686CE8597D05B
:10003000FFFFE780405CA1679387270248003EC42A
:100040002302910022C697D0FFFFE780E020410104
:100050001723FFFF6700A309A2851306110097E08D
:10006000FFFFE780001B2A8489444DD99767FF1F53
:100070009387C7F998433E8901CF044997B0FFFFA2
:10008000E780C043AA85268597400000E78000CB23
:100090001305040197000000E78080DB97B0FFFFA5
:1000A000E780C04195443DD9930521005E8597F0D6
:1000B000FFFFE78020B7AA8435F11C4803572100D1
:1000C00022852390E70097800000E7804021832766
:1000D0000900A9D70355210097400000E780A0BD83
:1000E00035BF1723FFFFE70203FD83C795004111CA
:1000F000AA8A93F7F707A384F5003285AE89328484
:1001000097C0FFFFE780603E93170501C1876351E9
:10011000F0062A8A228597C0FFFFE780003D2A89E2
:100120005285032B040097A0FFFFE780C03831E51C
:100130008357440085440144F11793B71700A30186
:10014000F10003483100DA8756854A87D286268631
:10015000CE8597D0FFFFE780004AA167F9074800E6
:100160003EC42302910022C697D0FFFFE780C00E55
:1001700041011723FFFF670083F7A28513063100B3
:1001800097E0FFFFE780E0082A8489445DD9916702
:10019000CA97C2071167C1831307F7EF8544E3626B
:1001A000F7FA9767FF1F938767E69843BE8B01CFE7
:1001B000044997B0FFFFE7806030AA852685974005
:1001C0000000E780A0B71305040197000000E78056
:1001D00020C897B0FFFFE780602E95443DD11C48B2
:1001E000228581442390270197800000E780200F1B
:1001F00083A70B00B9D74A8597400000E780A0ABE2
:1002000089B71723FFFFE70283ED2A844105B284F3
:1002100097000000E780C0C311C5228597800000C9
:10022000E780E00B81460146A68522859780000085
:10023000E780C04E1C4C89C7DC4799C32285829752
:100240001723FFFF6700E3EB9767FF1F938707BD47
:100250009C43014599C31385070182809767FF1F5F
:100260009387C7BB884382801723FFFFE70223E7FA
:100270009317C600DD8DC2054111C1812A8432C6A3
:1002800097C0FFFFE780A018324622851182937540
:10029000F60F97C0FFFFE780801541011723FFFF8E
:1002A000670023E61723FFFFE702C3E179713C08EB
:1002B0003ED2B7070C003ED43C083ED683C795001B
:1002C000AE842A8993F7F707A384F500A165938587
:1002D0003504481097A0FFFFE7800029C165FD1590
:1002E0000144176AFF1F130AEAD3930A400EAE892E
:1002F0002E8B2EC697B0FFFFE780401F4205931755
:1003000004014181C183B24563E9A702C167FD17BA
:100310006387F500481097C0FFFFE780400F50103B
:1003200001478146A6854A8597A0FFFFE7802049BF
:1003300045611723FFFF670023DC3307540383273E
:100340000A0BBA9703D6C701630A3601638A3501DF
:10035000481097000000E78060F1DA85050451BF7E
:10036000B285EDBF1723FFFFE702E3D479717C0864
:100370003EC8B70711003ECA7C083ECC83C7950033
:10038000AA89328593F7F707A384F5002E8997C0D1
:10039000FFFFE780801585676378F504A165AA846F
:1003A0008905080897A0FFFFE780001C2685974075
:1003B0000000E78060ED133415000A04A2850808E8
:1003C00097C0FFFFE780A002A685080897C0FFFF3F
:1003D000E780E00325CC014781461008CA854E8599
:1003E00097A0FFFFE780A03D45611723FFFF67004F
:1003F00003D0B30754030327CA0ABA9703D70700E9
:10040000631C970003D627006380650508089700E2
:100410000000E780A0E5DE8505042EC697B0FFFF4B
:10042000E780C00D4205931704014181C183B245A5
:10043000E3E1A7FCC167FD17E38FF5F8080897C053
:10044000FFFFE780C0FC41BFB285F9B7C165FD156C
:100450000144176AFF1F130AEABC930A80022E8B1D
:10046000AE8B65BF1723FFFFE70263C718418347C1
:10047000170083460700A207D58FD207D1832390A8
:10048000F50083472700034717008D45A207D98F42
:1004900091832310F60097C0FFFFE78060EA1723DF
:1004A000FFFF670003C61723FFFFE702A3C1C16474
:1004B00001441769FF1F1309E9B693098002FD146F
:1004C00097B0FFFFE78080036347A400014517232F
:1004D000FFFF670063C2330534038327C90A3E95D3
:1004E00083570500E38597FE0504D9BF1723FFFF57
:1004F000E70243BD2A8AAE89B284B68A97400000DB
:10050000E78080D819E591473E851723FFFF6700F4
:10051000A3BE2A894E8597C00000E780E08E2A841A
:10052000638E0A048D476DD103570500C547E31D4F
:1005300047FD0347F9018546AD47E317D7FC8347DD
:10054000450081CF4146A6855D0597F00000E78014
:10055000C09E814755D9AD4745BF130965012302A8
:10056000E500CA85268597100000E780606231C1EA
:10057000A547E38B0AF82302040079B705C1835726
:100580000500E39247F94146A685190597F000005A
:10059000E780A09A81472DD99947BDB74E8597002E
:1005A0000000E78080F02A84954739DD1309550063
:1005B0004DBF4146A6852310440123113401130584
:1005C000190097F00000E780A0992285978000002D
:1005D000E780A0EA81470DBF1723FFFFE70223B0A2
:1005E00079717C003ECCB7070A003ECE7C003ED03D
:1005F00083C79500B2842E8493F7F707A384F50090
:100600001306A1002A892C00268597000000E780A8
:10061000A0E5A16528088D0597A0FFFFE780C0F43D
:1006200090408355A1000355810085469700000046
:10063000E78000ECAA84AA85280897C0FFFFE7801E
:1006400000DB0356A10083558100280897000000B5
:10065000E780C0C1300801478146A2854A8597A03E
:10066000FFFFE780C015854748103ED42302910262
:1006700002D697D0FFFFE78020BE45611723FFFF1A
:10068000670023A81723FFFFE70263A579717C00A9
:100690003ECCB7070A003ECE7C003ED083C7950013
:1006A000B2842E8493F7F707A384F5001306A10004
:1006B0002A892C00268597000000E780E0DAA165F2
:1006C00028088D0597A0FFFFE78000EA904083553A
:1006D000A10003558100814697000000E78040E1BA
:1006E000AA84AA85280897C0FFFFE78040D0035658
:1006F000A10083558100280897000000E78000B71B
:10070000300801478146A2854A8597A0FFFFE78010
:10071000000B48102302910202D402D697D0FFFFAB
:10072000E78080B345611723FFFF6700839D172390
:10073000FFFFE702C39A97000000E78060DB172302
:10074000FFFF6700039C9757FF1F9387676D8843E0
:1007500082801723FFFFE70283988357250041110A
:10076000AE842A842307B10017F5FFFF1305254641
:100770006C002316F10097A0FFFFE780404691C46C
:10078000228597800000E780E0D6FD572310F40013
:10079000130620028145130554009720FFFFE780D0
:1007A000009741011723FFFF6700A3951723FFFF61
:1007B000E702439179717C003ECCB7070A003ECE38
:1007C0007C003ED083C79500AA89AE8493F7F707D3
:1007D0003285A384F5001306A1002C0097000000C9
:1007E000E78080C803558100114497400000E780EE
:1007F000A0A915C50355A100014497B00000E780EA
:10080000A06011CD0357050083578100454463184C
:10081000F700854597000000E780E0F30144216977
:1008200093053900280897A0FFFFE780E0D3A28551
:10083000280897C0FFFFE78080BB0356A1008355BF
:100840008100280897000000E78040A23008014797
:100850008146A6854E8597A0FFFFE78040F64810A9
:100860004AD42302810202D697D0FFFFE780C09EC0
:1008700045611723FFFF670023881723FFFFE70267
:1008800063849757FF1F938767592A8488432E896B
:1008900015C5035745038357C4016311F702232687
:1008A000050223180502410597D00000E780209C2F
:1008B0006306090097800000E78060DB8144975958
:1008C000FF1F93892976130A800297B0FFFFE78004
:1008D000E0C263C4A4049757FF1F9387E75C9C435F
:1008E00099C70355C40197200000E780C0BD630786
:1008F0000900228597800000E780C0A01306400E03
:10090000814522859720FFFFE7806080FD57231EE9
:10091000F4001713FFFF6700237E3385440383A78A
:10092000C90A3E95035705008357C4016317F700B2
:10093000CA8597000000E78000E2850479B71713A5
:10094000FFFFE702237883C795004111AA8993F737
:10095000F707A384F5003285AE8497C0FFFFE780D8
:10096000C0B885676378F5042A8997400000E7805E
:10097000A091014401CD83D704003144638827014D
:10098000854597000000E78080EF01444E85A286F0
:100990004A86A68597D0FFFFE780609DA167938771
:1009A000170448003EC42302810002C697D0FFFF0F
:1009B000E780808A41011713FFFF6700E373171375
:1009C000FFFFE70223709757FF1F93872745804358
:1009D00029C4014597C00000E780002181470148F4
:1009E000C1641CDC232E0403232004041759FF1FB9
:1009F0001309496301449309400EFD1497B0FFFFAA
:100A0000E780C0AE634FA400814517F5FFFF1305D3
:100A1000857F97A0FFFFE780801C1713FFFF67000B
:100A2000A36D330534038327090B3E958357C50116
:100A300063879700854597000000E78040E4050440
:100A400075BF9357050113D78700A380F50093174F
:100A50000501C183A1832380E5002381F500A381E3
:100A6000A50082801713FFFFE702636723000500DC
:100A700083C71500A300F50083C725002301F500F7
:100A800083C73500A301F50083C745002302F500A5
:100A900083C75500A302F50083C765009305950041
:100AA000A30305002303F500230405003285970006
:100AB0000000E78040F91713FFFF670083641713F6
:100AC000FFFFE70223604111E9540DCD85CD93F975
:100AD000C5FF2E842A89AA84338AA900B7EA0400B4
:100AE00063189A020D88854411CCB7E704009C5F17
:100AF00082972AC622866C003305390197E00000F0
:100B0000E7800046268541011713FFFF6700C35E9B
:100B100083A78A039104829793170501C183A18358
:100B2000A38EF4FE93570501238FF4FEA183238E39
:100B3000A4FEA38FF4FE6DB763E6D5021713FFFF83
:100B4000E702E359B28741113686BE8536C697E083
:100B50000000E780E040B246410136851713FFFFF1
:100B60006700235A81463685828083870500138774
:100B7000F5003D05FD8793F77708834607007D154F
:100B80008606B58FA300F5006307B7007D1783477E
:100B900017009D83DDB782801713FFFFE702235400
:100BA000B7E7040083A7070932872A863A85829728
:100BB000133515001713FFFF6700A35415C18147B4
:100BC0008DC11713FFFFE7028351414697E00000F4
:100BD000E780003985473E851713FFFF67006352A2
:100BE00081473E8582801DCD1713FFFFE702234F0B
:100BF000414681452A849710FFFFE78040514146D6
:100C00008145130504039710FFFFE780405001471B
:100C1000C1672322040438C87CC805451713FFFFA9
:100C20006700234E0145828081473DCDB5CD171326
:100C3000FFFFE702C34AB2842E891306800581456F
:100C40002A849710FFFFE780804CCA8524C426853C
:100C500097000000E780C0F6414681452285971045
:100C6000FFFFE780C04A3044A2852285970000003C
:100C7000E780C0F293040401A28526859700000056
:100C8000E780E0EEA6851305040297000000E780E8
:100C900000EE228597000000E78020F585473E851D
:100CA0001713FFFF6700E3453E8582801713FFFFA0
:100CB000E70243414111E9540DCD85CD93F9C5FFBC
:100CC0002E842A89AA84338AA900B7EA040063988B
:100CD00044030D88814411CCB7E704009C5F8297E0
:100CE0002AC622866C003305390197E00000E780B0
:100CF0002027268541011713FFFF6700E33F83A7E5
:100D00008A039104829793170501C183A183A38E5F
:100D1000F4FE93570501238FF4FEA183238EA4FED6
:100D2000A38FF4FE6DB765CD1713FFFFE70283397C
:100D3000B28411E605451713FFFF6700E33B2A84E1
:100D40002E890145EDD93C487848B3E6E700E5D661
:100D50009386F7FFB3B7F6007D17032A4404BA97CA
:100D600034C87CC863050A06C14913050A03B38960
:100D700049412295637D3601B2862E86A68597006D
:100D80000000E780A0DB7C40BE9464C065B7CE86DF
:100D90002E86CE8597000000E78040DAC114D294F9
:100DA0004E9923220404A2879306040103C7070077
:100DB00003C607038507318FA38FE7FEE398F6FE8E
:100DC0003044A285228597000000E78020DD269927
:100DD000C1493306994063EC9900A9DCA686A68533
:100DE0001305040397000000E78040D579BF8147D1
:100DF000B306F4003307F6000347070083C5060077
:100E000085072D8F2380E600E39437FF3044A285C9
:100E1000228597000000E78060D8C1145DBF0145BE
:100E200082800DC11713FFFFE702632B13068005B5
:100E300081459710FFFFE780802D05451713FFFFC1
:100E40006700232C01458280814749C5C1C517131E
:100E5000FFFFE702C328FC4141462E84AA84639920
:100E6000C70413860501A2878146C14503C7070051
:100E700003C507038507298F3305D6000345050001
:100E80008506298FA38FE7FEE392B6FE3044A28544
:100E9000268597000000E78060D02285970000003B
:100EA000E78060F885473E851713FFFF67006325DD
:100EB000138507031D8E814522959710FFFFE7805C
:100EC00000257C40130700F813060402A29723882C
:100ED000E70251BF3E8582801713FFFFE702232000
:100EE0006D712E84B284AA859010280036899700EF
:100EF0000000E780A0D309EDD55725A050400C4055
:100F0000280097000000E78040E27DD5FD14210411
:100F1000F5F42C004A8597000000E78020F3814714
:100F200061DD3E8551611713FFFF6700831D1713B5
:100F3000FFFFE702C31A41112EC432C62C0005463A
:100F400097000000E78080F941011713FFFF670059
:100F5000431B1713FFFFE702831801112A842EC6D3
:100F600002C802CA02CC02CE97E00000E780C0238C
:100F7000B2462A86A285080897000000E78060FB39
:100F80001375F50F05611713FFFF6700831717131C
:100F9000FFFFE702C3147971B2872A842146230830
:100FA000B10013051101BE853AC436C697E00000B2
:100FB000E78000FBB246930591013685970000005B
:100FC000E78060A82285141035460C0897000000C1
:100FD000E78020F62A84224701E921460C103A8551
:100FE00097E00000E780C0F7228545611713FFFFF7
:100FF000670023111713FFFFE702630E7171AE84C0
:10100000AA850A85328497000000E78060BB11C979
:101010000A86A685228597000000E78020B88147D0
:1010200011E1C5473E854D611713FFFF6700630D52
:101030001713FFFFE702A3071D712A8AB289BE8436
:1010400035468547130511012E8CB68A3A8BC28C22
:10105000468D2308F10097E00000E78060F0101053
:101060000C085285231F010097000000E780C0F89C
:101070002A843DEDA1476313FD089307900591E095
:10108000E5473546E2851305110113990A01230846
:10109000F1001359090197E00000E78060EC135755
:1010A000890093978A00D98F90080C085285231FD6
:1010B000F10097000000E78020F42A8415E9A1E4FC
:1010C0009387FA0091831379F9003EC663130900F0
:1010D0004149668B8144C14B854DB247639F970C54
:1010E0006A868C0033855C0197E00000E78040E76A
:1010F000228525611713FFFF670023FF93079004E4
:10110000C9F0A547BDBF834701050947C14B230867
:10111000F10083471105A58FA308F10093872400F0
:10112000814463E1FB04014714083386E6008C0820
:10113000B386E400BA95DA9683C6060083C5050037
:101140000507AD8E2300D600E390E7FE4147639C80
:10115000E70490080C08528597000000E780C0E97A
:1011600025D181A0B3069B00BA871008B305F6000D
:1011700090083E9603C506000346060085078506CF
:10118000298E2380C500E39277FF998F90080C0881
:101190005285BE9497000000E78000E6894701472A
:1011A00049D12A84B1B790083E9603460600140838
:1011B000BE962380C600850759BFB2478504638762
:1011C000971481471808B306F70098083E973386AE
:1011D000F90003470700034606008507318F238087
:1011E000E600E39177FF90080C0852859700000015
:1011F000E78080E05DF53546E2851305110123089F
:10120000B10197E00000E780A0D513970401418366
:10121000939784002183D98F10180C085285231FBF
:10122000F10097000000E78020DD25FD81471018C0
:101230003387F9003E960347070003460600B306CE
:10124000FB008507318F2380E600E39277FF65A8D6
:101250001808B306F70098083E973386F90003474D
:101260000700034606008507318F2380E600E3E18F
:1012700027FFCA87639E770990080C08528597005C
:101280000000E78060D711FD81479800B306F700A2
:10129000900818103E973E96034707000346060045
:1012A0008507318F2380E600E39177FF3546E2859D
:1012B000130511012308B10197E00000E78040CA3F
:1012C000139704014183939784002183D98F1018C9
:1012D0000C085285231FF10097000000E780C0D161
:1012E000E31105EC814710183387F9003E96034758
:1012F000070003460600B306FB008507318F2380F5
:10130000E600E3E227FFC109410BC1BB814785B776
:101310009408BE9683C6060018083E972300D7009F
:10132000850789BF638006321713FFFFE70223D8C2
:1013300059712A84BE89B28B85473546130511023F
:101340002E8B468C4289BA8A368A2300F10297E0B6
:101350000000E780E0C010180C102285231701025E
:1013600097000000E78040C963180512A147631F7A
:10137000FC069307900563930900E5473546DA8537
:101380001305110293140A012300F102C18097E0B2
:101390000000E780E0BC93178A0013D78400D98F40
:1013A00090080C1022852317F10297000000E780B7
:1013B000A0C47DE1639209049307FA00BD8891837C
:1013C00091E0C144C207C183DE8C814A3EC6414DD3
:1013D000B24763E2FA0E6286B3854B01881097E04C
:1013E0000000E78080B54DC93D557DA0930790046E
:1013F000E39609F8A54759B7834701050947C14C4A
:101400002300F10283471105B3C7F900A300F102DD
:1014100093872900814963E1FC0481461810330653
:10142000D7008C083387D900B69556970347070035
:1014300083C5050085062D8F2300E600E390D7FEC7
:1014400041476390E70690080C1022859700000042
:10145000E78080BA35D189A0B3863A01BA871010E7
:10146000B305F60090083E9603C506000346060045
:1014700085078506298E2380C500E39297FF338771
:10148000EC4090080C102285BA9997000000E78084
:10149000A0B68947014741D165611713FFFF670077
:1014A000C3C490083E96034606001410BE962380DF
:1014B000C600850779B7B247850A93990A01939DBB
:1014C0008A0093D909016391570F85473546DA851C
:1014D000130511022300F10293D9890097E000005F
:1014E000E78000A8B3ED3D0190000C102285231782
:1014F000B10397000000E78020B059FD8147A6891D
:1015000063EA970626860C084A8597E00000E78084
:1015100020A581471810B306F700100898083E97D9
:101520003E9603470700034606008507318F238058
:10153000E600E3E197FE639FA90590080C10228561
:1015400097000000E78040AB21F981479810B3066F
:10155000F700900818183E973E9603470700034689
:1015600006008507318F2380E600E391A7FF41093C
:10157000C10CB9BD18089000B306F7003E9633873A
:10158000FC0003470700034606008507318F2380D0
:10159000E600B5B798084E97034707001C10CE9792
:1015A0002380E700850941BF85473546DA85130565
:1015B00011022300F10293D9890097E00000E7802F
:1015C000209AB3ED3D0190000C1022852317B10342
:1015D00097000000E78040A2E31005EC814718085F
:1015E0009000B306F7003E963387FC0003470700E0
:1015F000034606008507318F2380E600E391A7FFAD
:1016000041460C084A8597E00000E78060958147D5
:101610001810B306F700100898083E973E96034747
:101620000700034606008507318F2380E600E3911B
:10163000A7FF90080C10228597000000E780C09B50
:101640001DD599BD7D5582801713FFFFE70223A9A1
:1016500001112A842E8593055100328902C002C2ED
:1016600002C402C69304740097F0FFFFE780A03D18
:101670001D46A6851305910097E00000E780408E87
:1016800010088A854A8597000000E780E09619EDEA
:1016900093071400180883C6070003460700850750
:1016A0000507B18EA38FD7FEE397F4FE05611713EC
:1016B000FFFF670003A51713FFFFE702A3A02E8417
:1016C0008C414111AA89838715003289914463D3E3
:1016D0000700A1449757FF1F938787CB9C43A1C75F
:1016E000C1CA8D472310F10083C725004A85230115
:1016F000F10083C73500A301F10083C74500230231
:10170000F10083C75500A302F10083C7650093056C
:101710009100A30301002303F1002304010097F0CB
:10172000FFFFE78040320C404A860A8597F0FFFFB2
:10173000E78080330328040083564400A6881D08F0
:1017400081470147E51642868A854E85970000004D
:10175000E780408E2A8919E5A685228597B0FFFF8C
:10176000E780A0C24A8541011713FFFF6700C398B5
:101770004A860A8597F0FFFFE780002F6DB71713A1
:10178000FFFFE70223942E848C414111AA898387AD
:1017900015003289914463D30700A1449757FF1F76
:1017A000938707BF9C43A1C7C1C68D472310F10093
:1017B00083C725004A852301F10083C73500A301B3
:1017C000F10083C745002302F10083C75500A3023F
:1017D000F10083C7650093059100A3030100230373
:1017E000F1002304010097F0FFFFE780C0250C40C3
:1017F0004A860A8597F0FFFFE7800027835644005A
:10180000032804008A85858EC2061D08C182231222
:10181000D400A68881470147E51642864E85970089
:101820000000E78060B041011713FFFF6700C38C21
:101830004A860A8597F0FFFFE78000234DBF171304
:10184000FFFFE702C389B335B000011185052A897E
:101850001315F601336515012308B1009305110135
:1018600036843AC632C03EC442C297F0FFFFE780DA
:10187000801DA2471248425593D68700230BF100E2
:101880009305910193578800A30AD100A30BF1009F
:10189000230C010197F0FFFFE780E01A3247024670
:1018A00003280400B337E0008356440092079144B4
:1018B00011C2A1444A85A68842860C0897F0FFFF12
:1018C000E78040772A8919E5A685228597B0FFFF32
:1018D000E780A0AB4A8505611713FFFF67006382AD
:1018E0001703FFFFE702037E01113EC68647B335AB
:1018F000B0008505AA891315F6015D8D2308B10096
:101900009305110136843A89B28442C446C297F0E5
:10191000FFFFE780401322489248164593578800FE
:10192000A30AF1009305910193D78800230B0101CD
:10193000A30BF100230C110197F0FFFFE780A0102B
:101940003247104083564400B337E0009207032823
:101950000900914891C0A1480C084E8597000000ED
:10196000E780809CAA8401E9835544004A8597B0AA
:10197000FFFFE78080A1268505611703FFFF670051
:10198000A377AA959307F00F170701001307876144
:101990006317B50013C5F7FF1375F50F82800505B2
:1019A0008346F5FFB58FBA9783C70700D5B70357AE
:1019B000450014419307F00F170601001306865ED9
:1019C000369742074183139506014181631BE50069
:1019D000AD8FB29703C50700130515F31335150036
:1019E0008280850603C5F6FFA98FB29783C70700DB
:1019F000D9BF1703FFFFE702836EB28736842E86B6
:101A0000BA86AA853E85BA8497F0FFFFE7806052C8
:101A1000634F0500228597D00000E780E0782A8692
:101A2000A686A285268597F0FFFFE78080501703E2
:101A3000FFFF6700036D1703FFFFE702A3685D71F7
:101A40002A8BAE8A17050100130545532C00B2847A
:101A5000368ABA893E8997F0FFFFE780C04F2A8413
:101A60005DE134104146DA85280097F0FFFFE780FA
:101A7000404C2A8449E98547A303F100A6C2930795
:101A800071002408BEC4A68685470D462C18281070
:101A900002DC02DED6C0BEC697F0FFFFE78000443E
:101AA0002A8435E183477102A6860D4693F7F7072E
:101AB0002300FA00C1473EDE2C188947281026DC97
:101AC000A303F10097F0FFFFE78040412A8405ED72
:101AD0004146A6854E8597D00000E78060488D4737
:101AE000A6860D462C182810A303F10097F0FFFFDF
:101AF000E780C03E2A8401E94146A6854A8597D001
:101B00000000E780E045228561611703FFFF670061
:101B1000A35E1703FFFFE702835C97F7000093873C
:101B2000E7A1984383C7470079712A89AE841705D6
:101B30000100130525450C083AC42306F10097F06F
:101B4000FFFFE78040412A8405ED14104146CA8515
:101B5000080897F0FFFFE780C03D2A8415E11408CC
:101B600015462C00081097F0FFFFE780803C2A8480
:101B700001E921462C08268597D00000E780403EE9
:101B8000228545611703FFFF6700A3571703FFFF77
:101B9000E702E35497F700009387479A9C477971CF
:101BA000AA842E84170501001305453E0C083EC685
:101BB00097F0FFFFE780203A0DE914104146A68513
:101BC000080897F0FFFFE780C03605E114081146CA
:101BD0006C00081097F0FFFFE780A03519E58347F8
:101BE000F10193F7F7032300F40045611703FFFFAA
:101BF000670023511703FFFFE702634E3688A148B1
:101C000081470147E54697F0FFFFE780A0421703B1
:101C1000FFFF6700034F1703FFFFE702434C3688BF
:101C2000A14881470147E54697F0FFFFE780C06F75
:101C30001703FFFF6700E34C1703FFFFE702234A88
:101C400001112A842E850C0832C697F0FFFFE78029
:101C5000803009ED3247970601009386A6311008BF
:101C6000C145228597000000E780E0D80561170391
:101C7000FFFF670003491703FFFFE70243464111D7
:101C8000C1472EC032C48A8509463EC23EC697F07F
:101C9000FFFFE780A02441011703FFFF67006346B1
:101CA0001703FFFFE702A3434111AE861306100995
:101CB000AA850A8502C002C202C402C697F0FFFFCD
:101CC000E780202741011703FFFF670083431703C5
:101CD000FFFFE702C3403287970601009386862BF9
:101CE0002E869305000297000000E780C0D01703FE
:101CF000FFFF670003411703FFFFE702433E7971CF
:101D0000C1472ACC2ED032D42C080D4628003ECE16
:101D10003ED23ED602C402C602C802CA97F0FFFFF6
:101D2000E780C01B45611703FFFF6700833D170372
:101D3000FFFFE702C33A0111AA842E8417050100B0
:101D40001305C5258A8597F0FFFFE780C02015E5BC
:101D500014084146A6850A8597F0FFFFE780601DBD
:101D600009ED8347E1010347F101A207D98FCA07B3
:101D7000C9836177D98F2310F40005611703FFFF32
:101D80006700233815CD1703FFFFE7024335974758
:101D9000FF1F9387670D90439745FF1F9385050DA0
:101DA0001745FF1F1305450897D00000E78000C5C1
:101DB0001745FF1F130545071703FFFF670063342F
:101DC0001745FF1F1305450682808DCD1703FFFFC2
:101DD000E702E3309747FF1F9387070994430111F8
:101DE0002E840A869745FF1F9385450897D00000EB
:101DF000E78040C60A850294014505611703FFFF8D
:101E0000670023307D5582801703FFFFE702232DF3
:101E100097D00000E78080D19747FF1F23A6A70433
:101E200017F5FFFF1305E5C997B00000E780C07400
:101E30001703FFFF6700E32C1747FF1F1307070572
:101E40009317150008433E95FD572310F500828037
:101E50001703FFFFE702A3282A84084009E51703B8
:101E6000FFFF6700032A1C4158401CC06313E500B4
:101E70005CC08347550023200500F99BA302F500B1
:101E800097A0FFFFE780E07CC9BF1703FFFFE702D1
:101E900063239747FF1F9387670198432A8411CBD9
:101EA0008347350093F7070289C703550500894525
:101EB00002971305440197B00000E780403B83552B
:101EC00004000355E40097300000E780A00C485858
:101ED00019C597A0FFFFE780C077232A04021305E6
:101EE000840397000000E780E0F68144B1499790B1
:101EF000FFFFE780E06A63CBA4028347340023201E
:101F0000040493F727FCA301F40000489790FFFF17
:101F1000E780006A13161500814522859700FFFFB0
:101F2000E780E01E1703FFFF6700031DB38734033C
:101F30000329040385043E994A8597000000E78041
:101F400060F12304090065B78347350093F7070262
:101F500099E3014582808357E500E39CB7FEC167A2
:101F6000FD176316F60005458280054599A81703FD
:101F7000FFFFE702C31693170601C187B2842A84C4
:101F800001496359F002835705009DCB0145636702
:101F9000F600034584003E953325A6001375F50F22
:101FA0000DA01C4813171900BA9783D70700E38EBA
:101FB00097FA05099790FFFFE780805FE343A9FE4A
:101FC00001451703FFFF6700C3131703FFFFE70275
:101FD000630FAE89AA849790FFFFE78020532A847D
:101FE00097D0FFFFE780A02EAA8601471306840141
:101FF00097050000938585E41745FF1F130545E904
:102000009790FFFFE780A0192A8925C98C44130403
:10201000C50022859E0593F5050897A0FFFFE78080
:10202000003DCC4083877400E18163DD070493E5C4
:102030000508228597A0FFFFE780603B0D4693854A
:102040004400228597A0FFFFE780803783D50400F6
:10205000228597A0FFFFE780A03E83D5240022853C
:1020600097A0FFFFE780C03D03D6490083A5090084
:10207000228597A0FFFFE780A0344A851703FFFF62
:102080006700830793F5F5076DB71703FFFFE702B6
:10209000030501112A84328532C697A0FFFFE7802D
:1020A000A0289780FFFFE7808031835704001747FF
:1020B000FF1F130727F73246231BF100930700F891
:1020C000A30DF1001C471843231AA1008983858BB7
:1020D000B307F740B28548083ECE231C0100230D0C
:1020E000010097000000E78080EE05611703FFFF05
:1020F000670023011703FFFFE702C3FC004101450E
:102100003DC49304C40026853289AE8997A0FFFFA1
:10211000E780802595452A8A2685035B040197A0E0
:10212000FFFFE780E021268597A0FFFFE780203FA3
:102130008D45AA8A268597A0FFFFE7806020268527
:1021400097A0FFFFE780A03D5C48420A135A0A01AE
:10215000D2975CC423186401814763983A0146050D
:102160004D81330625419337160013F5F70F1703FA
:10217000FFFF670063F81703FFFFE702C3F38969F6
:102180002A8BAE8B328AB68A81440144314CFD19C8
:102190009790FFFFE780C04063CDA4009790FFFFBA
:1021A000E7800043018D33B5AA001703FFFF6700E6
:1021B00003F43389840383270B003E9963170A00D5
:1021C0008347890085043E94E1B703560A00DE8503
:1021D0004A8533F6C90097000000E780E0F16DD131
:1021E0000545E1B71703FFFFE70263EF01112A84FA
:1021F0007C000355E5003ECAB70707003ECC7C00D3
:102200003ECE97200000E78020082A8985454808AF
:1022100097A0FFFFE780E0399945480897A0FFFFA6
:10222000E780A016AA844A8597200000E780A008CE
:102230002380A4009747FF1F9387C7DE9C43416616
:10224000130606F09396870113D78701558F93D60F
:102250008700F18E558FA207B706FF00F58FD98F43
:1022600011462C00138514003EC497D00000E7806F
:1022700020CF5008A38204008945228597000000E2
:10228000E780E0E019C9AA851305840397A0FFFF42
:10229000E780A0323C4085073CC005611703FFFF83
:1022A000670023E61703FFFFE70263E39790FFFF52
:1022B000E78000322A8405049790FFFFE7804030D2
:1022C0003305A402F14791453305F502972000003C
:1022D000E78020BA11E565551703FFFF670063E249
:1022E0009747FF1F23ACA7BA9790FFFFE780402EC8
:1022F0002A8405049790FFFFE780802C3305A40211
:102300008945060597200000E780A0B669D5974764
:10231000FF1F23ADA7B69790FFFFE780602B2A84AD
:1023200005049790FFFFE780A0293304A402974794
:10233000FF1F239F87B49790FFFFE78060292A84BF
:102340009790FFFFE780C027930714003385A7020B
:102350009747FF1F239FA7B2970701009387C7875F
:102360001747FF1F232AF7B20145BDB71703FFFF29
:10237000E70243D5AA842E8901449749FF1F938918
:1023800069CA130A80069790FFFFE78060236347BE
:10239000A40001451703FFFF670003D6330544037C
:1023A00083A709024A86A6853E9597000000E7802C
:1023B000E0B919E10504C1BF0545E9BF1703FFFFF7
:1023C000E70263CFAA8A2E8BB28B368C3A8A81447D
:1023D00001448149974CFF1F938CCCC4130D800698
:1023E0009790FFFFE780C01D63C9A40011E08549F5
:1023F0004E851703FFFF670083CF3389A40383A7AC
:102400000C025E86D6853E994A8597000000E780DB
:10241000E0B31DC19790FFFFE780801B0544636D0B
:102420004501D2866286DA8513050903970000000C
:10243000E780A0D411C1854985045DB71703FFFF6C
:10244000E70243C8C16441112A8901449749FF1F2B
:10245000938949BD130A8006FD1436C632C42EC2C4
:102460009790FFFFE780C01592452246B246634829
:10247000A400014541011703FFFF6700E3C73305CF
:10248000440383A709023E9509C683473500C18BE3
:102490009DC791C68347350093F707028DC3630636
:1024A00099008357E500639C27010357050001CB82
:1024B00063E7E50083478500BA97E3CDF5FA0504A5
:1024C00069BF1703FFFFE702E3BFC1642A89014424
:1024D0009749FF1F938909B5130A8006FD14979049
:1024E000FFFFE780E00D6346A4001703FFFF6700CE
:1024F000A3C03305440383A709023E958357E50033
:10250000638A97006304990063962701970000008F
:10251000E780E0970504E1B71703FFFFE70223B95F
:1025200089692A8AAE8A328BB68B8144174CFF1F89
:10253000130C4CAF930C8006314DFD199790FFFFA3
:10254000E780000863C6A4001703FFFF6700E3B934
:102550003389940383270C028355CA015A863E9916
:102560004A8597000000E780609E31C1814D15A02B
:102570003384AD038327090303D60B00D68533F6D6
:10258000C9003E94228597000000E780E0B609E983
:10259000850D9790FFFFE780A000E3CBADFC01A87D
:1025A000228597000000E780E08A23040400850468
:1025B00071B71703FFFFE70203B04169AA8A014A16
:1025C000174BFF1F130B0BA67D19C14B054C9790A2
:1025D000FFFFE780E0FE6346AA001703FFFF6700E6
:1025E00003B193098006B3073A0383290B02BE990E
:1025F00083D7E900638E270163842A01639A570118
:1026000003A4890301E84E8597000000E780C0BD60
:10261000050A75BF83570401639977099304C400C1
:10262000268597A0FFFFE78020D485452A8D268543
:10263000835C040197A0FFFFE78080D0268597A0E8
:10264000FFFFE78060E862056185635905048D45F9
:10265000268597A0FFFFE780A0CE8945268597A015
:10266000FFFFE780E0CD8945268597A0FFFFE78043
:1026700020CD8545268597A0FFFFE780A0CD834725
:102680000500094793F7F707639AE7009945268500
:1026900097A0FFFFE78000CCA30285014848337D67
:1026A0002D01231894016A9548C40040A1BF170367
:1026B000FFFFE702C3A237E404008327041D8297CB
:1026C0009747FF1F83C707831715FF1F130505E6ED
:1026D000A300F5008327441C82978327841C81462E
:1026E0001306F00F8145014582971703FFFF67002E
:1026F00043A11737FF1F1307E76F18439735FF1FD5
:1027000083C5457F9737FF1F9387477D83468703A0
:10271000034697036397D5009737FF1F238CC77C29
:10272000828083C587010347A7036317B6009737E5
:10273000FF1F2381E77C828003C687016317C700E0
:102740009737FF1F2388D77A828083C687011307B4
:1027500050026319D700930760021737FF1F230B3E
:10276000F778828083C68701130660026315D6005E
:1027700093077002DDB783C7870155BF9737FF1FE7
:102780009387C775D44B0947638DE6081703FFFF8E
:10279000E702E3941739FF1F130989713E848347C9
:1027A0000900918B9DCFB7E4040083A7041D829795
:1027B00083A7441C1735FF1F13050570829783A755
:1027C000841C81461736FF1F03460671814501456B
:1027D000829721C583470900ED9B1737FF1F230907
:1027E000F76C8347040093F7F70F85CB91471737B2
:1027F000FF1F232FF76E97000000E78080EB970004
:102800000000E78040EFB7E70400BC4F4146914528
:102810001735FF1F0345056D82971703FFFF6700FC
:10282000438E82801703FFFFE702638B8D474111C0
:102830006306F504C5476308F50285476310F50292
:102840009737FF1F238AA76AB7E70400BC4B93059D
:1028500000101735FF1F0345E568829741011703F4
:10286000FFFF6700038A85471737FF1F2306F768B6
:10287000B7E70400BC4B93050020E1BF9737FF1F6B
:102880009387C765D44B1147638DE600B7E7040013
:1028900083A7071D8297B7E70400BC4B930500048C
:1028A0004DBF05491737FF1F2324276583C707003E
:1028B00032C62E8493F7F70FD5D3B7E4040083A76D
:1028C000041D7D141374F40F8297E37689FCB245DE
:1028D000994703C61500E3F0C7FCFC440906173509
:1028E000FF1F1305A5618297BC48930500081735A3
:1028F000FF1F0345255F829779BF17F3FEFFE702AD
:10290000037E1737FF1F1307675D4047184B1C40B6
:102910009736FF1F23AAF65C6316E4001737FF1FE4
:102920002326F75C130584FE9790FFFFE78020A71E
:10293000035564FF9780FFFFE780A06F97A0FFFF1C
:10294000E78020D117F3FEFF6700A37B17F3FEFF9C
:10295000E702E3789737FF1F93874758D84BDC4748
:1029600089C797000000E78080F985471737FF1F68
:102970002320F7589737FF1F9387C7479C4393053A
:1029800000021735FF1F0345E55583C78703173737
:10299000FF1F2301F756B7E70400BC4B829717F3DC
:1029A000FEFF670003769737FF1F23ABA752828095
:1029B00017F3FEFFE702037137E404007C4CA145E6
:1029C0001735FF1F0345055282977C48A1451735EF
:1029D000FF1F034525519734FF1F9384245082978E
:1029E000DC4489EB97000000E78080D917F3FEFFF5
:1029F0006700837003D567FF9780FFFFE780606300
:102A0000AA896DD1D84891476310F7027C4C914553
:102A10001735FF1F0345054D82977C4891451735B3
:102A2000FF1F0345254C829703A9490103D40901DF
:102A30008947B7E904001737FF1F232BF74A83A7FD
:102A4000091D21044204829783C784011715FF1FC3
:102A50001305C5AD61191717FF1FA309F7AC83A7AD
:102A6000491C418082979737FF1F2387074883A718
:102A7000C91C814609469375F40F4A85829711E96E
:102A80009737FF1F83C7875789C79700FF1FE780C6
:102A90006016B7E70400BC4F2146A1451735FF1F5C
:102AA00003454544829799B717F3FEFFE702236376
:102AB00093F7052001112E8481CF97000000E78055
:102AC00020E913450420056117F3FEFF67006363E7
:102AD00093F70510A9CF9734FF1F93842440DC4857
:102AE00097000000E78020C11737FF1F13078730CA
:102AF000184383C78401034787036318F700DC4446
:102B000089C797000000E78080DF85471737FF1FE0
:102B10002320F73EB7E70400BC4B930500021735AE
:102B2000FF1F0345253C82971345041069BF93F7A7
:102B30000508BDC79737FF1F83C7573CE9171946DC
:102B40009735FF1F9385A53B1305D10093F4F70F2D
:102B50001739FF1F0349893A97C00000E7804040BA
:102B600093970401C1831737FF1F1307A739231D4C
:102B7000F100231CF1009737FF1F938727363ACEC9
:102B80003ACAD8432306010009CBDC4393158901D7
:102B900054080D46E185680082971345040825B75F
:102BA00093F72500A5C39737FF1F93872733D84B8B
:102BB00089476306F7029737FF1F83C7672F13F70D
:102BC000270011EF918B99CFB7E70400BC4F130694
:102BD000000A89451735FF1F0345C5308297134505
:102BE0002400D5B59737FF1F9387C7209C4383C721
:102BF00087031737FF1F230FF72E97000000E7808A
